:020000040000FA
:100000000020040000000000C2000100C200010046
:10001000C2000100C2000100C2000100C2000100D4
:10002000C2000100C2000100C2000100C2000100C4
:10003000C2000100C2000100C2000100C2000100B4
:10004000C2000100C2000100C2000100C2000100A4
:10005000C2000100C2000100C200010056FF000002
:10006000C2000100C2000100C2000100C200010084
:10007000C2000100C2000100C2000100C200010074
:10008000C2000100C2000100C2000100C200010064
:10009000C2000100C2000100C2000100C200010054
:1000A000C2000100C2000100C2000100C200010044
:1000B000C2000100C2000100C2000100C200010034
:1000C000C2000100C2000100C2000100C200010024
:1000D000C2000100C2000100C2000100C200010014
:1000E000C2000100C2000100C2000100C200010004
:1000F000C2000100C2000100C2000100C2000100F4
:10010000C2000100C2000100C2000100C2000100E3
:10011000C2000100C2000100C2000100C2000100D3
:10012000C2000100C2000100C2000100C2000100C3
:10013000C2000100C2000100C2000100C2000100B3
:10014000C2000100C2000100C2000100C2000100A3
:10015000C2000100C2000100C2000100C200010093
:10016000C2000100C2000100C2000100C200010083
:10017000C2000100C2000100C2000100C200010073
:10018000D2FC0000C2000100C2000100C200010058
:10019000C2000100C2000100C2000100C200010053
:1001A000C2000100C2000100C2000100C200010043
:1001B000C2000100C2000100C2000100C200010033
:1001C000C2000100C2000100C2000100C200010023
:1001D000C2000100C2000100C2000100C200010013
:1001E000C2000100C2000100C2000100C200010003
:1001F000C2000100C2000100C2000100C2000100F3
:10020000FFFFFF00FFFFFF00C2000100C20001006E
:10021000C2000100C2000100C2000100C2000100D2
:10022000C2000100C2000100C2000100C2000100C2
:10023000C2000100C2000100C2000100C2000100B2
:10024000C2000100C2000100C2000100C2000100A2
:10025000C2000100C2000100C200010056FF000000
:10026000C2000100C2000100C2000100C200010082
:10027000C2000100C2000100C2000100C200010072
:10028000C2000100C2000100C2000100C200010062
:10029000C2000100C2000100C2000100C200010052
:1002A000C2000100C2000100C2000100C200010042
:1002B000C2000100C2000100C2000100C200010032
:1002C000C2000100C2000100C2000100C200010022
:1002D000C2000100C2000100C2000100C200010012
:1002E000C2000100C2000100C2000100C200010002
:1002F000C2000100C2000100C2000100C2000100F2
:10030000C2000100C2000100C2000100C2000100E1
:10031000C2000100C2000100C2000100C2000100D1
:10032000C2000100C2000100C2000100C2000100C1
:10033000C2000100C2000100C2000100C2000100B1
:10034000C2000100C2000100C2000100C2000100A1
:10035000C2000100C2000100C2000100C200010091
:10036000C2000100C2000100C2000100C200010081
:10037000C2000100C2000100C2000100C200010071
:10038000D2FC0000C2000100C2000100C200010056
:10039000C2000100C2000100C2000100C200010051
:1003A000C2000100C2000100C2000100C200010041
:1003B000C2000100C2000100C2000100C200010031
:1003C000C2000100C2000100C2000100C200010021
:10400000EF6423000E7F24000E01880000000000F2
:104010000C00070060AB2E0001002000110007001B
:10402000000020000000E00002003200000002005A
:1040300000000000FCFB0200000000000040DA006D
:104040000000FE004440A900604020000000E000A5
:104050000300320000002000A00188004440A800B6
:104060000000060091018800800078000000EB004D
:1040700015003700E280400032A0B4009101BA0080
:10408000E280400032A0B4009102BA00E280400019
:1040900032A0B4000002EB00472BDE00F507B200AF
:1040A000602CE10004003A000059EB008301E900B4
:1040B000FDFF3E00040037006128E10001003200EE
:1040C0000082EB00040007001101BA000200E000CA
:1040D000E8FF3A00000006003159BA008301E90008
:1040E0000C0032002159BA008301E90008003200B7
:1040F0000400E00003003A00E280400032A0B40077
:10410000F5FF370011D9BA008301E900FAFF3A0040
:104110008100E800E180400032A0B4000000060009
:1041200046CE04000000000078FF040000000000FC
:104130008AFF040000000000A0FF0400000000004F
:10414000B4FF040000000000C8FF040000000000ED
:10415000DCFF040000000000F0FF0400000000008D
:10416000FEFF04000000000062B304000000000035
:10417000FAAF040000000000ECAF040000000000F3
:1041800046B004000000000032B00400000000004F
:1041900026B004000000000018B004000000000079
:1041A0000AB004000000000072B00400000000002B
:1041B0005AB004000000000054B3040000000000E6
:1041C000068C040000000000288C040000000000A1
:1041D000E486040000000000848604000000000063
:1041E000448C040000000000FC8A04000000000071
:1041F0008C87040000000000F28A04000000000028
:10420000C28C040000000000F486040000000000DE
:104210000A9E0400000000006A9E040000000000E6
:104220008C9D0400000000003A9D04000000000086
:10423000CE9F040000000000DE9E0400000000008D
:10424000BA9F04000000000072A1040000000000FA
:10425000B09E040000000000867A04000000000008
:10426000507A040000000000BC7A04000000000046
:10427000F67A040000000000EA7A04000000000062
:10428000BE7D040000000000987B040000000000D8
:10429000B67D040000000000B47E040000000000B1
:1042A0001A7B040000000000BADC040000000000DB
:1042B000D4DC040000000000AADC040000000000C0
:1042C000A0DC04000000000012DD0400000000007B
:1042D00006DD04000000000036DD040000000000E0
:1042E0002ADD040000000000FADC040000000000E9
:1042F0001EDD040000000000EEDC040000000000F1
:1043000038DE04000000000078DD0400000000003A
:1043100070DE04000000000042DD04000000000028
:1043200084F104000000000046F1040000000000D9
:10433000C2F104000000000020F1040000000000B1
:1043400014F104000000000024F20400000000004A
:1043500030F20400000000003CF204000000000005
:1043600048F20400000000000CF20400000000000D
:1043700018F204000000000000F204000000000039
:1043800098F2040000000000BEF3040000000000EA
:1043900054F2040000000000CAD80400000000002D
:1043A000BAD804000000000000D90400000000009A
:1043B000AAD804000000000038EE0400000000004D
:1043C0004CEE04000000000020EE0400000000009D
:1043D000B4EE0400000000005EEE040000000000E7
:1043E000667F0400000000001EF0040000000000D2
:1043F0002AB90400000000005AB9040000000000BF
:1044000084BA04000000000078B904000000000035
:1044100066BC04000000000048B804000000000072
:104420001CB90400000000000EBD040000000000E4
:1044300096000400010000008E000400010000004E
:104440008800040001000000D05C040000000000AF
:1044500092CB04000000000070CC040000000000BB
:1044600062CC040000000000F0CC0400000000005A
:10447000E2CC04000000000046AF04000000000091
:1044800076AF040000000000D873040000000000B4
:10449000E873040000000000FE7304000000000048
:1044A000067504000000000076750400000000009E
:1044B000C6730400000000009875040000000000AE
:1044C000AA75040000000000F2750400000000005E
:1044D0005E7604000000000080760400000000000A
:1044E000C4770400000000002678040000000000EB
:1044F0009878040000000000BC7804000000000070
:1045000080740400000000001E7904000000000018
:104510003C79040000000000889FBE008A9FBE0016
:10452000010578000100E0000400350008003C00AF
:104530000000E0002000320005003700600010009D
:10454000E080180002003B0001F02C001A00370048
:104550000004BE006011B8006B0920000982CF0082
:10456000020039000882CF000441B00069425200C5
:104570000E00320008003B0082817100610164007E
:104580008904D1000884D3008B05E8000442E800C8
:10459000F9FF3A00050037000804440089844C0004
:1045A0008B05E9000442E900FBFF3A001A0107000D
:1045B0000AF0A70001F0A0004F05BE004F04BE00A6
:1045C00000000600F4FF2F0039013700140020001E
:1045D00037013700889FBE008A9FBE008C1F78007D
:1045E0004E0107005501330003866C006450E10062
:1045F0002E0032006420E100330032006150E100FF
:104600002F0032006120E100310032008585550025
:10461000EB07B00009002000080420000500370067
:104620000804440089844C000A003100060343005A
:1046300087834B000001530081815B00F8FF33004A
:104640000203BE000800A0000804440089844C0056
:10465000F6FF3900C639DD00830173000100320026
:10466000130020008904D1000884D3000998A30016
:10467000050032000800A7000300A0008904D10053
:104680000884D3008B05E8008904D1000884D30096
:104690000001EB000281D200DF00070001F0A10061
:1046A0000CF0A70001F0A0002D0137006420E1000C
:1046B0002F0132000801BE000200BE00F7FF3700E4
:1046C0006120E1002A0132006000B800F3FF3700EA
:1046D0000000200001F82700F0FF370003F0A200DF
:1046E000889FBE008A9FBE008C1F78000B010700C8
:1046F000120133006450E1004F0032006420E100F9
:104700005200320003826C0007003B000905D00014
:104710000306D000820F54000C065D000200390031
:104720000200320089017800030678008582550076
:1047300004003D000003FD008103FD008502EA0046
:104740008B854200840F720002003B006000100065
:10475000E08018006011B8000005EB007A28E10045
:104760000A00390006007800C75DDD00F707B200D7
:10477000878075002D003700828171000A01780062
:10478000610560008180D1000080D3008502E900CE
:10479000F9FF3B00060440008784480002003B000C
:1047A00060041400E0841C000988A30007003200A4
:1047B0008A81710082817100610164008904D100E5
:1047C0000884D3008B05E800170037000978A300A0
:1047D00013003A000B00E000130034008B05E900E1
:1047E0000804440089844C000A4474000978A3003A
:1047F0000D003A000B00E000070034008B05E900D3
:104800000804440089844C0001003A000B00200099
:104810000978A300F7FF32000001EB000200370027
:10482000828171000A0178007B0007000CF0A7006C
:1048300001F0A000CA0037006420E10002003A0045
:10484000838F6C00CA0033000801BE000200BE0066
:10485000C3003700889FBE008A9FBE008C1F78006F
:10486000AE000700B500330003866C006450E10021
:10487000240032006420E100270032006150E10092
:10488000220032006120E100210032008B854200CD
:10489000EB07B1000134B800003AB8000804420048
:1048A00089844A00013AB8000030B800888040008E
:1048B00009014A00040033000000400081804800E4
:1048C000020149008B05E900C909DD008301700080
:1048D0000100320013002000C814DE004814DD007F
:1048E0004709DE001200B200C808DE00088470002C
:1048F0004900070001F0A1000CF0A70001F0A000A2
:10490000970037006120E100990032000801BE00E5
:104910000200BE00F7FF37006150E100FCFF3A00E3
:10492000930037000001BE00940007000470A70048
:1049300003F0A10003F8A30013003A006509B100D9
:1049400010003200090035006928E100020035003E
:1049500001002800000005000000400081804800A0
:104960008502E900FCFF3A0000000600F88F4200D3
:10497000050035008100D1000080D3008502E800E9
:10498000FCFF3A00000006008000EB00000005007C
:104990006022B800060220000000D0008180D20012
:1049A0000482D2008582D2000000A00002025200E0
:1049B00083825A00030031000202420083824A00CF
:1049C0000000A1000603E900F3FF3A000000060022
:1049D000EFFF07000400BE0000000600839F680090
:1049E0000100E00002003D0060001000E0801800BF
:1049F0000300E00002003D0060011100E0811900A9
:104A0000E3FF07004F00E00002003B0060001000E1
:104A1000E080180000000600810020006180550041
:104A20000B003D000B00200061FE2F000100E100A3
:104A30001D00340082817100610164008904D1008D
:104A40000884D3000000E800FAFF3A00710020005B
:104A50006100640003007000020060000900320081
:104A600061044400E0844C000988A5000500320080
:104A70008B05E8006808E10002003A008904D100D3
:104A80000884D300F20F20000258E10005003D0029
:104A9000C75DDD00F907B200898075000800780065
:104AA000000006000BF827008B00780000000500CE
:104AB000889FBE008A9FBE00841F780017000700F1
:104AC0004F00780011003300F0FF2F00838F6C003F
:104AD00006003B00040565000A00A7000800370037
:104AE00009F0A6001000200008003700820F5400D3
:104AF000838F5C00030039001000200001003E009D
:104B00000000200009F0A7000000EA004F05BE00E9
:104B10004F04BE000000E000000006000004BE00DC
:104B2000160007000003BE000405BE000200BE0020
:104B300012000700844F7500000006000200BE004E
:104B40006450E100050036006420E10002003600F8
:104B50000968A30001003A000800BE000160A0003F
:104B60004F0678004F05BE004F04BE00000006004F
:104B7000F0FF2F00F1FF2700F9FF3700C70ADE0022
:104B8000F107B200F50FB20008003200E1CF420099
:104B9000020032000170A00024000500810F7000A7
:104BA000010032000408050044000500810F700078
:104BB00002003A00140005008502E90000004000F0
:104BC00081C04800FCFF3B000170A00024000500EC
:104BD0008001EB000200370061F079008301E800FA
:104BE000828F5100FCFF3A00000006003E000000EA
:104BF00008200000080000001B5B000044000000CB
:104C00001B5B000000440000001B00005B43000031
:104C1000001B00005B3200004B0D00000043000051
:104C2000000000001B5B0000324400000057000041
:104C3000617200006E6900006E6700003A2000009B
:104C40006E6F0000207600006F6C00007461000041
:104C500067650000206F00006E20000056700000A5
:104C6000756C00006C750000702000007069000019
:104C70006E000000203D00002000000052450000B2
:104C800053450000540D00000A0000005652000079
:104C900045470000207400006F6F0000206C00008A
:104CA0006F7700002C200000697300002074000062
:104CB000686500007265000020610000207300003C
:104CC000686F0000727400003F0000002E2000009A
:104CD0003C0000002E20000000200000000D00001D
:104CE0000A28000000780000002900003E000000B3
:104CF00042750000732000005069000072610000DE
:104D00007465000020760000340000004669000051
:104D1000726D00007761000072650000207600006F
:104D2000362E0000322D0000626500007461000024
:104D300031200000723100003938000031200000BD
:104D40000020000028320000344600004A320000F3
:104D500035360000474200003130000036200000A8
:104D60000041000033000000413500000055000004
:104D70004E4B0000002900000043000046470000A1
:104D8000303A00002000000056700000753D000021
:104D9000355600002C200000005600007075000001
:104DA0003D330000563300002C2000000049000075
:104DB000090000004F090000004800000900000041
:104DC0004C090000004500006E7400006572000090
:104DD000207200006177000020760000616C000006
:104DE00075650000206600006F7200002042000020
:104DF0005247000000570000617200006E69000019
:104E00006E6700003A200000616C000072650000CF
:104E1000616400007920000061200000766F0000CE
:104E20006C74000061670000652000006F6E000078
:104E300020560000707500006C6C0000757000005A
:104E400020700000696E0000000000004C4500006A
:104E5000540000004946000000540000484500008E
:104E60004E000000454C0000534500000047000084
:104E70004F5400004F000000474F00005355000002
:104E8000420000005245000054550000524E000000
:104E900000520000454D0000005000005249000043
:104EA0004E540000004900004E50000055540000D0
:104EB000004600004F520000005400004F00000068
:104EC0004E450000585400000052000045410000CB
:104ED0004400000044410000544100000053000021
:104EE000544100005254000052000000535400008E
:104EF0004152000054000000535400004F50000085
:104F000052000000535400004F50000000530000B6
:104F1000454E00004400000052450000434500009B
:104F20004956000045000000434C00004B000000C3
:104F30004441000054000000424900005452000067
:104F400045410000440000004144000043000000CF
:104F50004155000058500000494E0000005000002C
:104F60005355000000500000554C00004C55000007
:104F700050000000444500004C4100005900000072
:104F80004155000058000000465200004551000005
:104F90000044000055540000590000004D4100003D
:104FA000435200004F000000454E00004400000046
:104FB00000520000554E0000004C00004953000014
:104FC000540000004558000049540000004400000F
:104FD0004542000055470000004E000045570000C4
:104FE00000000000120100000002000002000000AA
:104FF00000080000D804000000FB000002000000D0
:10500000010200000301000009020000430000004B
:10501000020100000080000064090000040000009C
:105020000001000002020000010000000524000051
:10503000001000000104000024020000020500002E
:10504000240600000001000005240000010100000A
:105050000107000005810000030A00000040000075
:105060000904000001000000020A00000000000026
:1050700000070000050200000240000000000000E0
:10508000070500008202000040000000000400004C
:1050900003090000042A000003440000006100002E
:1050A000006E000000670000006500000072000054
:1050B000006F000000750000007300000020000079
:1050C0000050000000720000006F0000007400003B
:1050D000006F000000740000007900000070000004
:1050E0000065000000730000001E00000342000085
:1050F0000075000000730000002000000050000058
:1051000000690000007200000061000000740000EF
:105110000065000000200000005600000034000080
:1051200000200000001200000330000000300000EA
:1051300000300000003000000030000000300000AF
:10514000003000000031000000000000426100005B
:105150007564000020640000657400006563000051
:10516000746900006F6E000020730000656C000021
:105170006563000074650000642E00002E000000CE
:1051800020000000000000000000000000000000FF
:105190002C01000000000000580200000000000088
:1051A000B0040000000000006009000000000000E2
:1051B000C012000000000000802500000000000078
:1051C0004038000000000000004B0000000000001C
:1051D0008070000000000000009600000000000049
:1051E000C0DA00000000000000E100000000000044
:1051F00000C200000100000000F4000001000000F7
:1052000000E800000300000041520000543100009B
:1052100000000000002900000020000057000000EE
:1052200020520000004E00006F7700002075000043
:10523000736900006E670000206F00006E2D000093
:10524000626F0000617200006420000045450000AC
:10525000505200004F4D0000204900003243000032
:10526000206900006E740000657200006661000035
:1052700063650000004F00006E2D0000626F0000AB
:10528000617200006420000045450000505200009B
:105290004F4D000020770000726900007465000027
:1052A00020700000726F00007465000063740000DD
:1052B0002064000069730000616200006C650000FA
:1052C000640000004932000043310000000000008B
:1052D0003062000000300000303000002C00000080
:1052E0003030000000300000313200003334000064
:1052F00035360000373800003941000042430000D5
:10530000444500004630000078000000436F000074
:10531000756C0000646E000027740000206B0000B4
:10532000656500007020000075700000000000003E
:105330005350000049310000000000002900000027
:10534000007500006E6B00006E6F0000776E00004D
:10535000206D00006F6400006500000050490000EF
:1053600043310000000000003A200000000000006F
:105370002E00000031570000303100000000000016
:1053800042420000494F0000310000005853000025
:105390005631000000000000314100004C53000075
:1053A00000420000507600003400000008080000B1
:1053B000080800000800000000000000204800006D
:1053C0007A00000000000000524100005731000048
:1053D000000000004E4F0000454D0000530000004B
:1053E0000000000029000000000000000000000094
:1053F00020000000000000002800FA000000EB0080
:10540000600F98000000EB00E09789000000EB00BF
:10541000D0978900D0978100200798000000EB000A
:10542000100798000000EB00000F78000000EB0070
:1054300010AE89000000EB00500798000000EB0060
:10544000F09789000000EB00400798000000EB0097
:10545000000F9800130037000000EB006007980071
:105460000A0037000E089000EE0090004500DD00B5
:1054700001014000013023000040EB0000F1780002
:105480006E0090000000E800600798006E00900039
:10549000FF0F5000F3FF34000E0890000000E800FA
:1054A000000F98000E089000E40F5000EAFF34004F
:1054B0000000EB00009D890011AE8100E002200099
:1054C0000088B900610220008080400000002300B5
:1054D0000080400008D002000000000041AE8100C2
:1054E00000202000008060000000E0000400320086
:1054F000710020004065200030F80200000000002C
:10550000605F2A0008D00200000000001F0437007E
:10551000009D81000000E0005F003200009D8100DE
:105520000000E900009D89000000EB006007980082
:105530001B003700D2978100009D8100EE00900093
:105540004500DD008100400000302300E14078008C
:10555000A01F230001717800009D8100EE009000E3
:105560004500DD00810040000030230061407800EC
:10557000FED3020000000000D09781000000E80088
:10558000D09789006E0090000000E8006007980046
:10559000D1978100F00F200000806000D097890033
:1055A000009D8100EE0090004500DD00810040007C
:1055B00000302300614078000004E000DDFF3A0085
:1055C0000000EB00009D89003300370000DF22005F
:1055D00010407800644060000004E0002D003200BC
:1055E00011AE8100E00220000088B900FA004000FE
:1055F000000023000080400010007800000001003F
:105600000000E0002300320011AE8100E002200023
:105610000088B90061022000808040000000230063
:105620000080400008D0020000000000605F2A00F7
:1056300008D0020000000000E1978100D0978100AF
:10564000808F500013003200E097810060079800BF
:105650000C003700EE009000A01F2300614078008E
:10566000FED3020000000000EE009000F00F2000CA
:1056700000806000600798006E0090000000E80065
:1056800060079800EE009000D0978100808F500056
:10569000F0FF3A00D3C2BF0034D402000000000083
:1056A0000004E000C9FF320072D4020000000000D4
:1056B0000004E0000300320086D402000000000075
:1056C000B20337005CD4020000000000604F980075
:1056D0006E4890000080FB006101B900021798003D
:1056E00013179800F0072000010020000E11900011
:1056F0009E119000800F5100818F590036033E00AB
:105700000E1090009E1090000060010027033700EB
:10571000DD0237004D0137002F033700D30037007B
:10572000F4023700620137002B033700770037009F
:10573000290337000A033700270337002603370001
:1057400007033700040237002303370069013700DD
:1057500021033700200337001F0337001E033700E3
:105760001D0337001C0337001B0337001A033700E3
:105770001903370018033700F90037001603370004
:1057800015033700140337001303370012033700E3
:1057900011033700100337000F0337000E033700E3
:1057A0000D0337000C0337000B0337000A033700E3
:1057B00009033700080337000703370006033700E3
:1057C00005033700040337000303370002033700E3
:1057D0000103370000033700FF023700FE023700E5
:1057E000FD023700FC023700FB023700FA023700E7
:1057F000F9023700F8023700F7023700F6023700E7
:10580000F5023700F4023700F3023700F2023700E6
:10581000F1023700F0023700EF023700EE023700E6
:10582000ED023700EC023700EB023700EA023700E6
:10583000E9023700E8023700E7023700E6023700E6
:10584000E5023700E4023700E3023700E2023700E6
:10585000E1023700E0023700DF023700DE023700E6
:10586000DD023700DC023700DB023700DA023700E6
:10587000D9023700D8023700D7023700D6023700E6
:10588000D5023700D4023700D3023700D2023700E6
:10589000D1023700D0023700CF023700CE023700E6
:1058A000CD023700CC023700CB023700CA023700E6
:1058B000C9023700C8023700C7023700C6023700E6
:1058C000C5023700C4023700C3023700C2023700E6
:1058D000C1023700C0023700BF023700BE023700E6
:1058E000BD023700BC023700BB023700BA023700E6
:1058F000B9023700B8023700B7023700B6023700E6
:10590000B5023700B402370058003700E197810034
:105910002E009000810F500050003200D19781007E
:105920002E009000810F50000F003A00D0978100A8
:105930008000E900F00F200000806000D09789000F
:10594000D2978100A11F23000040EB0000F17800F6
:10595000D197810021079800805F2A0008D00200BB
:1059600000000000090337000000EB00000F980062
:105970002E0090008000E900F00F20000080600001
:1059800020079800C05F2A0008D002000000000035
:105990002E019000620798001D0037006E019000F4
:1059A0006E0090008000E800A01F2300E140780016
:1059B000A01F230001717800EE009000A01F2300BB
:1059C000614078000004E000060032006E009000A4
:1059D000A11F230060C07800FED302000000000079
:1059E0000300370000C2B300FED302000000000035
:1059F0000E0890000000E800000F98006E00900074
:105A00008000E800F00F2000008060006007980030
:105A1000EE009000D0978100808F5000DFFF3A00A9
:105A2000D09781008000E900F00F20000080600026
:105A3000D097890000602A0008D002000000000012
:105A40000E089000A0D202000000000030602A0082
:105A500008D0020000000000CC02370070C0B30084
:105A6000FED3020000000000C8023700D197810079
:105A70002E009000810F5000350032000000EB0036
:105A8000000F9800AE019000630798001D003700DA
:105A90006E0190006E0090008000E800A01F2300BF
:105AA000E1407800A01F230001717800EE00900013
:105AB000A01F2300614078000004E00006003200CF
:105AC0006E009000A11F230060C07800FED302008A
:105AD000000000000300370000C2B300FED3020044
:105AE000000000000E0890000000E800000F980081
:105AF0006E0090008000E800F00F20000080600041
:105B000060079800EE009000D0978100808F5000D1
:105B1000DFFF3A00D09781008000E900F00F2000FD
:105B200000806000D097890000602A0008D0020041
:105B3000000000000E089000A0D20200000000004B
:105B400030602A0008D00200000000008F023700F9
:105B500070C0B300FED30200000000008B023700CB
:105B60005CD4020000000000604F9800EE489000F6
:105B7000B0C5B30080CF500084023A005CD402006C
:105B800000000000604F98006E4890000080FB000D
:105B9000700F980010042000FE089000808F5000C5
:105BA00054003200100420007E099000800F510044
:105BB00009003C0010032000FE099000808F510076
:105BC0001200320040032000FE089000808F500039
:105BD000160032006D023700300420007E0990006C
:105BE000800F51003200320030042000FE09900086
:105BF000808F5100D800350040042000FE0890003E
:105C0000808F500011003200600237005CD4020027
:105C100000000000604F9800EE489000E0C7B3001D
:105C200080CF500098013200580237005CD4020047
:105C300000000000604F9800EE489000E0C7B300FD
:105C400080CF5000AB013200500237004E00900070
:105C5000E40F50000500340034E0020000000000B2
:105C60000000EB004007980048023700E1978100F0
:105C70002E009000810F5000090032002E0090008D
:105C80008000E900F00F20000080600020079800ED
:105C9000C05F2A0008D00200000000003B0237006D
:105CA00070C0B300FED302000000000037023700CE
:105CB000D19781002E009000810F50000900320022
:105CC0002E0090008000E800F00F200000806000AF
:105CD0002007980050602A0008D002000000000051
:105CE0002A02370070C0B300FED30200000000009B
:105CF000260237000000EB00000F7800E0978100DB
:105D00000000E90080007800F00F200000806000B3
:105D100060079800840037006E009000A11F2300E8
:105D200060C078000004E0007A003A006E00900045
:105D30008000E900F00F200080806000A01F230099
:105D4000614078000004E000720032001E0FE8009D
:105D50001E0090009E0F10006E0036001E00900086
:105D60000000E80010079800E1978100D0978100BB
:105D7000808F50001200320009003700D297810056
:105D8000A11F23000040EB0000F17800D0978100B4
:105D90008000E900F00F200000806000D0978900AB
:105DA000D1978100E0978100808F5000F3FF3A0087
:105DB000D2978100A11F23000040EB0000F1780082
:105DC0006E0090008000E900F00F2000008060006D
:105DD000000F9800100037000E089000A11F23004C
:105DE00060C078000004E00006003A000E08900051
:105DF0008000E800F00F200000806000500798004D
:105E0000090037000E0890008000E900F00F200024
:105E100000806000000F98008E089000D0978100ED
:105E2000808F5000ECFF3A0090602A0008D00200FA
:105E30000000000011AE8100E00220000088B900DF
:105E400061022000808040000000230000804000AC
:105E500008D002000000000041AE810000202000B8
:105E6000008060000000E0000400320071002000AB
:105E70004065200030F8020000000000605F2A004A
:105E800008D00200000000005E019000020F9800A0
:105E9000150037008E089000A01F23006140780095
:105EA000FED3020000000000D29781008E0890000F
:105EB000A01F2300E1407800A01F2300017178009B
:105EC000D09781008000E800F00F20000080600083
:105ED000D09789000E0890008000E800F00F2000A5
:105EE00000806000000F98008E0890006E00900007
:105EF000808F5000E7FF3A00D2978100A11F230056
:105F00000040EB0000F17800D39781002307980050
:105F1000090037006E0090008000E900F00F2000BB
:105F20000080600060079800EE009000D09781002C
:105F3000808F500078FF3A00EE009000D0978100EB
:105F4000808F500091013A0070C0B300FED3020070
:105F5000000000008D0137000000EB00000F78000A
:105F6000E09781000000E90080007800F00F200039
:105F70000080600060079800850037006E00900088
:105F8000A11F230060C078000004E0007B003A00FD
:105F90006E0090008000E900F00F2000808060001B
:105FA000A01F2300614078000004E000730032006D
:105FB0001E0FE8001E0090000000E9009E0F500038
:105FC0006E003A001E0090000000E90010079800E3
:105FD000E1978100D0978100808F5000120032003D
:105FE00009003700D2978100A11F23000040EB0079
:105FF00000F17800D09781008000E900F00F2000C8
:1060000000806000D0978900D1978100E0978100DF
:10601000808F5000F3FF3A00D2978100A11F230028
:106020000040EB0000F178006E0090008000E90075
:10603000F00F200000806000000F98001000370073
:106040000E089000A11F230060C078000004E0004B
:1060500006003A000E0890008000E800F00F2000D3
:106060000080600050079800090037000E0890007B
:106070008000E900F00F200000806000000F980011
:106080008E089000D0978100808F5000ECFF3A007E
:1060900090602A0008D002000000000011AE8100CC
:1060A000E00220000088B9006102200080804000EA
:1060B000000023000080400008D002000000000023
:1060C00041AE810000202000008060000000E00060
:1060D00004003200710020004065200030F802000A
:1060E00000000000605F2A0008D0020000000000ED
:1060F0005E009000000F9800150037008E08900099
:10610000A01F230061407800FED3020000000000C1
:10611000D29781008E089000A01F2300E1407800F4
:10612000A01F230001717800D09781008000E80053
:10613000F00F200000806000D09789000E089000CA
:106140008000E800F00F200000806000000F980041
:106150008E0890006E009000808F5000E7FF3A009C
:10616000D2978100A11F23000040EB0000F17800CE
:10617000D197810021079800090037006E00900038
:106180008000E900F00F20000080600060079800A8
:10619000EE009000D0978100808F500077FF3A008A
:1061A000EE009000D0978100808F5000F7003A00F9
:1061B0001E009000E10F50002F003A0090602A006E
:1061C00008D002000000000011AE8100E0022000B3
:1061D0000088B90061022000808040000000230098
:1061E0000080400008D002000000000041AE8100A5
:1061F00000202000008060000000E0000400320069
:10620000710020004065200030F80200000000000E
:10621000605F2A0008D0020000000000090037007B
:10622000D2978100A11F23000040EB0000F178000D
:10623000D09781008000E900F00F2000008060000E
:10624000D0978900D1978100E0978100808F50001E
:10625000F3FF3A00D2978100A11F23000040EB001A
:1062600000F17800D2978100220798000000EB002F
:1062700010079800C500370070C0B300FED30200BD
:1062800000000000C1003700E19781002E0090005F
:10629000810F500013003200E19781002E00900022
:1062A0000100500080007800F00F200000806000A6
:1062B000000F980000602A0008D0020000000000D3
:1062C0000E089000A0D202000000000030602A00FA
:1062D00008D0020000000000E39781002307980027
:1062E000AA00370070C0B300FED302000000000017
:1062F000A6003700D19781002E009000810F50003A
:1063000013003200D19781002E00900000805000D1
:1063100080007800F00F200000806000000F9800DF
:1063200000602A0008D00200000000000E08900063
:10633000A0D2020000000000F0602A0008D0020095
:1063400000000000D0978100200798008F003700E0
:1063500070C0B300FED30200000000008B003700C5
:1063600010002000600F98000000EB00100798005C
:10637000D2978100A11F23000040EB0000F17800BC
:10638000D09781008000E800F00F200000806000BE
:10639000D0978900D19781002107980010612A00C9
:1063A00034D0020000000000780037004E0090005A
:1063B0000000E800400798004E009000F40F5000E5
:1063C00072003A0070C50200000000000000EB00FF
:1063D0004007980007023700D09781008000E8004E
:1063E000F00F200080806000E0978100808F5000D7
:1063F000630032006E489000FF4F5000600036008E
:10640000EE489000E0C7B30080CF50005C003E0033
:10641000D19781002E009000808F500013003A0029
:106420006E489000FED3020000000000D297810069
:10643000EE489000A01F230001717800D0978100E2
:106440008000E800F00F200000806000D0978900F5
:10645000D2978100A11F23000040EB0000F17800DB
:10646000D29781002207980048003700D197810019
:106470002E0090000080500080007800F00F200077
:1064800000806000000F980000602A0008D0020021
:10649000000000000E089000A0D2020000000000E2
:1064A000F0602A0008D0020000000000D0978100B0
:1064B00060079800190037006E0090000001E800A6
:1064C000EE009000A01F2300E1407800A01F2300F1
:1064D00001717800EE009000A01F23006140780059
:1064E0000004E000080032006E009000A11F2300AD
:1064F00060C07800FED302000000000020612A0086
:1065000008D00200000000006E0090008000E9004A
:10651000F00F200000806000600798006E0190007E
:106520002E0090008000E900F00F20000080600045
:10653000800F5100E0FF3A006E489000FED3020049
:10654000000000002E019000EE489000A01F2300E4
:10655000017178002E0090008000E800F00F20000C
:106560000080600020079800D09781008000E8003C
:10657000F00F200000806000D097890003003700F2
:1065800070C0B300FED30200000000006E0890004F
:106590000000E000DEFB3200D0978100400F980041
:1065A000E0978100300F98000000EB00600F98002A
:1065B0000000EB00500F98000000EB00F0978900FE
:1065C00041AE810000202000008060000000E0005B
:1065D000140532007E590200000000005100200026
:1065E000B0652000BAF80200000000001000200092
:1065F000500F98000B053700E1978100A01F230082
:1066000061407800604F98006E4890000080FB0069
:106610006101B9002217980033179800E0072000A5
:10662000010020002E119000BE119000800F51003B
:10663000818F5900CF043E002E109000BE109000B4
:1066400000600100CD043700CA043700C9043700D8
:10665000C8043700C7043700C6043700C504370034
:10666000C4043700C3043700C2043700C304370032
:10667000C0043700BF043700C0043700BD04370032
:10668000BC043700BB043700BA043700B904370034
:10669000B8043700B7043700B6043700B504370034
:1066A000B4043700B3043700B2043700B104370034
:1066B000B0043700AF043700AE043700AD04370034
:1066C000AC043700AD0437008A043700D30237002A
:1066D0004501370049013700F2013700E00137007A
:1066E000A4043700AD023700A2043700A10437002C
:1066F000A2043700A1043700360437004F043700E6
:106700001A043700470337004603370045033700B4
:106710004403370043033700420337004103370087
:10672000400337003F0337003E0337009104370032
:1067300090043700FB013700E30037008D04370079
:10674000470037005B0137004D01370089043700EF
:106750006C003700BF01370086043700850437001E
:106760008404370083043700820437008104370033
:1067700078003700810037007E0437007D04370041
:106780007C043700A70037007A043700790437000B
:10679000D9013700770437007604370075043700D5
:1067A0005A01370073043700720437007104370050
:1067B000F8023700FA033700080337002E043700C9
:1067C000110437006B043700200137002F00370019
:1067D0004200370091013700B9003700310037001F
:1067E00033003700160037002000370061043700FF
:1067F0004E0037006D003700220037005D0437007F
:1068000024003700750037005A0437007F03370033
:10681000B501370057043700560437001F00370012
:106820006C0137005304370052043700510437001D
:10683000E1023700BF003700F1023700DD0037000A
:10684000DC0607000000E0004C043A00E0978100FD
:10685000300F9800D0978100400F98004704370010
:10686000D0F80200000000004404370016090700B9
:1068700010AE81000000E000400432004C09070027
:106880003E043700450607003C043700C00A0700F5
:106890003A0437009A0A070038043700060A07004E
:1068A000360437007CC102000000000033043700CA
:1068B00010AE81000000E00005003A00D101200088
:1068C000B0682000BAF80200000000002B04370076
:1068D000E6BF0200000000002804370001DF2200AC
:1068E000114078000000A1000010A100804878004D
:1068F0006101200000662000BAF8020000000000DC
:106900001E04370001DF2200114078000000A000C3
:106910000010A1008048780051012000606720002D
:10692000BAF80200000000001404370001DF220062
:10693000114078000000A1000010A00080487800FD
:1069400071012000B0452100BAF8020000000000EB
:106950000A04370001DF2200114078000000A00087
:106960000010A0008048780071012000204721001D
:10697000BAF80200000000000004370001DF220026
:10698000114078000030A00080487800C10120004C
:10699000408D200030F802000000000010612A0045
:1069A00034D0020000000000F403370001DF2200B1
:1069B000114078000030A10080487800B10120002B
:1069C000908B200030F802000000000010612A00C7
:1069D00034D0020000000000E803370010AE810050
:1069E0000000E00005003A00D1012000B06820005E
:1069F000BAF8020000000000E0033700E282A900BC
:106A0000E082A90051012000806A200030F80200D5
:106A10000000000010612A0034D0020000000000D5
:106A2000D603370010AE81000000E00005003A00F8
:106A3000D1012000B0682000BAF802000000000078
:106A4000CE03370000DF2200104078007040600065
:106A50000004E00004003A0021022000D0FB2000E6
:106A6000BAF8020000000000E082A800E282A9005B
:106A700041012000D06B200030F80200000000002F
:106A800010612A0034D002000000000021E3A800B9
:106A900050C0B30088F402000000000080007800BD
:106AA000F0042000808F500003003E0070612A0037
:106AB00034D002000000000021E3A900AF0337003A
:106AC0008B0A0700AD033700E09781008000E800E3
:106AD000F00F200000806000E0978900A00507000B
:106AE000DA030700600798006E00900002D30200EE
:106AF00000000000A0632A0008D00200000000008F
:106B00006E009000A0D2020000000000A0632A00E6
:106B100008D00200000000006E00900068D0020063
:106B20000000000010612A0034D0020000000000C4
:106B300092033700E09781008000E800F00F20000A
:106B400000806000E097890085050700BF0307000B
:106B5000600798006E0090000080FB001AF60200AB
:106B600000000000600798006E00900002D3020051
:106B700000000000A0632A0008D00200000000000E
:106B80006E009000A0D2020000000000A0632A0066
:106B900008D00200000000006E00900068D00200E3
:106BA0000000000010612A0034D002000000000044
:106BB0007203370010AE81000000E00005003A00CB
:106BC00011C0B30010C0B30044E702000000000091
:106BD0006A033700A1012000106D2000BAF80200FE
:106BE0000000000065033700E0632A0008D00200BF
:106BF00000000000340807006003370060F902005D
:106C0000000000000000E0005C033200A100200052
:106C1000006F2000BAF802000000000040062000CB
:106C2000B8F5020000000000FAF3020000000000C6
:106C30002CD40200000000000004E000FCFF320041
:106C400081BF2A00014001004C0337000405070002
:106C50000000E800000F98000200370064C3020043
:106C6000000000000E0890000000E900000F9800EE
:106C70000E0890000000E000F8FF3A003F033700E4
:106C8000F70407000000E800000F9800020037003A
:106C900014C30200000000000E0890000000E9008C
:106CA000000F98000E0890000000E000F8FF3A0086
:106CB00032033700EA0407000000E800000F9800E4
:106CC0000B00370061012000A06F200030F80200A7
:106CD00000000000B4C3020000000000F2CF020078
:106CE0000000000010612A0034D002000000000003
:106CF0000E0890000000E900000F98000E089000B8
:106D00000000E000EFFF3A001C03370010AE8100E6
:106D10000000E00005003A00D1012000B06820002A
:106D2000BAF802000000000014033700C922A900CD
:106D3000CB22A80021E3A80020002000B8F5020023
:106D4000000000000040EB0088F40200000000009A
:106D500080007800001B2000808F50000F0036005C
:106D600020C0B30088F4020000000000800078001A
:106D7000702B2000808F5000080036001101200089
:106D80000071200030F802000000000010612A00AD
:106D900034D00200000000000C003700C922A90016
:106DA000CB22A90060642A0034D002000000000059
:106DB000210120001072200030F8020000000000C5
:106DC00010612A0034D002000000000021E3A90075
:106DD000EA02370010AE81000000E00005003A0032
:106DE000D1012000B0682000BAF8020000000000C5
:106DF000E2023700C922A900CB22A900210120000C
:106E00001072200030F802000000000010612A001B
:106E100034D0020000000000D8023700F10020004A
:106E2000C036200030F8020000000000A2F402008A
:106E30000000000011002000B037200030F80200F0
:106E40000000000010612A0034D0020000000000A1
:106E5000CA023700B4F4020000000000C702370085
:106E60007F040700000F980061002000F0732000ED
:106E700030F80200000000000E08900042D202002C
:106E8000000000002100200050742000BAF8020029
:106E9000000000000E089000E4F502000000000071
:106EA000B60237006E040700000F98006100200052
:106EB000F073200030F80200000000000E0890007F
:106EC00042D202000000000021002000100021003A
:106ED000BAF80200000000000E089000B8F50200A9
:106EE00000000000A502370040AE81000090A00025
:106EF00040AE8900A102370010AE81000000E00022
:106F000005003A00D1012000B0682000BAF8020064
:106F1000000000009902370026C4020000000000B3
:106F20009602370010002000F09789001000200022
:106F3000600798000F003700E19781006E00900015
:106F400080804000F00F200080806000A01F2300A0
:106F5000E1407800E0C3B30080CF500002003A0067
:106F60000000EB00F09789006E0090000000E80040
:106F700060079800E19781006E00900080804000DB
:106F8000F00F200080806000A01F23006140780087
:106F90000004E000E8FF3A00EE009000200220002C
:106FA000808F50000200340010002000F09789000C
:106FB000F09781000000E00070023A00E097810045
:106FC0008000E800F00F200000806000E09789005A
:106FD0009E02070060079800E1978100F00F2000F3
:106FE00080806000A01F2300E1407800D0C3B30080
:106FF00080CF50003C003A006E0090000000E0009E
:10700000360034006E009000E50F500033003C0065
:10701000E09781008000E800F00F20000080600011
:10702000E09789006E0090000000E900600798007A
:107030000000EB00000F98000A0037006E0090007F
:107040008E0890004500DD00010140000130230062
:107050000040EB0000F178000E0890000000E8000E
:10706000000F98000E089000FF0F5000F3FF34004F
:107070000000EB00000F9800110037006E01900037
:107080008E099000E1978100A01F230061427800E3
:107090004510DD008300400000302300847078003C
:1070A0000E0890000000E800000F9800E0978100B3
:1070B0008000E800F00F200000806000E097890069
:1070C000E1978100A01F2300E1407800E0C3B300F6
:1070D00080CF5000E9FF3A0028023700100020005E
:1070E000F0978900250237006E0090000000E00054
:1070F0001B003A000000EB00000F9800140037005E
:107100000E0890000040E800A0D20200000000003D
:1071100060662A0008D00200000000000E089000FF
:107120004500DD0080007800003023000080400032
:1071300008D0020000000000605F2A0034D0020086
:10714000000000000E0890000000E800000F98000A
:107150000E089000E40F5000E9FF340007023700EA
:107160006E0090000000E000090034006E00900006
:10717000E50F500006003C0010612A0034D00200E8
:1071800000000000EE009000019D8900FB01370027
:1071900010002000F0978900F8013700E097810087
:1071A0008000E800F00F200000806000E097890078
:1071B00026020700200F9800E9030700E1978100ED
:1071C000F00F200080806000A01F2300E1407800C5
:1071D00090C2B30080CF50000D003A0011AE810084
:1071E000E00220000088B900FC00400000002300FD
:1071F00000804000900078002E08900001000100FF
:1072000010612A0034D0020000000000DB013700CA
:1072100010002000F0978900D801370010002000EE
:10722000F097890010002000600798000F003700D9
:10723000E19781006E00900080804000F00F2000F8
:1072400080806000A01F2300E140780020C2B300CE
:1072500080CF500002003A000000EB00F097890058
:107260006E0090000000E80060079800E197810040
:107270006E00900080804000F00F20008080600051
:10728000A01F2300614078000004E000E8FF3A00FE
:10729000F09781000000E000B8013A007100200082
:1072A0007074200030F802000000000020C2B3001B
:1072B000FED302000000000020003700E1978100AB
:1072C000F00F200000806000E0978900E1978100C6
:1072D000A01F230061407800FED3020000000000E0
:1072E000E1978100A01F2300614078000000FB00AF
:1072F000200F980000DF22001040780068406000F6
:107300000004E000040032002E0890001AF602008B
:1073100000000000200F980011AE8100E002200064
:107320000088B900E8004000000023000080400011
:10733000900078002E08900001000100E097810085
:107340000000E800E0978900E1978100F00F20003D
:1073500080806000A01F2300E140780020C2B300BD
:1073600080CF5000D5FF3A00E0978100F10F200058
:1073700001006000E097890020C2B300FED3020044
:107380000000000010612A0034D00200000000005C
:107390007A01370011AE8100E00220000088B900B8
:1073A000800078000000230000804000100078007A
:1073B000000001007101370011AE8100E0022000E1
:1073C0000088B9008080E8000000230000804000B1
:1073D00010007800000001006801370011AE810044
:1073E000E00220000088B900E40040000000230013
:1073F0000080400010007800000001005F013700AD
:1074000011AE8100E00220000088B900E6004000D3
:107410000000230000804000100078000000010000
:1074200056013700710020007074200030F802000F
:107430000000000085010700200F9800E097810000
:107440000000E900E0978900E1978100F00F20003B
:1074500000806000E0978900010307000000E80059
:10746000000F980020030700300798003E009000AE
:107470000000E0005B0032003E0090008040780099
:10748000F0DD2200014878003E009000E80F500037
:107490000500340001DF2200114078000050A000F8
:1074A000804878004F00370001DF2200114078004B
:1074B0000050A100804878004A0037002E08900054
:1074C00012F502000000000000DF220010407800EA
:1074D0000042B2000004E00004003A00F0DD2200A7
:1074E00010407800E84F500009003A0000DF220009
:1074F000104078000042B2000004E0000B003200AF
:10750000F0DD220010407800F04F500007003200FC
:10751000B0C3B300FED3020000000000F0DD220083
:1075200010407800A0D202000000000000DF22001E
:1075300010407800684060000004E0000400320061
:107540002E0890001AF6020000000000200F98009C
:1075500011AE8100E00220000088B900E800400080
:107560000000230000804000900078002E0890006A
:1075700001000100100F980000C2B300FED302000A
:107580000000000000DF2200104078000044B2003C
:107590000004E0001300320061002000E0742000CD
:1075A00030F802000000000000DF220010407800E8
:1075B000684060000004E000040032001E089000F3
:1075C0001AF6020000000000100F98001E0890003C
:1075D00012F502000000000000C2B300FED302005A
:1075E000000000000E0890000000E900000F980065
:1075F0000E0890000000E000B0FF3A0010612A0081
:1076000034D0020000000000DC00370061002000E0
:10761000E074200030F80200000000009002070033
:107620000000E800000F9800AF0207003007980044
:107630003E0090000000E000420032003E0090005A
:1076400080407800F0DD2200014878003E00900084
:10765000E80F50000500340001DF220011407800DF
:107660000050A000804878003600370001DF22007B
:10767000114078000050A1008048780031003700A8
:1076800011AE8100E00220000088B900EA0040004D
:10769000000023000080400010007800000001007E
:1076A000100F980000DF2200104078006840600052
:1076B0000004E000040032001E0890001AF60200E8
:1076C00000000000100F98001E08900012F5020044
:1076D0000000000000DF2200104078000042B200ED
:1076E0000004E00004003A00F0DD220010407800C1
:1076F000E84F500009003A0000DF220010407800F7
:107700000042B2000004E0000B003200F0DD220075
:1077100010407800F04F500007003200B0C3B300B3
:10772000FED3020000000000F0DD220010407800CF
:10773000A0D202000000000000C2B300FED302008D
:10774000000000000E0890000000E900000F980003
:107750000E0890000000E000C9FF3A0010612A0006
:1077600034D00200000000008400370081002000B7
:1077700040752000BAF802000000000011AE810040
:10778000E00220000088B900EC0040000000230067
:1077900000804000100078000000010077003700F2
:1077A00081002000C0752000BAF80200000000002F
:1077B00011AE8100E00220000088B900EE00400018
:1077C000000023000080400010007800000001004D
:1077D0006A003700E100200040762000BAF802007D
:1077E0000000000011AE8100E00220000088B90016
:1077F000F0004000000023000080400010007800EE
:10780000000001005D003700E1002000207720002B
:10781000BAF802000000000011AE8100E002200072
:107820000088B900F2004000000023000080400002
:10783000100078000000010050003700C100200057
:107840003073200030F802000000000011AE81000B
:10785000E00220000088B900F4004000000023008E
:10786000008040001000780000000100F2CF02000C
:107870000000000041003700F9010700000F9800E8
:10788000D10020000079200030F802000000000044
:107890000E08900012F50200000000000E08900093
:1078A0000000E800000F98000800370011AE8100CA
:1078B000E00220000088B900F6004000000023002C
:1078C0000080400010007800000001000E089000C9
:1078D0000000E900000F98000E0890000000E00092
:1078E000F2FF3A0010612A0034D0020000000000CC
:1078F00022003700DA0107000000E800000F9800BE
:10790000A1002000D079200030F802000000000023
:107910000D00370011AE8100E00220000088B900A0
:10792000F8004000000023000080400010007800B4
:1079300000000100F2CF02000000000000C2B3000E
:10794000FED30200000000000E0890000000E900D5
:10795000000F98000E0890000000E000EDFF3A00D4
:107960000101200000782000BAF8020000000000A9
:107970000200370010002000F0978900E097810096
:107980008000E800F00F200000806000E097890090
:10799000F09781000000E0001C003200510120003F
:1079A000707A200030F8020000000000BE0890004D
:1079B000E0978100808F500007003100E097810040
:1079C000804078003E08900000C05000A0D2020025
:1079D0000000000006003700E0978100804078003A
:1079E0003E08900000C05000A0D20200000000003D
:1079F0000000EB00F097890010002000500F980065
:107A000010612A0034D0020000000000E1978100DC
:107A1000D0978100808F500002003A0010002000B3
:107A2000500F98005E0890000000E000F2FA32006B
:107A30004E089000E09789004E089000D09789008A
:107A40000000EB00600F98009BF637000600FA007C
:107A50000000EB00100798000000EB00000F78001A
:107A6000E19781001E00900080804000F00F200010
:107A700080806000A01F2300E140780000C3B300B5
:107A800080CF50003E003400E19781001E0090003E
:107A900080804000F00F200080806000A01F230045
:107AA000E140780090C3B30080CF500034003C0028
:107AB000E19781001E00900080804000F00F2000C0
:107AC00080806000A01F2300614078008000FB00E0
:107AD00000FD2F00008F40001E0090000000E80015
:107AE00010079800110037001E0078006A00B900E6
:107AF000000F7800E19781001E0090008080400018
:107B0000F00F200080806000A01F230061407800FB
:107B10000000FB009E00400000FD2F00008F400091
:107B20001E0090000000E80010079800E197810017
:107B30001E00900080804000F00F200080806000D8
:107B4000A01F2300E1407800F0C2B30080CF5000B6
:107B500036013400E19781001E00900080804000D3
:107B6000F00F200080806000A01F2300E14078001B
:107B700090C3B30080CF5000DBFF34002B013700EF
:107B8000E19781001E00900080804000F00F2000EF
:107B900080806000A01F2300E140780000C3B30094
:107BA00080CF50001C013A001E0090000000E80049
:107BB00010079800E19781001E009000808040002F
:107BC000F00F200080806000A01F2300E1407800BB
:107BD00020C6B30080CF50000A003200E197810038
:107BE0001E00900080804000F00F20008080600028
:107BF000A01F2300E140780020C4B30080CF5000D4
:107C00002A003A001E0090000000E80010079800CB
:107C1000110037001E00780000004000000F7800BF
:107C2000E19781001E00900080804000F00F20004E
:107C300080806000A01F2300614078000000FB00EE
:107C40009E00400000FD2F00008F40001E009000AD
:107C50000000E80010079800E19781001E009000E6
:107C600080804000F00F200080806000A01F230073
:107C7000E140780010C3B30080CF5000E5FF320030
:107C8000E19781001E00900080804000F00F2000EE
:107C900080806000A01F2300E140780000C3B30093
:107CA00080CF5000DBFF3200E0003700E197810019
:107CB0001E00900080804000F00F20008080600057
:107CC000A01F2300E140780080C7B30080CF5000A0
:107CD0000A003200E19781001E0090008080400081
:107CE000F00F200080806000A01F2300E14078009A
:107CF00080C5B30080CF500082003A001E00900083
:107D00000000E80010079800410037001E007800CE
:107D10004400DD00000F7800E19781001E00900014
:107D200080804000F00F200080806000A01F2300B2
:107D3000E1407800F0C2B30080CF5000160034005C
:107D4000E19781001E00900080804000F00F20002D
:107D500080806000A01F2300E140780090C3B30042
:107D600080CF50000C003C00E19781001E00900085
:107D700080804000F00F200080806000A01F230062
:107D8000614078000000FB009E00400000FD2F00D5
:107D9000008F40001B003700E19781001E0090001B
:107DA00080804000F00F200000816000E19781009A
:107DB0001E00900080804000F00F20008080600056
:107DC000A01F2300E140780000C2B30080C0700013
:107DD000A01F230001717800E19781001E00900030
:107DE00080804000F00F200080806000A01F2300F2
:107DF000614078000000FB009E00400090FA2F00D8
:107E0000008F40001E0090000000E800100798005E
:107E1000E19781001E00900080804000F00F20005C
:107E200080806000A01F2300E1407800F0C2B30012
:107E300080CF50000A003400E19781001E009000BE
:107E400080804000F00F200080806000A01F230091
:107E5000E140780090C3B30080CF5000ABFF340006
:107E6000E19781001E00900080804000F00F20000C
:107E700080806000A01F2300E140780000C4B300B0
:107E800080CF50000A003400E19781001E0090006E
:107E900080804000F00F200080806000A01F230041
:107EA000E140780060C4B30080CF500097FF3400F9
:107EB000E19781001E00900080804000F00F2000BC
:107EC00080806000A01F2300E140780000C6B3005E
:107ED00080CF500055003400E19781001E009000D3
:107EE00080804000F00F200080806000A01F2300F1
:107EF000E140780060C6B30080CF500083FF3400BB
:107F00004A003700E19781001E0090008080400009
:107F1000F00F200080806000A01F2300E140780067
:107F2000F0C2B30080CF500040003400E1978100E0
:107F30001E00900080804000F00F200080806000D4
:107F4000A01F2300E140780090C3B30080CF500011
:107F500036003C00E19781001E00900080804000C8
:107F6000F00F200080806000A01F23006140780097
:107F70008000FB0000FD2F00008F40001100370043
:107F80001E0078006A00B900000F7800E1978100B8
:107F90001E00900080804000F00F20008080600074
:107FA000A01F2300614078000000FB009E004000FD
:107FB00000FD2F00008F40001E0090000000E80030
:107FC00010079800E19781001E009000808040001B
:107FD000F00F200080806000A01F2300E1407800A7
:107FE000F0C2B30080CF500010003400E197810050
:107FF0001E00900080804000F00F20008080600014
:10800000A01F2300E140780090C3B30080CF500050
:10801000DBFF34000500370010002000F0978900D6
:108020000000EB00200798000A003700E19781006C
:108030001E00900000804000E0978900E1978100D9
:10804000F00F200000806000E09789001E0078009B
:10805000200798002E0090000080FA000000060023
:108060000400FA00E09781008000E800F00F200093
:1080700080806000A01F2300E1407800A0C3B3000F
:1080800080CF500013003A00E09781000080E800A4
:10809000E0978900E1978100F00F200000806000E8
:1080A000E097890069FE0700000F7800E0978100E3
:1080B0000000E900E0978900E1978100F00F2000BF
:1080C00000806000E09789001E007800100798008B
:1080D0000200370010002000100798001E009000DA
:1080E0000080FA00000006000400FA00E09781001A
:1080F0008000E800F00F200080806000A01F2300B7
:10810000E1407800B0C3B30080CF50000F003A00C8
:10811000E09781008080E800F00F20000080600080
:10812000E097890049FE0700000F7800E097810082
:108130008000E900F00F200000806000E0978900D7
:108140001E00780010079800020037000000EB00C6
:10815000100798001E0090000080FA000000060042
:108160000000FA0005003700E09781008000E80079
:10817000F00F200000806000E0978900E197810007
:10818000A01F2300E140780000C2B30080CF500060
:10819000F5FF32000080FA00000006000400FA003B
:1081A0000000EB00000F7800E09781008000E800FD
:1081B000F00F200000806000E0978900E8FF0700D2
:1081C00022FE0700000F78001E00E0004D003A007C
:1081D0000000EB0010079800130037001E0090000D
:1081E0000040E800A0D2020000000000A0662A00C3
:1081F00008D00200000000009E009000E002200075
:108200000088B90061022000808040000000230047
:108210000080400034D00200000000001E009000EA
:108220000000E800100798001E009000EA0F5000C0
:10823000EAFF340071012000C07B2000BAF8020080
:10824000000000000000EB00F09789001300200000
:10825000B20020001100200010002000F4000700F0
:10826000000FE900E0FF2F009E0F10000300320016
:108270000080EB009E0F100005003A00E100200096
:10828000307D2000BAF802000000000042003700F4
:1082900011AE8100E00220000088B9000102200038
:1082A0008080400000002300008040001000780023
:1082B00000000100FAF30200000000001E00780038
:1082C00010AE890011AE8100E00220000088B900E4
:1082D000FE004000000023000080400010007800F5
:1082E000000001001E00E00001003200CB02A800E7
:1082F00051002000B0652000BAF802000000000024
:10830000250037001E0FE900A00020009E0F10007E
:108310001D003C0011AE8100E00220000088B90081
:108320000102200080804000000023000080400007
:108330001000780000000100FAF3020000000000C5
:108340001E00780010AE890011AE8100E00220000E
:108350000088B900FE0040000000230000804000BB
:1083600010007800000001001E00E0000100320053
:10837000CB02A80051002000B0652000BAF802002E
:10838000000000000400370051012000208120007F
:10839000BAF8020000000000D09781008000E900D8
:1083A000F00F200000806000E09789000080FA0054
:1083B000000006002600FA001000200020079800A8
:1083C000E09781000000E90080007800F00F2000B5
:1083D00000806000100798003D0037001E009000EC
:1083E000A11F230060C078000004E00033003A00C1
:1083F0001E0090008000E800F00F200080806000E8
:10840000A01F2300614078000004E0002B00320030
:108410002E009000A0D2020000000000A0662A00FA
:1084200008D002000000000010002000000F7800BB
:10843000090037001E0090009E004000F00F200051
:1084400080806000A01F230061407800FED30200FE
:10845000000000001E0FE8001E0090009E0040007B
:10846000F00F200080806000A01F23006140780092
:108470000004E000EFFF3A00AE0190001E00900003
:108480008000E800F00F200000816000E600470057
:108490000380410002B078002E0090000000E80048
:1084A000200798002E009000EF0F50000C003200C3
:1084B00010612A0034D00200000000001E0090006D
:1084C0008000E900F00F2000008060001007980095
:1084D0009E009000E0978100808F5000BFFF3A001F
:1084E000D0662A0034D00200000000007100200095
:1084F00070822000BAF80200000000001300200083
:108500002E019000110020000000EB004800070041
:10851000100798001E009000E10F40000300320099
:108520001E0090000000E00006003A0010612A00E2
:1085300034D0020000000000100020002017980036
:10854000380037000000EB002007980014003700C7
:10855000D19781002E00900080804000F00F200015
:10856000008160001E009000E6004700000040000F
:10857000E08078002E00900080804000F00F200006
:1085800080806000A01F2300E1407800A01F23002E
:10859000017178002E0090000000E800200798008C
:1085A0001E009000E600470000004000E0807800D8
:1085B0002E00900080804000F00F2000808060003E
:1085C000A01F2300614078000004E000E0FF3A00B3
:1085D000D09781008000E900F00F2000008060004B
:1085E000E0978900E19781002E0090000080400014
:1085F0008080E800F00F200000806000D0978900A4
:10860000D09781008000E900F00F20000081600019
:10861000A11F23000040EB0000F178000000EB00F8
:10862000201798002E1090000080FA00000006002D
:108630001E00FA00100F9800210F9800320F9800CA
:10864000430F98000000EB00400798000000EB008B
:10865000200798000000EB00100798000000EB00D6
:10866000000F7800F0662A0008D002000000000029
:108670001E0890000000E00004003D0030672A0062
:1086800008D0020000000000030037001E08900020
:10869000A0D202000000000050672A0008D00200AB
:1086A00000000000670037005CD4020000000000FA
:1086B000204F98002E4890000000FB00600F9800AB
:1086C0006E089000ED0F500029003200EE08900077
:1086D000ED8F500007003C006E099000E80F51003C
:1086E0000D0032006E089000EA0F500020003200AA
:1086F00035003700D0022000EE089000808F500037
:108700001E003200800720006E099000800F51008B
:10871000270032002C0037004E0090000000E000DF
:10872000070032004E0090000000E900400798006A
:10873000805F2A0008D002000000000041003700DE
:108740001E00E000060032000000EB00000F780081
:10875000805F2A0008D002000000000039003700C6
:1087600070C0B300FED302000000000035003700E7
:108770001000200020079800320037004E009000C3
:108780000000E00006003A00D0C2B300FED30200B1
:108790000000000010002000000F780029003700C2
:1087A00070C0B300FED302000000000025003700B7
:1087B0004E0890000000E000030032000080EB0053
:1087C000500F98005D003700AE489000F0C2B30033
:1087D00080CF500018003400AE48900090C3B30022
:1087E00080CF500014003C004E009000E30F50007A
:1087F0000600340070C0B300FED302000000000089
:1088000040002000400798000E0037002E489000DE
:10881000FED3020000000000CE0090006B00470075
:108820002E499000827078004E0090000000E80011
:10883000400798000300370070C0B300FED3020069
:10884000000000002E0090000000E00096FF3200C3
:1088500010612A0034D00200000000004E00900099
:108860000000E00003003A001E089000500F98003E
:10887000320037000000EB00100798004E00900017
:108880000000E90040079800CE00900031079800F2
:10889000110037001E0090006A00B9001007980010
:1088A000BE0090004E009000808050006B0047009A
:1088B000614078008000FB001E0090008080400036
:1088C00000FD2F0000804000100798004E0090002F
:1088D0000000E900400798004E0090000000E00012
:1088E000ECFF3D009E0090002E089000808F50000D
:1088F0000D0035009E0090003E089000808F5000D3
:1089000009003C001E00E000040032001E00900040
:108910000000EA00500F9800080037001E01900088
:10892000520F980005003700B101200060FE2000C2
:10893000BAF802000000000042FF37005E08900015
:108940000080FA00000006002C00FA00500F98008A
:10895000610F9800720F980004179800151798007F
:10896000231798000000EB00500798000000EB0070
:10897000300798006000B800008FBE000000EB00D8
:1089800020079800F0662A0008D0020000000000CE
:108990005E089000EE089000E00F5000E08F580055
:1089A00004003D0030672A0008D0020000000000EB
:1089B000040037005E089000EE089000A2D002008C
:1089C0000000000050672A0008D0020000000000EC
:1089D0006A0037005CD4020000000000404F98009D
:1089E0004E4890000000FB00501798005E10900069
:1089F000ED0F50002A003200DE109000ED8F500085
:108A000007003C005E119000E80F51000D0032009D
:108A10005E109000EA0F500021003200380037004D
:108A2000D0022000DE109000808F50001F00320026
:108A3000800720005E119000800F51002800320056
:108A40002F0037005E0090000000E00007003200B9
:108A50005E0090000000E90050079800805F2A0047
:108A600008D0020000000000440037002E009000F3
:108A70000000E000060032000000EB002007980034
:108A8000805F2A0008D00200000000003B00370091
:108A900070C0B300FED302000000000037003700B2
:108AA0001000200030079800340037005E0090006E
:108AB0000000E00006003A00D0C2B300FED302007E
:108AC0000000000010002000200798002B00370055
:108AD00070C0B300FED30200000000002700370082
:108AE0002E1090000000E000050032000080EB0036
:108AF0008080EB0030179800411798006E00370017
:108B0000CE489000F0C2B30080CF5000180034006F
:108B1000CE48900090C3B30080CF500014003C00BA
:108B20005E009000E90F50000600340070C0B300F2
:108B3000FED3020000000000A000200050079800B3
:108B40000E0037004E489000FED3020000000000E7
:108B5000DE0090006D0047004E4990008270780062
:108B60005E0090000000E800500798000300370006
:108B700070C0B300FED30200000000003E00900071
:108B80000000E00093FF320010612A0034D00200A0
:108B9000000000005E0090000000E00005003A00C8
:108BA0005E089000EE08900030179800411798007A
:108BB000410037006000B800008FBE005E009000EA
:108BC0000000E90050079800DE009000410798007F
:108BD0001A0037009E007800A0002000000AB800AC
:108BE0001E0078006000B900050178000001410016
:108BF0001E0090006A00B900000141008202780066
:108C0000048FBE00CE0090005E0090008080500077
:108C10006D004700614078008000FB0000FD2F00E0
:108C200000804000CF80DE001E0F40005E974800AD
:108C30005E0090000000E900500798005E00900080
:108C40000000E000E3FF3D007E089000CF80DE00E2
:108C5000BE0F5000AE8F580012003C000E10900066
:108C60009E109000BE0F1000AE8F18000D003C004B
:108C70002E0090000000E000060032001E00BE0042
:108C800060001000E080180030179800411798002D
:108C9000090037001E00BE003017980041179800E9
:108CA00005003700B101200060FE2000BAF8020084
:108CB000000000002BFF37003E109000CE10900007
:108CC0000080FA00000006000400FA0080672A0015
:108CD00034D002000000000060682A0008D00200C2
:108CE0000000000010612A0034D0020000000000E3
:108CF000610020009084200030F802000000000095
:108D000020AE810052D3020000000000710020005C
:108D1000F0FD200030F802000000000030AE8100BD
:108D200052D3020000000000106A2A0008D002009E
:108D30000000000030AE8100100798001E00900077
:108D4000E10F5000040032001E009000E30F5000BD
:108D50000500320008003700106B2A0008D002001E
:108D60000000000007003700406B2A0008D0020016
:108D70000000000003003700706B2A0008D00200DA
:108D800000000000B06B2A0034D002000000000098
:108D9000E1012000F0842000BAF802000000000089
:108DA0000000EB00000F78000080FA0000000600D1
:108DB0000200FA00D06B2A0008D002000000000078
:108DC000A17F250010002000D8D302000000000081
:108DD00052D302000000000000C2B300FED3020024
:108DE0000000000051002000C0A3200030F8020065
:108DF00000000000C17F250010002000D8D3020031
:108E00000000000052D302000000000061002000BA
:108E100010A4200030F8020000000000E17F2500CF
:108E200010002000D8D302000000000052D302003E
:108E30000000000010612A0034D002000000000091
:108E4000C1002000D0862000BAF802000000000017
:108E500099000700CBC2BF00624060000004E00040
:108E600005003200110120000071200030F80200DE
:108E700000000000040037002101200010722000D3
:108E800030F8020000000000C0C2B300FED30200B0
:108E90000000000000C2B300FED30200000000008A
:108EA000E2C2BF00704060000004E0000500320034
:108EB00041012000D06B200030F8020000000000CB
:108EC0000400370051012000806A200030F80200C1
:108ED00000000000C0C2B300FED30200000000008A
:108EE00000C2B300FED3020000000000E8C2BF00D1
:108EF0000042B2000004E00003003A00406C2A0087
:108F000008D0020000000000E8C2BF00704060000E
:108F10000004E00003003A00D06C2A0008D00200F0
:108F20000000000000DF2200104078007040600068
:108F30000004E0000500320021022000908720009C
:108F4000BAF802000000000004003700E101200030
:108F5000B0892000BAF802000000000000DF220003
:108F600010407800684060000004E00005003A000E
:108F7000B1012000908B200030F8020000000000BA
:108F800004003700C1012000408D200030F80200AD
:108F900000000000C0C2B300FED3020000000000C9
:108FA00000C2B300FED3020000000000B1012000A7
:108FB0000035210030F8020000000000F0DD220042
:108FC00010407800A0D202000000000010612A00CA
:108FD00034D002000000000000DF22009040780042
:108FE00063C060000080FB00000F78001E00780066
:108FF000E10F5000130032009E007800E18F500016
:1090000004003C001E0078000000E0000800320070
:109010001A0037009E007800E28F50000E003200E8
:109020001E007800E30F50001000320013003700DC
:109030005101200060672000BAF802000000000023
:109040000E0037006101200000662000BAF802001F
:10905000000000000900370071012000B045210028
:10906000BAF802000000000004003700710120007F
:1090700020472100BAF802000000000011AE810074
:10908000E00220000088B9004102200080804000FA
:109090000000230000804000100078000000010064
:1090A000C1002000D0862000BAF8020000000000B5
:1090B0000080FA00000006000000FA00A100200075
:1090C00020192100BAF8020000000000610520000C
:1090D000703A2100BAF802000000000041022000AE
:1090E000D03F210030F802000000000011AE8100E6
:1090F000E00220000088B9002102200080804000AA
:1091000000002300008040001000780000000100F3
:10911000A1002000601B210030F8020000000000C8
:109120001000200058000700001020005600070023
:109130000002200054000700000120005200070038
:109140008000200050000700400020004E00070073
:10915000200020004C00070010612A0034D00200DB
:1091600000000000410020000023210030F8020030
:109170000000000021E3A80020C0B30088F4020032
:109180000000000094D30200000000001100200045
:10919000B037200030F802000000000090C0B3009B
:1091A000FED30200000000000040EB0088F4020043
:1091B0000000000094D30200000000001100200015
:1091C000B037200030F802000000000090C0B3006B
:1091D000FED302000000000050C0B30088F402007B
:1091E0000000000094D302000000000011002000E5
:1091F000B037200030F802000000000090C0B3003B
:10920000FED302000000000010C0B30088F402008A
:109210000000000094D302000000000011002000B4
:10922000B037200030F802000000000090C0B3000A
:10923000FED302000000000021E3A900100020007E
:1092400020000700001020001E0007000002200080
:109250001C000700000120001A0007008000200009
:109260001800070040002000160007002000200022
:109270001400070010612A0034D002000000000032
:109280000080FA00000006000200FA00000F7800DB
:10929000C01680001E0060000000E00004003200E4
:1092A000706D2A0008D002000000000003003700A3
:1092B000A06D2A0008D00200000000000080FA0023
:1092C000000006000200FA00000F7800D0168000AF
:1092D0001E0060000000E00004003200D06D2A0093
:1092E00008D002000000000003003700006E2A00D2
:1092F00008D00200000000000080FA000000060014
:109300000200FA00E09781008000E800F00F2000E2
:1093100000806000E097890091FB0700CBF907000F
:10932000000F78001E00E00006003400400020001E
:109330009E0F100003003C001E00E90000AE8900F3
:109340000D0037000000EB00F0978900210220009B
:10935000D08F2000BAF80200000000008001EB006E
:10936000420020001100200010002000B0FC070087
:109370000000E90000AE890021012000F0912000EA
:10938000BAF80200000000000080FA0000000600A9
:109390000200FA000040EB00004F7800E0978100E7
:1093A0008000E800F00F200000806000E097890056
:1093B0006BFB0700A5F90700104798001E409000BE
:1093C0000004E000090032001E409000EA4F500007
:1093D00006003E001E4090000040E90080407800FA
:1093E000E05B2300014878000F0037000000EB002D
:1093F000F0978900E10B2000C0952000BAF8020028
:10940000000000008001EB00A200200011002000FD
:109410009000200086FC07000040E90080407800B2
:10942000E05B230001487800E05B230010407800F7
:10943000E94F500010003A0049FB070083F907008C
:10944000004F78001E04E0000B003A000000EB0023
:10945000F0978900306E2A0034D00200000000002E
:109460008001EB00F2FF27008000EB0020022000CB
:109470006FFC0700004F780041012000A0A12000F0
:10948000BAF802000000000011012000F0332100B2
:10949000BAF80200000000002CD402000000000016
:1094A0000004E000FCFF3200E05B23001040780085
:1094B000E94F500003003A001E40780092D40200A9
:1094C000000000008CD40200000000005CD4020008
:1094D000000000008040780000C2B30080CF500040
:1094E00001003200F9FF37000080FA00000006009A
:1094F0000400FA0010AE81000000E00007003A000E
:10950000D1012000B0682000BAF80200000000007D
:1095100010002000F09789007500370000DF22005E
:1095200010407800704060000004E00007003A003E
:1095300021022000D0FB2000BAF802000000000049
:1095400010002000F097890069003700E8A2A80009
:10955000E882A80020002000B8F50200000000000A
:1095600021E3A80050C0B30088F40200000000000E
:109570008000780000102000808F5000030036002B
:10958000B06F2A0034D002000000000021E3A900DF
:10959000E09781008000E800F00F2000008060006C
:1095A000E0978900EEFA070028F90700000F78001D
:1095B000F09781000000E0000C0032000000EB009A
:1095C000F097890071052000504A2100BAF8020086
:1095D000000000008001EB0032002000110020009C
:1095E0001000200012FC0700000F78001E00780019
:1095F000100798001E009000E20F50001200320089
:109600001E009000E30F50001F0032001E0090006B
:10961000E10F5000010032002B003700E8A2A80043
:10962000E882A80091012000C04F210030F802001C
:109630000000000081002000C0512100BAF80200A3
:10964000000000002A003700E8A2A800EA82A90072
:10965000E882A9004100200000C6200030F8020086
:109660000000000091012000C04F210030F80200EE
:10967000000000007100200050512100BAF80200E3
:10968000000000001A003700E882A800EAA2A90042
:10969000E8A2A90021002000B0C5200030F8020097
:1096A0000000000091012000C04F210030F80200AE
:1096B000000000007100200050512100BAF80200A3
:1096C000000000000A003700E8A2A800E882A80015
:1096D00091012000C04F210030F80200000000007E
:1096E00081002000C0512100BAF8020000000000F3
:1096F0000080FA00000006000000FA00214381000B
:10970000C0862200E140780030C8B30080CF50000E
:109710000D003A00204381000000E800204389004A
:1097200003003700204381000000E8002043890047
:1097300021438100C0862200E140780000CEB300C2
:1097400080CF5000F7FF36000080FA0000000600CE
:109750000A00FA00300798000000EB00200798008C
:10976000AE009000C0862200E140780000CEB30039
:1097700080CF500003003E000080EB0040079800BF
:1097800020003700AE009000C086220061407800C3
:109790008080FB0000F22F0000804000100798003E
:1097A0002E0090008000E800C08622006140780012
:1097B0000080FB004801DD002E0090008080E80062
:1097C000C0862200614078000080FB00000F41004D
:1097D0009E0078003E009000808F500003003A0009
:1097E0002E00900040079800060037009E00900071
:1097F0002E00900000804000630040002007980089
:10980000D7FF37004E0090000080FA0000000600ED
:109810000600FA00881F78000000EB00000F7800B7
:1098200021438100C0862200E140780080C2B3005D
:1098300080CF50000F003A00204381000000E80074
:109840002043890013010700000F780021438100A5
:10985000C0862200E140780090C2B30080CF500063
:10986000B4003A00204381000000E8002043890052
:10987000B000370021438100C0862200E14078001B
:1098800000C4B30080CF5000140036002143810093
:10989000C0862200E1407800A0C5B30080CF500010
:1098A0000E003E0022438100C08622006240780004
:1098B0008080FB00F0FB2F00008040008000400013
:1098C00040802200008040001000780020079800AF
:1098D0000200E800204389009800370021438100FE
:1098E000C0862200E140780000C8B30080CF50005D
:1098F0008400360021438100C08622006140780048
:109900000080FB00100798000100E8002043890058
:10991000700920009E009000808F50004A003200A5
:10992000700920009E009000808F50000D003C00C8
:10993000400920009E009000808F50001F003200E0
:10994000600920009E009000808F5000340032009B
:10995000300920009E009000808F500021003200CE
:1099600058003700A00920009E009000808F500012
:109970003F003200A00920009E009000808F500020
:1099800005003C00800920009E009000808F500060
:10999000450032004B003700B00920009E009000C7
:1099A000808F500039003200D00920009E009000C6
:1099B000808F5000160032004200370011AE810047
:1099C000E00220000088B900EA0040000000230007
:1099D000008040001000780000000100000F7800B7
:1099E0005400370011AE8100E00220000088B90069
:1099F000E8004000000023000080400010047800D0
:109A0000A400070008000100000F7800490037009B
:109A1000B4C3020000000000000F780045003700CA
:109A200011AE8100E00220000088B900F40040007F
:109A300000002300008040001000780000000100BA
:109A4000000F78003B00370011AE8100E0022000DB
:109A50000088B900F80040000000230000804000AA
:109A60001000780000000100000F7800310037007E
:109A7000CBC2BF000080FB000000D100614060004D
:109A80000080FB00000F78002A003700E2C2BF0010
:109A90000080FB004400DE00614060000080FB00AD
:109AA000008FEA002300370021E3A80010C0B300B4
:109AB00088F4020000000000000F780021E3A900F4
:109AC0001C0037000000EB00000F78001900370081
:109AD0001E0078006A00B900000F78002143810061
:109AE000C0862200614078000080FB009E0040009C
:109AF00000FD2F00008F4000204381000000E8009F
:109B00002043890021438100C0862200E140780083
:109B1000F0C2B30080CF5000060036002143810020
:109B2000C0862200E140780090C3B30080CF50008F
:109B3000E7FF36001E007800200798002E009000F6
:109B40004F0478000080FA00000006000600FA00CA
:109B50002FFF0700000F780000003700214381002D
:109B6000C0862200E1407800A0C2B30080CF500040
:109B70001500320021438100C0862200E1407800B8
:109B8000F0C2B30080CF50000F00320021438100AB
:109B9000C0862200E140780060C2B30080CF500050
:109BA0000900320021438100C0862200E140780094
:109BB000C0C7B30080CF5000030032001E00780001
:109BC000200798003000370021438100C086220022
:109BD000614078000080FB00100798000100E80059
:109BE00020438900A00220009E009000808F50003A
:109BF00012003200A00220009E009000808F5000D2
:109C000005003C00600220009E009000808F500004
:109C100017003200D1FF3700F00220009E009000B4
:109C2000808F50000B003200C00720009E00900083
:109C3000808F500011003200C8FF3700F4FE07008B
:109C4000800078001E0078000180B900000F7800C5
:109C5000C2FF3700EEFE0700000178001E0078000A
:109C6000110009000200D800000F7800BBFF370088
:109C7000E7FE07001E0F6000B8FF3700E4FE070094
:109C80001E0F7000B5FF37002E0090000080FA0014
:109C9000000006001200FA00ACFF0700000F780079
:109CA0000000370021438100C0862200E140780097
:109CB000D0C2B30080CF50001B003200214381008E
:109CC000C0862200E1407800B0C2B30080CF5000CF
:109CD0001500320021438100C0862200E140780057
:109CE000C0C3B30080CF50000F0032002143810079
:109CF000C0862200E1407800E0C3B30080CF50006E
:109D00000900320021438100C0862200E140780032
:109D1000D0C3B30080CF5000030032001E00780093
:109D2000200798008100370021438100C08622006F
:109D3000614078000080FB00100798000100E800F7
:109D400020438900C00320009E009000808F5000B7
:109D50003A003200C00320009E009000808F500027
:109D600009003C00B00220009E009000808F50004F
:109D700011003200D00220009E009000808F500021
:109D80000A003200C7FF3700D00320009E00900079
:109D9000808F50005B003200E00320009E009000A6
:109DA000808F500007003200BEFF370067FF0700BA
:109DB0001E0F1000BBFF370064FF07001E0F40009E
:109DC000B8FF3700204381008000E800C0862200F1
:109DD000E1407800D0C3B30080CF50000D003A00BE
:109DE0005AFF07008000EB00310798009E0F5000DB
:109DF00002003E001000200030079800BE009000D6
:109E0000010F7800204381000000E8002043890012
:109E1000A4FF37004DFF07008000EB0041079800CA
:109E20009E0F5000020031001000200040079800F3
:109E3000CE009000010F78009AFF37002043810088
:109E40008000E800C0862200E1407800E0C3B30053
:109E500080CF50000D003A003CFF07008000EB006F
:109E6000510798009E0F50000200320010002000A1
:109E700050079800DE009000010F78002043810019
:109E80000000E8002043890086FF3700204381005E
:109E90008000E800C0862200E1407800D0C3B30013
:109EA00080CF50000D003A0028FF07008000EB0033
:109EB000610798009E0F500002003900100020003A
:109EC00060079800EE009000010F780020438100A9
:109ED0000000E8002043890072FF37001BFF0700E5
:109EE0008000EB00710798009E0F500002003600C2
:109EF0001000200070079800FE009000010F78000D
:109F000068FF370011FF07008000EB00010F980089
:109F10009E0F500002003A0010002000000F980031
:109F20008E089000010F78005EFF37002E00900031
:109F30000080FA00000006001C00FA00881F78006C
:109F40000000EB00204389000000EB003007980080
:109F50000000EB00200798000000EB0010079800BD
:109F60000000EB00304389000000EB004043890013
:109F70000000EB00504389000000EB005007980000
:109F800040AE81000080A00040AE89000000EB00E0
:109F900040079800090037004E0090008000400004
:109FA00040802200808040000000EB0080087800A4
:109FB0004E0090000000E800400798004E0090001E
:109FC000F90F5000F4FF34000B0437001E0090001E
:109FD0000000E0001D003A0021438100C0862200FD
:109FE000E1407800F0CDB30080CF500003003E0088
:109FF0002000200030079800020437002143810030
:10A00000C0862200614078008080FB0000F22F00B3
:10A010000080400060079800204381008000E80035
:10A02000C0862200614078000080FB004801DD000E
:10A03000204381008080E800C086220061407800D3
:10A040000080FB0000007100500798000000EB004A
:10A050001007980020438100E3004000C0862200E2
:10A06000614078000080FB006101B90000F82F001A
:10A07000F1FF2F000201400083814800420F980049
:10A08000530F980010022000010020004E0990009C
:10A09000DE099000800F5100818F5900CA033E00F5
:10A0A0004E089000DE08900000600100210037009B
:10A0B00034003700C4033700C30337006C00370097
:10A0C0007C0037009E003700B2003700B90037002F
:10A0D0002B01370073013700BB033700D501370070
:10A0E0001B023700770237008D0237007D023700F0
:10A0F000A902370099023700B6023700B2033700D1
:10A100005403370038033700AF033700AE0337007E
:10A11000DE023700CE0237007B03370089033700A9
:10A12000BC023700EE0237000E0337009103370000
:10A13000A203370010002000200798002043810070
:10A140006600400020438900204381008080E900B0
:10A15000C0862200614078008080FB00F0FB2F0069
:10A1600000844000CBFE0700000178008800440016
:10A170004080220000804000020878005EFD070059
:10A18000930337001000200020079800204381002F
:10A190006400400020438900BEFE07000000E0008C
:10A1A0001B00320021438100310F9800C08622003D
:10A1B0003E099000E24078008041EB004357980050
:10A1C00020C8B30080CF500002003A0010C0B30096
:10A1D00040579800BE0890000100E8002043890025
:10A1E0004E5190000204E00079033200100020007C
:10A1F000100798002043810063005000204389002D
:10A2000073033700204381000000E80020438900E9
:10A2100021438100C0862200E140780030C8B300AD
:10A2200080CF50000600320021438100C08622000A
:10A23000E140780000CEB30080CF5000F1FF36003F
:10A2400021438100C0862200E140780030C8B3007D
:10A2500080CF50005E033A001000200010079800E5
:10A26000204381000080E900204389005803370023
:10A270001000200020079800204381006400400067
:10A280002043890083FE070031FD0700000F78009E
:10A290008081EB009E8F1100030032001E007800C9
:10A2A000204389004A0337006000200030079800EF
:10A2B000470337001000200020079800204381004A
:10A2C000640040002043890040438100E90F5000B2
:10A2D00018003C0042438100214381006E00900041
:10A2E000008040008001E90082004100808322005C
:10A2F0000080400003087800404381000000E8002F
:10A300004043890063FE070011FD0700000F78003D
:10A310008080EB009E8F1000030032001E01780049
:10A32000224389002A03370060002000300798008C
:10A3300027033700700020003007980024033700FF
:10A3400020742A0008D00200000000001000200045
:10A3500020079800404381000000E0000A0032001E
:10A36000404381000000E9004043890040438100F0
:10A3700080004000808322000080400010007800B0
:10A380002043890012033700800020003007980026
:10A390000F033700100020002007980021438100A0
:10A3A0006E00900000804000630040002043890060
:10A3B0000703370010002000200798002043810089
:10A3C00064004000204389004F0037002143810092
:10A3D000C0862200E140780020C2B30080CF500048
:10A3E0001D003A00204381000000E800204389005E
:10A3F0000F00370040AE81000080A10040AE890010
:10A4000021438100C086220061407800004178002D
:10A410000100E8002043890002407800FED30200DA
:10A420000000000040AE81000080A00040AE890026
:10A4300021438100C0862200E140780020C2B300A1
:10A4400080CF5000EBFF3A00204381000000E8007D
:10A45000204389002C00370021438100C086220060
:10A46000E140780000C4B30080CF50000600360001
:10A4700021438100C0862200E1407800A0C5B300DE
:10A4800080CF50000B00360021438100C08622009F
:10A49000614078000004E00012003D00214381008B
:10A4A000C0862200E1407800F0CDB30080CF50009C
:10A4B0000C003E00F7FD0700000F780040AE810061
:10A4C0000080A10040AE89001E00780042D2020048
:10A4D0000000000040AE81000080A00040AE890076
:10A4E0000900370021438100C0862200E140780046
:10A4F000B0C3B30080CF500003003A002043810076
:10A500000000E8002043890021438100C08622002A
:10A51000E1407800F0CDB30080CF500006003E004F
:10A5200021438100C0862200E140780030C8B3009A
:10A5300080CF5000A5FF3A00204381008000E90051
:10A54000C0862200E1407800B0C3B30080CF500045
:10A550000900320040AE81000080A10040AE8900B9
:10A56000807D2A0034D002000000000040AE81004F
:10A570000080A00040AE89005FFC07009402370015
:10A58000100020002007980040AE81000080A1004C
:10A5900040AE8900204381006400400020438900D0
:10A5A00021438100C0862200E140780020C2B30030
:10A5B00080CF500016003A00204381000000E800E0
:10A5C000204389000900370021438100C086220012
:10A5D00061407800004178000100E80020438900D4
:10A5E00002407800FED302000000000021438100F9
:10A5F000C0862200E140780020C2B30080CF500026
:10A60000F1FF3A00204381000000E8002043890068
:10A6100021438100C0862200E1407800C0C2B3001F
:10A6200080CF500004003A00204381000000E80081
:10A6300020438900020037003000200030079800D6
:10A6400021438100C0862200614078008080FB00A9
:10A65000F0FB2F00008440008001EB00F2FF270098
:10A660008000EB000000EB00184302000000000037
:10A6700000017800880044004080220000804000F3
:10A6800002087800204381000000E8002043890090
:10A6900019FC070040AE81000080A00040AE890098
:10A6A0004B02370010002000200798002043810053
:10A6B000640040002043890030438100E30F5000D4
:10A6C00004003C00304381000000E8003043890072
:10A6D000020037004000200030079800324381001C
:10A6E00023438100C0862200634078008080FB0005
:10A6F00000FC2F00008240006610B9008080E80056
:10A70000C084220000804000040878000300E800B4
:10A710002043890021438100C0862200E140780067
:10A72000D0C3B30080CF500011003A002043810015
:10A730000000E80020438900304381006600B90032
:10A740008080E800C0842200008040001000780073
:10A750000004E9004FFD0700000178008800440074
:10A76000408022000080400002087800020037008C
:10A77000300020003007980023438100130F980019
:10A78000C08622001E099000E24078008041EB0064
:10A7900003579800B0C8B30080CF500002003A00C1
:10A7A00010C0B300005798009E0890000100E80018
:10A7B000204389000E5190000204E000090032009D
:10A7C0003843810033FD0700000178006640B9007E
:10A7D000E4004000C08422000080400002087800AD
:10A7E000020037003000200030079800214381002C
:10A7F000C0862200E1407800F0CDB30080CF500049
:10A800000800360030438100224381006600B90011
:10A8100080007800C0842200008040000208780098
:10A82000020037003000200030079800B2FB07001C
:10A83000E701370010002000200798002043810026
:10A84000640040002043890022438100C08622002A
:10A85000624078008080FB0000FC2F00008F4000E9
:10A860000200E800204389005000200030079800D3
:10A870000000EB00400798002F0037004E009000CA
:10A880006600B9008080E800C0842200008040009B
:10A89000100078009E0F500024003A001E00E900CE
:10A8A00080004000408022000080400010017800BD
:10A8B0004E0090006600B900E4004000C084220011
:10A8C0000080400010007800800F510012003D0011
:10A8D0009E00E9000181400040802200000041000C
:10A8E000100078000001E8008180400040802200D4
:10A8F00000804000020878004E0090006600B90019
:10A9000080007800C08422000080400010007800A1
:10A910002043890003003700304381000000E90034
:10A92000304389000000EB00300798004E00900093
:10A930000000E80040079800314381004E0090007D
:10A94000810F5000CDFF34006BFB0700A0013700E2
:10A950001000200020079800204381006400400080
:10A9600020438900504381000000E00023003A00AA
:10A970000000EB004007980009003700CE0090006F
:10A98000C0862200614078008080FB004E0090006D
:10A990008080400030F22F00008040004007980087
:10A9A0004E009000E3004000C0862200E1407800A5
:10A9B000E0C8B30080CF5000050032004E00900088
:10A9C000C186220060C078000004E000EBFF3A007E
:10A9D0004E009000C186220060C078000004E000B4
:10A9E000040032004E009000640040005043890093
:10A9F00002003700900020003007980023438100B8
:10AA0000030F780050438100204389009E007800A6
:10AA1000C0862200614078008080FB00F0FB2F00A0
:10AA2000008440007AFB07000001780088004400A1
:10AA3000408022000080400002087800204381000E
:10AA4000504389001E00E8002043890051438100E3
:10AA5000C0862200E1407800C0C2B30080CF500021
:10AA600003003A00504381000000E8005043890091
:10AA700051438100C0862200E140780000CEB3003F
:10AA800080CF50000D00360050438100E3004000AD
:10AA9000C0862200E1407800E0C8B30080CF5000BB
:10AAA000030032000000EB00504389000300370030
:10AAB0005043810064004000504389000EFB0700B2
:10AAC0004301370010002000200798002143810037
:10AAD0006E00900000804000630040002043890029
:10AAE0003B01370010002000200798002043810020
:10AAF000640040002043890011AE8100E002200084
:10AB00000088B90080007800000023000080400029
:10AB10001000780000000100F7FA07002C01370050
:10AB200010002000200798002043810064004000AE
:10AB30002043890011AE8100E00220000088B900A6
:10AB40008080E800000023000080400010007800B2
:10AB500000000100E8FA07001D0137001000200086
:10AB600020079800204381006400400020438900B2
:10AB700011AE8100E00220000088B900E40040002E
:10AB80000000230000804000100078000000010059
:10AB9000D9FA07000E0137001000200020079800A6
:10ABA00020438100640040002043890011AE8100F1
:10ABB000E00220000088B900E60040000000230009
:10ABC000008040001000780000000100CAFA070071
:10ABD000FF0037001000200020079800204381006C
:10ABE000640040002043890011AE8100E002200093
:10ABF0000088B900E8004000000023000080400009
:10AC00001004780023FC070008000100BAFA0700CE
:10AC1000EF0037001000200020079800204381003B
:10AC200064004000204389001AFC07000000E00097
:10AC30000300320014C302000000000002003700CD
:10AC400064C3020000000000ABFA0700E000370018
:10AC5000100020002007980020438100640040007D
:10AC6000204389000BFC07000000E00003003200D5
:10AC7000C922A900CB22A80002003700C922A900DE
:10AC8000CB22A9009CFA0700D10037001000200059
:10AC90002007980020438100640040002043890081
:10ACA000FCFB07000000E0000600320001DF22008C
:10ACB000114078000000A0000010A100804878003A
:10ACC0000500370001DF2200114078000000A000DD
:10ACD0000010A1008048780087FA0700BC00370008
:10ACE00010002000200798002043810064004000ED
:10ACF00020438900E7FB070030AF890030AF8100B7
:10AD00000000E00002003D000000EB0030AF8900D1
:10AD100031AF810000FA2000808F50000200340023
:10AD200000FA200030AF890040AF8100E10F5000F1
:10AD300002003C002000200040AF890041AF8100AC
:10AD400030062000808F50000200340030062000C2
:10AD500040AF890044BF02000000000066FA07000F
:10AD60009B0037001000200020079800204381003E
:10AD70006400400020438900C6FB070040AF890003
:10AD800030AF81000000E00002003D000000EB0059
:10AD900030AF890031AF810000FA2000808F500071
:10ADA0000200340000FA200030AF890040AF81007B
:10ADB000E10F500002003C002000200040AF89005D
:10ADC00041AF810030062000808F50000200340027
:10ADD0003006200040AF890044BF020000000000A0
:10ADE00045FA07007A00370010002000200798007D
:10ADF000204381006400400020438900A5FB070038
:10AE00000000E0000900320011AE8100E0022000E5
:10AE10000088B900F00040000000230000804000DE
:10AE200010007800000001000800370011AE81001A
:10AE3000E00220000088B900F2004000000023007A
:10AE40000080400010007800000001002AFA07008E
:10AE50005F00370010002000200798002043810089
:10AE600064004000204389008AFB070070079800B7
:10AE70007E009000E10F500010003200FE009000B4
:10AE8000E28F5000160032007E0190000200E000C8
:10AE9000010032001A00370011AE8100E0022000EC
:10AEA0000088B900EE004000000023000080400050
:10AEB00010007800000001001100370011AE810081
:10AEC000E00220000088B900EC00400000002300F0
:10AED00000804000100078000000010008003700EA
:10AEE00011AE8100E00220000088B900F6004000A9
:10AEF00000002300008040001000780000000100E6
:10AF0000FDF90700320037001000200020079800EC
:10AF10002043810064004000204389005DFB07005E
:10AF20000000E00003003200E082A800E282A900F5
:10AF300002003700E282A900E082A900EEF90700D2
:10AF400023003700100020002007980020438100D4
:10AF500064004000204389004EFB0700000F78008A
:10AF60001E007800B8F5020000000000E2F90700BA
:10AF700017003700100020002007980020438100B0
:10AF8000640040002043890042FB0700000F780066
:10AF900011AE8100E00220000088B900FC004000F2
:10AFA0000000230000804000900078001E00780020
:10AFB00001000100D0F90700050037001000200053
:10AFC000300798000200370030002000300798005A
:10AFD0002E0090000000E00005003A0021438100AF
:10AFE0006E00900000804000630040002043890014
:10AFF0000000EB00200798003E0090000000E000F9
:10B00000F2FB320040AE81000080A10040AE89001A
:10B010003E009000E10F5000180032006100200057
:10B02000C037200030F80200000000003E00900011
:10B0300042D20200000000008100200020382000E1
:10B0400030F80200000000005E00900042D20200D2
:10B0500000000000B1002000A038200030F80200FD
:10B06000000000002043810042D2020000000000E6
:10B07000807D2A0034D00200000000004F047800D8
:10B080000080FA00000006000200FA00000F7800BD
:10B0900000C2B300FED30200000000001E007800D2
:10B0A00008D002000000000000C2B300FED302007E
:10B0B000000000000080FA00000006000400FA0012
:10B0C0000000EB00204389003C0037002043810052
:10B0D000C186220060C17800224798002E4090006F
:10B0E0000004E000040035002E409000FED3020072
:10B0F000000000002E003700AE40900000CEB300EC
:10B1000080CF50001A003600807D2A0034D0020023
:10B1100000000000204381008000E800C08622007B
:10B12000614078000080FB004801DD002043810081
:10B130008080E800C0862200614078000080FB002B
:10B1400000004100000F7800204381000080E800EB
:10B15000204389001E00780042D202000000000057
:10B1600000C2B300FED30200000000001000370050
:10B1700000C2B300FED30200000000002E40900089
:10B180008080FB0000F82F0000804000800040001D
:10B1900020502300008040001000780008D00200FA
:10B1A0000000000000C2B300FED302000000000057
:10B1B000204381000000E8002043890020438100F3
:10B1C000C186220060C078000004E000BFFF3A00A2
:10B1D000807D2A0034D0020000000000204381005E
:10B1E0000000E90042D202000000000071002000CF
:10B1F00050392000BAF80200000000000080FA0078
:10B20000000006000600FA0010079800E097810091
:10B21000000F7800140037001E00900010417800E5
:10B22000E1978100A01F230061407800804F51000A
:10B23000050032001E007800E09789000000EB0056
:10B24000200798000E003700E09781008000E8009A
:10B25000F00F200000806000E09789001E00900041
:10B260000000E800100798001E00900010407800D1
:10B270000004E000E8FF3A001000200020079800DA
:10B280002E0090000080FA00000006000400FA0082
:10B290000000EB00000F7800100037001E0078005F
:10B2A0008000400020502300008040001000780003
:10B2B000D4FF07000000E000070032001E00780005
:10B2C0008040780000C8B30000C040000080FB0050
:10B2D00010079800060037001E0FE800100220003B
:10B2E0009E0F1000EDFF34000000EB0010079800E7
:10B2F0001E0090000080FA00000006003600FA00F0
:10B30000E0978100000F98001B0037008E08900026
:10B31000A01F2300E140780000C6B30080CF50009A
:10B320000E0034008E089000A01F2300E14078003A
:10B33000A0C7B30080CF500008003C000E09900069
:10B340008E089000A01F2300E1407800F0CDB300EC
:10B3500080C06000A01F2300017178000E089000DB
:10B360000000E800000F98008E089000F00F200009
:10B3700000806000000F98008E089000D097810038
:10B38000808F5000E1FF3A000000EB00000F9800B2
:10B39000E1978100A01F2300E1407800F0C2B300D4
:10B3A00080CF50001E013400E1978100A01F2300D0
:10B3B000E140780090C3B30080CF500018013C00FA
:10B3C0000000EB00000F9800080037008E08900086
:10B3D00072004700808040000040EB008048780009
:10B3E0000E0890000000E800000F98008E08900002
:10B3F00020022000808F5000F4FF3400263D020020
:10B4000000000000600798006E0090004880DE0099
:10B410008040780072004700114098006E00900054
:10B420008040780000C0EB0080C0600072004700E0
:10B43000214098006E009000C5F807005007980062
:10B440005E009000E10F400027003200DE00900017
:10B45000C0862200614078008080FB0030F22F001F
:10B4600000804000300798005E009000000F9800B8
:10B470000B0037000E0990008E0890003E009000EF
:10B4800080804000C0862200E1407800C086220013
:10B49000017178000E0890000000E800000F98008D
:10B4A000014020003E009000808050000E08900077
:10B4B000808F5000EFFF3C00070037000E0990001E
:10B4C000C18622000040EB0000F178000E089000D9
:10B4D0000000E800000F98008E089000F03F200068
:10B4E000808F5000F5FF340030002000000F9800DE
:10B4F0000000EB0020079800B040020000000000B0
:10B50000400037002E0090000000E00002003A00EA
:10B51000B0400200000000002E0090000000E0009B
:10B5200004003A0059FF07000080FB006007980004
:10B53000020037000000EB00600798006E009000EA
:10B540000000E0000D0032000E0990006E00900037
:10B5500080407800720047000000410001487800F8
:10B56000EE00900070082000808F500019003A0013
:10B57000100020002007980016003700E197810096
:10B58000A01F2300E140780020C2B30080CF50000C
:10B5900003003A002E0090000000A200200798004F
:10B5A0000E099000E1978100A01F23006140780000
:10B5B0008040780072004700000041000148780098
:10B5C000E09781008000E800F00F2000008060001C
:10B5D000E09789000E0890000000E800000F980036
:10B5E0008E08900030022000808F5000050034004B
:10B5F00091002000C0392000BAF8020000000000CD
:10B60000CB003700E1978100D0978100808F5000F8
:10B61000BCFF3A000E089000E30F5000C400320057
:10B620000E089000E40F5000C10032000E08900098
:10B6300080407800C0CDB30000C04000804078005A
:10B6400072004700014878000000EB00000F9800EE
:10B650000000EB00400798000000EB005007980046
:10B66000400037008E089000C0862200E14078003C
:10B6700000CEB30080CF50002B0036008E08900023
:10B68000C0862200614078008080FB0000F22F001D
:10B6900000804000300798000E0890008000E8000D
:10B6A000C0862200614078000080FB004801DD0078
:10B6B0000E0890008080E800C0862200614078007B
:10B6C0000080FB0000004100100798007200470056
:10B6D000104090000080FB00C800DD0072004700B1
:10B6E000204090000080FB0000804000000F7800A8
:10B6F0001E0090009E0F5000050031008E08900043
:10B700003E00900000804000630040005007980019
:10B71000BE0090000E0890000080400063004000D2
:10B72000000F9800020037000E08900040079800B4
:10B730000E0890008000E800C0862200614078007A
:10B740000080FB004801DD000E0890008080E800CA
:10B75000C0862200614078000080FB0000004100AC
:10B76000600798004E0090000000E000BDFF32002E
:10B7700072004700104078008080FB0030F22F00FC
:10B7800000804000600798004E009000000F980075
:10B790000B0037008E0890006E0090000081400082
:10B7A0008E089000C0862200E1407800C08622000A
:10B7B000017178000E0890000000E900000F980069
:10B7C0008E0890005E009000808F5000F1FF3D00D9
:10B7D0000000EB00000F98000C003700DE00900026
:10B7E0000E089000008140008E0890007200470013
:10B7F0000080400090407800C086220001717800EF
:10B800000E0890000000E800000F98008E089000DD
:10B810006E009000808F5000F0FF3500440037002C
:10B82000907D2A0077FE07000000E000050032004E
:10B83000C1F90700807D2A0034D00200000000001A
:10B840003B003700D07D2A006EFE07000000E000BC
:10B850000200320019FE070035003700207E2A0062
:10B8600068FE07000000E0000400320040AE8100E6
:10B870000090A10040AE89002D003700707E2A00A4
:10B8800060FE07000000E0001F0032000000EB0037
:10B89000000F9800170037000000EB0070079800B9
:10B8A0000E0037008E0890007E00900080804000DF
:10B8B000C0862200614078000080FB0002D30200B5
:10B8C0000000000000C2B300FED302000000000030
:10B8D0007E0090000000E800700798007E00900055
:10B8E000EF0F5000EFFF34000E0890007000400092
:10B8F000000F98008E089000F03F2000808F5000CD
:10B90000E5FF34000A003700D07E2A003DFE070024
:10B910000000E000020032000700070004003700CA
:10B92000C1002000503A2000BAF8020000000000D8
:10B930000080FA00000006000200FA000000EB00A0
:10B94000000F7800050037001E017800C186220034
:10B950000040EB0000F178001E0FE800F03F2000EF
:10B960009E0F1000F8FF3400C186220010CEB300F5
:10B9700080487800D186220000C0EB008048780023
:10B98000E186220000C0EB0080487800F1862200AA
:10B9900010CAB300804878000080FA00000006005A
:10B9A0005752490054452000424954003A20200093
:10B9B0002A6E650078742000636C6F00636B200052
:10B9C000285E2900207769006C6C20007573650083
:10B9D000207468006973200076616C0075654E0004
:10B9E0006F2064006576690063652C002074720026
:10B9F00079202800414C4100524D29002053450038
:10BA00004152430048206D00616372006F20660060
:10BA1000697273007441440044524500535320003E
:10BA20004D414300524F200020302E004D616300F5
:10BA3000726F20006D656E00754D610063726F005E
:10BA4000202020002020310057495200452061006D
:10BA500064647200657373000D0A200020202A00C0
:10BA60003157490052452000524F4D0020434F00AE
:10BA70004D4D41004E4420004D414300524F730054
:10BA80003A0D0A00203531002E5245004144200075
:10BA9000524F4D00202830007833330029202A00EF
:10BAA000666F7200207369006E676C006520640029
:10BAB0006576690063652000627573000D0A2000D9
:10BAC00038352E004D41540043482000524F4D0060
:10BAD000202830007835350029202A00666F6C0058
:10BAE0006C6F770065642000627920003634620054
:10BAF000697420006164640072657300730D0A004C
:10BB000020323000342E53004B49500020524F0059
:10BB10004D20280030784300432920002A666F001A
:10BB20006C6C6F00776564002062790020636F00A1
:10BB30006D6D61006E640D000A20320033362E00F8
:10BB4000414C4100524D20005345410052434800B2
:10BB50002028300078454300290D0A0020323400A7
:10BB6000302E53004541520043482000524F4D00B3
:10BB7000202830007846300029414C0041524D00C9
:10BB800020534500415243004820280030784500AA
:10BB90004329530045415200434820002830780093
:10BBA00046302900446576006963650020494400F9
:10BBB000732061007265200061766100696C61002C
:10BBC000626C650020627900204D410043524F00B5
:10BBD0002C20730065652000283029002E52450076
:10BBE00041442000524F4D0020283000783333006C
:10BBF000293A20004D41540043482000524F4D0047
:10BC0000202830007835350029534B00495020005A
:10BC1000524F4D00202830007843430029556E00D4
:10BC20006B6E6F00776E20006D616300726F2C0089
:10BC30002074720079203F00206F720020283000AD
:10BC4000292066006F72200068656C007042550004
:10BC500053205200455345005420570061726E0036
:10BC6000696E67003A202A0053686F0072742000E2
:10BC70006F7220006E6F200070756C006C2D750067
:10BC800070202A004E6F20006465760069636500AD
:10BC9000206465007465630074656400204453008B
:10BCA0003138530032302000486967006820500066
:10BCB0007265730020446900672054006865720053
:10BCC0006D445300313842003230200050726F0012
:10BCD00067205200657320004469670020546800A3
:10BCE00065726D00445331003832320020456300E4
:10BCF0006F6E2000446967002054680065726D0013
:10BD00004453320034303400204563006F6E7200BB
:10BD1000616D200074696D006520430068697000E2
:10BD2000445332003433310020314B00204545006C
:10BD300050524F004D556E006B6E6F00776E2000B5
:10BD4000646576006963650050574D0020646900A2
:10BD5000736162006C656400314B48007A2D3400D9
:10BD60002C303000304B48007A205000574D4600B0
:10BD70007265710075656E0063792000696E200040
:10BD80004B487A002050720065736300616C650057
:10BD90003A505200323A44007574790020637900B9
:10BDA000636C650020696E002025200050574D000F
:10BDB000206163007469760065455200524F52005D
:10BDC0003A205000574D2000616374006976650089
:10BDD0002C20670020746F0020646900736162008A
:10BDE0006C6541005558200046726500717565000C
:10BDF0006E6379003A20410055582000494E5000AA
:10BE000055542F0048492D005A41550058204800EC
:10BE10004947480041555800204C4F0057564F00A5
:10BE20004C544D004554450052204D004F444500B0
:10BE3000564F4C005441470045205000524F42009D
:10BE4000453A200056457200726F72002829200082
:10BE5000406C69006E653A0020407000676D7300A9
:10BE600070616300653A20006279740065732E008A
:10BE7000546F6F00206C6F006E67210053796E0065
:10BE80007461780020657200726F72004E6F20003E
:10BE900045455000524F4D004572610073696E0078
:10BEA00067646F006E655300617669006E672000FD
:10BEB000746F2000736C6F00742049006E7661000F
:10BEC0006C69640020736C006F744C006F616400D7
:10BED000696E6700206672006F6D2000736C6F00E2
:10BEE0007420450052524F00523A2000636F6D009B
:10BEF0006D616E0064206800617320006E6F200029
:10BF000065666600656374002068650072654100BF
:10BF1000434B4E0041434B004932430020535400F1
:10BF200041525400204249005449320043205300FA
:10BF3000544F5000204249005449320043206D00C4
:10BF40006F6465003A0D0A0020312E0020536F0007
:10BF500066747700617265000D0A2000322E2000A1
:10BF60004861720064776100726553006574200057
:10BF70007370650065643A000D0A2000312E2000C0
:10BF80007E354B00487A0D000A2032002E207E00BC
:10BF900035304B00487A0D000A2033002E207E00F9
:10BFA000313030004B487A000D0A2000342E20003A
:10BFB0007E343000304B48007A574100524E4900E1
:10BFC0004E473A0020484100524457004152450034
:10BFD000204932004320690073206200726F6B00B9
:10BFE000656E20006F6E2000746869007320500039
:10BFF00049432100202852004556200041332900A2
:10C000005365740020737000656564003A0D0A0082
:10C0100020312E0020313000304B48007A0D0A00CC
:10C0200020322E0020343000304B48007A0D0A00B8
:10C0300020332E0020314D00487A49003243200041
:10C04000286D6F0064207300706429003D28200073
:10C0500020302E004D616300726F20006D656E0010
:10C06000750D0A0020312E003762690074206100CE
:10C07000646472006573730020736500617263000D
:10C08000680D0A0020322E004932430020736E00F2
:10C090006966660065720D000A2033002E436F004A
:10C0A0006E6E650063742000746F20006F6E2D004B
:10C0B000626F61007264200045455000524F4D0090
:10C0C0000D0A2000342E45006E6162006C65200070
:10C0D0005772690074696E006720740068652000FB
:10C0E0006F6E2D00626F6100726420004545500044
:10C0F000524F4D005365610072636800696E6700BE
:10C10000204932004320610064647200657373004B
:10C1100020737000616365002E2046006F756E000D
:10C1200064206400657669006365730020617400B3
:10C130003A536E0069666600657243006F6D6D006C
:10C14000616E64006D6F6400653F0D000A312E0062
:10C15000203662002F313400620D0A00322E20009A
:10C1600034622F003136620044656C0061793F0013
:10C1700050494300286D6F00642064006C792900E9
:10C180003D2843004D44440054416E006F2072002E
:10C1900065616400756E6B006E6F77006E206D00D8
:10C1A0006F646500283129002067650074206400F1
:10C1B000657649004444650076494400203D2000EE
:10C1C0002052650076203D00204E6F0074206900EB
:10C1D0006D706C00656D65006E74650064202800EC
:10C1E0007965740029506C006561730065206500F5
:10C1F000786974002050490043207000726F670016
:10C2000072616D006D696E0067206D006F6465007E
:10C210002842410053494300295265006164790076
:10C22000612F41002F402000636F6E0074726F0019
:10C230006C73200041555800207069006E612F001A
:10C24000412F400020636F006E7472006F6C7300AA
:10C2500020435300207069006E436F006D6D6100D4
:10C260006E6420006E6F740020757300656420009A
:10C27000696E20007468690073206D006F6465004A
:10C2800050756C006C2D750070207200657369002C
:10C2900073746F00727320004F46460050756C0037
:10C2A0006C2D7500702072006573690073746F00E7
:10C2B000727320004F4E5300656C66002D7465004C
:10C2C00073742000696E200048695A00206D6F0069
:10C2D000646520006F6E6C00795245005345540030
:10C2E000424F4F00544C4F004144450052415500CD
:10C2F000582049004E505500542F4800492D5A00EF
:10C300002C205200454144003A2050004F57450030
:10C3100052205300555050004C49450053204F00C7
:10C320004E504F00574552002053550050504C007E
:10C3300049455300204F46004644410054412000E7
:10C340005354410054453A00204445004C415900A3
:10C35000207573005752490054453A002052450059
:10C3600041443A0020434C004F434B002C20310005
:10C37000434C4F00434B2C002030440041544100BB
:10C38000204F550054505500542C2000314441009A
:10C39000544120004F555400505554002C2030007B
:10C3A000202A7000696E2000697320006E6F77008C
:10C3B000204869005A434C004F434B002054490029
:10C3C000434B53003A20520045414400204249006B
:10C3D000543A200053796E00746178002065720031
:10C3E000726F720020617400206368006172200027
:10C3F000782E2000657869007428770069746800D9
:10C400006F75740020636800616E670065296E00B7
:10C410006F206D006F64650020636800616E6700C7
:10C4200065233A00204E6F0020736F00667477001A
:10C43000617265002072650073657400206F6E0084
:10C44000207634002C207500736520007468650028
:10C4500020726500736574002062750074746F004B
:10C460006E2E4E006F6E65007869730074656E0005
:10C4700074207000726F74006F636F006C2178001D
:10C480002E206500786974000D0A49006E766100FF
:10C490006C696400206368006F696300652C20008C
:10C4A000747279002061670061696E00444556002E
:10C4B00049443A0068747400703A2F002F64610098
:10C4C0006E676500726F7500737072006F746F0035
:10C4D0007479700065732E00636F6D002A2D2D0036
:10C4E0002D2D2D002D2D2D002D2D2A004F70650096
:10C4F0006E206400726169006E206F0075747000B8
:10C5000075747300202848003D4869002D5A2C009E
:10C51000204C3D00474E4400294E6F00726D610073
:10C520006C206F00757470007574730020284800CB
:10C530003D332E0033762C00204C3D00474E440006
:10C54000294D53004220730065743A00204D4F007E
:10C5500053542000736967002062690074206600EC
:10C5600069727300744C53004220730065743A0082
:10C57000204C45004153540020736900672062003D
:10C58000697420006669720073742000426F6F0046
:10C59000746C6F00616465007220760020312E009B
:10C5A00020484500580D0A0020322E002044450046
:10C5B000430D0A0020332E00204249004E0D0A0090
:10C5C00020342E00205241005744690073706C00E3
:10C5D00061792000666F72006D61740020736500E0
:10C5E00074566F006C746100676520006D6F6E009B
:10C5F00069746F0072733A00203556003A202000AB
:10C600007C2033002E3356003A2020007C20560038
:10C6100050554C004C5550003A2053006574200092
:10C620007365720069616C0020706F007274200085
:10C630007370650065643A002028620070732900F9
:10C640000D0A2000312E2000333030000D0A20006A
:10C65000322E200031323000300D0A0020332E00FF
:10C660002032340030300D000A2034002E203400F7
:10C67000383030000D0A2000352E200039363000C9
:10C68000300D0A0020362E002031390032303000C3
:10C690000D0A2000372E20003338340030300D00D2
:10C6A0000A2038002E20350037363000300D0A00C1
:10C6B00020392E002031310035323000300D0A0093
:10C6C00031302E0020496E007075740020437500D3
:10C6D00073746F006D204200415544000D0A310013
:10C6E000312E2000417574006F2D42006175640089
:10C6F000204465007465630074696F006E20280033
:10C700004163740069766900747920005265710094
:10C71000756972006564290041646A00757374006C
:10C7200020796F0075722000746572006D696E006B
:10C73000616C410072652000796F7500207375008F
:10C7400072653F002043460047313A0020434600CF
:10C7500047323A00285C2D002F5F5C002D2928000D
:10C760005C5F2F002D295300656C65006374200009
:10C770006F757400707574002074790070653A00EC
:10C780000D0A2000312E20004F7065006E206400DD
:10C79000726169006E202800483D4800692D5A00EA
:10C7A0002C204C003D474E0044290D000A20320049
:10C7B0002E204E006F726D00616C200028483D00F5
:10C7C000332E3300562C20004C3D47004E442900A8
:10C7D00052325700202873007064200068697A0084
:10C7E000293D2800202030002E4D610063726F002B
:10C7F000206D65006E750D000A2031002E49530032
:10C800004F37380031362D003320410054520D008F
:10C810000A2032002E4953004F37380031362D00A0
:10C82000332070006172730065206F006E6C7900B8
:10C8300049534F002037380031362D003320410056
:10C84000545220002852450053455400206F6E007A
:10C8500020435300290D0A0052455300455420003F
:10C8600048494700482C2000434C4F00434B2000D0
:10C87000544943004B2C200052455300455420009E
:10C880004C4F570049534F002037380031362D00A8
:10C890003320720065706C00792028007573650084
:10C8A0007320630075727200656E7400204C530033
:10C8B0004220730065747400696E6700293A200095
:10C8C00050726F00746F63006F6C3A0020736500E4
:10C8D000726961006C332000776972006532200054
:10C8E000776972006552460055756E006B6E6F0079
:10C8F000776E5200656164002074790070653A00BB
:10C9000020746F0020656E006476610072696100BA
:10C91000626C6500206C65006E677400684461009D
:10C9200074612000756E690074733A00206E6F00A8
:10C9300020696E0064696300617469006F6E440071
:10C940006174610020756E00697420006C656E0072
:10C95000677468002028620069747300293A200017
:10C9600043532000454E4100424C45004443530090
:10C9700020444900534142004C4544005233570083
:10C98000202873007064200063736C0020686900C5
:10C990007A293D00282029000D0A440069736300AC
:10C9A0006F6E6E006563740020616E007920640014
:10C9B00065766900636573000D0A43006F6E6E0053
:10C9C000656374002028410044432000746F2000F8
:10C9D0002B332E0033562900437472006C415500EE
:10C9E000584D4F00444520004C45440050554C00E4
:10C9F0004C55500020485000554C4C0055502000DC
:10CA00004C5652004547410044432000616E64008B
:10CA10002073750070706C007935560056505500C3
:10CA2000332E3300564144004342750073206800A2
:10CA30006967680042757300204869002D5A20001C
:10CA40003042750073204800692D5A0020314D0096
:10CA50004F4445002C205600524547002C206100D1
:10CA60006E64200055534200204C45004473200062
:10CA700073686F00756C640020626500206F6E0043
:10CA800021466F00756E64002020650072726F0091
:10CA900072732E004D4F530049434C004B4D4900DB
:10CAA000534F430053204F004B20460041494C0058
:10CAB0005365740020737000656564003A0D0A00C8
:10CAC00020312E00203330004B487A000D0A200020
:10CAD000322E2000313235004B487A000D0A2000FA
:10CAE000332E2000323530004B487A000D0A2000EA
:10CAF000342E2000314D48007A436C006F636B0088
:10CB000020706F006C617200697479003A0D0A0040
:10CB100020312E00204964006C6520006C6F770086
:10CB2000202A640065666100756C74000D0A20009F
:10CB3000322E200049646C00652068006967680037
:10CB40004F7574007075740020636C006F636B0028
:10CB50002065640067653A000D0A2000312E200030
:10CB600049646C00652074006F2061006374690083
:10CB700076650D000A2032002E20410063746900A2
:10CB800076652000746F200069646C0065202A00BF
:10CB90006465660061756C0074496E0070757400A0
:10CBA000207361006D706C00652070006861730017
:10CBB000653A0D000A2031002E204D0069646400A2
:10CBC0006C6520002A646500666175006C740D0058
:10CBD0000A2032002E2045006E6453005049200088
:10CBE00028737000642063006B702000736B650015
:10CBF00020736D0070206300736C200068697A00F8
:10CC0000293D2800202030002E4D610063726F0006
:10CC1000206D65006E750D000A2031002E536E00E8
:10CC20006966660020435300206C6F00770D0A0090
:10CC300020322E00536E690066662000616C6C0025
:10CC4000207472006166660069632D0070202D00FB
:10CC500066202A00427974006573200064726F00B8
:10CC600070706500642A460041494C0045442C0020
:10CC7000204E4F0020444100544144006174610043
:10CC80002062690074732000616E6400207061008E
:10CC900072697400793A0D000A2031002E203800A4
:10CCA0002C204E004F4E4500202A6400656661002E
:10CCB000756C7400200D0A0020322E0020382C00E4
:10CCC00020455600454E20000D0A2000332E20003E
:10CCD000382C20004F444400200D0A0020342E0040
:10CCE00020392C00204E4F004E455300746F7000C9
:10CCF0002062690074733A000D0A2000312E200072
:10CD000031202A006465660061756C00740D0A00AC
:10CD100020322E002032520065636500697665007E
:10CD200020706F006C617200697479003A0D0A001E
:10CD300020312E00204964006C65200031202A003B
:10CD40006465660061756C00740D0A0020322E0067
:10CD5000204964006C652000305541005254200089
:10CD600028737000642062007267200064627000A3
:10CD7000207362002072780070206800697A2900B0
:10CD80003D28200020302E004D616300726F20008E
:10CD90006D656E00750D0A0020312E005472610021
:10CDA0006E737000617265006E74200062726900BB
:10CDB000646765000D0A2000322E4C00697665001C
:10CDC000206D6F006E6974006F720D000A203300D1
:10CDD0002E427200696467006520770069746800FC
:10CDE00020666C006F772000636F6E0074726F00B6
:10CDF0006C0A0D0020342E00417574006F20420033
:10CE000061756400204465007465630074696F0097
:10CE10006E202800416374006976690074792000EF
:10CE20004E65650064656400295541005254200038
:10CE30006272690064676500526573006574200062
:10CE4000746F200065786900745261007720550086
:10CE50004152540020696E007075740055415200B3
:10CE600054204C00495645002044490053504C0082
:10CE700041592C00207D2000544F200053544F0076
:10CE8000504C49005645200044495300504C410045
:10CE900059205300544F5000504544005741520010
:10CEA0004E494E00473A200070696E0073206E00B4
:10CEB0006F7420006F7065006E20640072616900FD
:10CEC0006E20280048695A00292052004556490022
:10CED000443A0D000A496E0076616C0069642000D6
:10CEE00063686F00696365002C207400727920000C
:10CEF00061676100696E6D0073525300204C4F00F2
:10CF0000572C2000434F4D004D414E0044204D0012
:10CF10004F4445005253200048494700482C200008
:10CF20004441540041204D004F4445004164640099
:10CF30007265730073206F0066205000434638000E
:10CF4000353734003F546800697320006D6F64000A
:10CF5000652072006571750069726500732061005B
:10CF60006E20610064617000746572004C4344007F
:10CF70002074790070653A000D0A2000312E2000DF
:10CF80004844340034373800302028007573690075
:10CF90006E67200050434600383537003420490082
:10CFA0004F206500787061006E64650072294C0046
:10CFB000434420002874790070206100646472008A
:10CFC00029203D002028200020302E004D616300E4
:10CFD000726F20006D656E00750D0A0020312E0005
:10CFE0004C43440020526500736574000D0A200014
:10CFF000322E49006E697400204C4300440D0A0033
:10D0000020332E00436C6500617220004C434400C5
:10D010000D0A2000342E4300757273006F722000D9
:10D02000706F7300697469006F6E200065783A0054
:10D030002834290020300D000A2036002E577200B7
:10D040006974650020746500737420006E756D004E
:10D050006265720073206500783A28003629200046
:10D0600038300D000A2037002E57720069746500B1
:10D07000207465007374200063686100726163004E
:10D080007465720073206500783A28003729200003
:10D0900038304400697370006C617900206C69005D
:10D0A0006E6573003A0D0A0020312E0020312000F9
:10D0B0000D0A2000322E20004D756C00746970003E
:10D0C0006C6549004E495400434C450041524300B1
:10D0D000555253004F522000534554004E6F2000CC
:10D0E00041434B002C206300686563006B206100A6
:10D0F0006461700074657200434C4B00094D4F0031
:10D1000053490900435309004D4953004F506900EA
:10D110006E73740061746500733A47004E440900F1
:10D12000332E3300560935002E3056000941440095
:10D13000430956005055090041555800095009004F
:10D14000500950000949090049092D00094F5700AD
:10D1500044092D00092D2D000954780044092D00A3
:10D1600009527800445343004C09530044410900DC
:10D170002D092D00504743000950470044092D0058
:10D18000092D31002E28420052290900322E280094
:10D190005244290009332E00284F52002909340037
:10D1A0002E28590057290900352E2800474E2900FE
:10D1B00009362E0028424C00290937002E2850003D
:10D1C00055290900382E28004752290009392E0018
:10D1D00028575400290930002E2842006C6B290082
:10D1E000474E440009474E004409410044430900AA
:10D1F000352E3000560933002E33560009565000A4
:10D20000550941005558090065786500637574003B
:10D2100065203A0020205400494D45004F555400E8
:10D2200020302E00204D610063726F00206D65007C
:10D230006E750D000A2031002E204C0069766500C5
:10D2400020696E0070757400206D6F006E69740047
:10D250006F7249006E70750074206D006F6E69000A
:10D26000746F72002C2061006E7920006B6579006C
:10D270002065780069747300202A7300746172005D
:10D28000746269007420650072726F0072202A0057
:10D29000706172006974790020657200726F7200AB
:10D2A000202A7300746F7000626974002065720038
:10D2B000726F7200204E4F004E452000554E4B00BD
:10D2C0004E4F57004E20450052524F0052206100F1
:10D2D00075746F0072616E00676520002B4D480009
:10D2E0007A292B006B487A0029496E00707574000A
:10D2F0002061200063757300746F6D00204241004F
:10D300005544200072617400653A570041524E0046
:10D31000494E47003A2050006F73730069626C00F9
:10D32000652062007566660065726F007665720042
:10D33000666C6F0077416E0079206B006579200084
:10D34000746F200065786900745370006163650034
:10D3500020746F0020636F006E7469006E75650045
:10D360004E756D0062657200206F66002062690074
:10D370007473200072656100642F77007269740015
:10D38000653A200043533A000D0A2000312E200058
:10D3900043530D000A2032002E202F00435320005B
:10D3A0002A646500666175006C7450006F736900D3
:10D3B00074696F006E2069006E20640065677200FA
:10D3C0006565730053657200766F200061637400B9
:10D3D00069766500233132002020200020092300D7
:10D3E000313120002020200009233100302020008E
:10D3F000202009002330390020202000092330009C
:10D400003820200020092300303720002020090088
:10D410002330360020202000092330003520200052
:10D42000200923003034200020200900233033005D
:10D430002020200009233000322020002009230072
:10D4400030312000202047004E440900352E3000A6
:10D45000560933002E335600095650005509410035
:10D4600044430900415558003209410055583100E4
:10D47000094155005809430053094D0049534F00D5
:10D4800009434C004B094D004F5349002D092D0015
:10D49000092D09004F5744002D0952007844090016
:10D4A0002D09540078442D00092D090053434C00E8
:10D4B00009534400412D09002D095000474309003C
:10D4C00050474400612F41002F402000636F6E00E1
:10D4D00074726F006C732000415558003120700049
:10D4E000696E61002F412F00402063006F6E740051
:10D4F000726F6C0073204100555832002070690033
:10D500006E45450050524F004D5343004C5344006C
:10D51000415750005245410044265700524954009B
:10D520004556750073625300656C65006374200096
:10D530005670750020285000756C6C0075702900BD
:10D5400020536F0075726300653A0D000A203100A8
:10D550002920450078746500726E61006C202800F7
:10D560006F7220004E6F6E0065290D000A20320098
:10D5700029204F006E626F006172640020332E001C
:10D5800033760D000A20330029204F006E626F00B1
:10D590006172640020352E00307620006F6E2D0001
:10D5A000626F61007264200070756C006C757000B1
:10D5B00020766F006C74610067652000656E610005
:10D5C000626C650064646900736162006C6564008C
:10D5D0004E6F72006D616C0020746F0020657800E2
:10D5E0006974570061697400696E670020616300A7
:10D5F00074697600697479002E2E2E002A2A200084
:10D60000456172006C7920004578690074212A0018
:10D610002A204200617564003E3136006D3A2000D8
:10D620005468650020425000206361006E6E6F00F8
:10D6300074206D0065617300757265002061620081
:10D640006F766500203136003030300030303000E9
:10D650002C2044006F6E65002E0A0D0043616C00A3
:10D6600063756C0061746500643A2000090A0D005E
:10D6700045737400696D6100746564003A20200090
:10D680000920620070734700656E650072616C006E
:10D690000909090009095000726F74006F636F0077
:10D6A0006C2069006E7465007261630074696F00BC
:10D6B0006E2D2D002D2D2D002D2D2D002D2D2D000D
:10D6C0002D2D2D002D2D2D002D2D2D002D2D2D003E
:10D6D0002D2D2D002D2D2D002D2D2D002D2D2D002E
:10D6E0002D2D2D002D2D2D002D2D2D002D2D2D001E
:10D6F0002D2D2D002D2D2D002D2D2D002D2D2D000E
:10D700002D2D2D002D2D2D002D2D2D002D2D2D00FD
:10D710002D2D2D002D3F09005468690073206800ED
:10D72000656C70000909090028302900094C69005E
:10D73000737420006375720072656E0074206D0052
:10D74000616372006F733D00582F7C0058094300DD
:10D750006F6E760065727400732058002F7265003A
:10D760007665720073652000580909002878290041
:10D77000094D610063726F0020787E0009536500D7
:10D780006C66740065737400090909005B09530035
:10D7900074617200746F090053657400206F750026
:10D7A00074707500742074007970650009090900AF
:10D7B0005D095300746F700024094A00756D700094
:10D7C00020746F0020626F006F746C006F616400E2
:10D7D00065720900097B09005374610072742000AE
:10D7E000776974006820720065616400262F250047
:10D7F000094465006C6179002031200075732F00A9
:10D800006D73090009097D00095374006F70610090
:10D810002F412F004009410055585000494E20002B
:10D82000286C6F00772F4800492F52004541440073
:10D8300029090900226162006322090053656E0014
:10D8400064207300747269006E676200095365009A
:10D8500074206200617564007261740065090900DA
:10D860000931320033095300656E640020696E008F
:10D87000746567006572200076616C0075656300F1
:10D880002F432F006B2F4B0009415500582061009A
:10D8900073736900676E6D00656E74002028410027
:10D8A000302F4300532F4100312F4100322909000E
:10D8B000307831003233090053656E00642068000F
:10D8C0006578200076616C00756564002F4409005E
:10D8D0004D6561007375720065204100444320006E
:10D8E000286F6E0063652F00434F4E00542E2900B1
:10D8F0000930620031313000095365006E64200048
:10D9000062696E0061727900207661006C75650055
:10D9100066094D00656173007572650020667200CE
:10D9200065717500656E630079090900720952001E
:10D9300065616400672F5300094765006E657200DA
:10D9400061746500205057004D2F530065727600BA
:10D950006F0909002F0943004C4B200068696800DB
:10D9600009436F006D6D61006E6468006973740037
:10D970006F727900090909005C0943004C4B2000D3
:10D980006C6F690009566500727369006F6E6900FB
:10D990006E666F002F7374006174750073696E009A
:10D9A000666F0900095E0900434C4B002074690052
:10D9B000636B6C002F4C0900426974006F72640045
:10D9C00065722000286D7300622F4C0053422900BD
:10D9D00009092D000944410054206800696D0900BF
:10D9E000436861006E676500206D6F006465090023
:10D9F00009095F000944410054206C006F6509006B
:10DA000053657400205075006C6C750070204D00DB
:10DA1000657468006F640900092E090044415400D0
:10DA200020726500616470002F50090050756C0011
:10DA30006C7570002072650073697300746F7200FA
:10DA4000732028006F6666002F4F4E0029092100C1
:10DA50000942690074207200656164007309530013
:10DA60006372690070742000656E6700696E6500FE
:10DA7000090909003A0952006570650061742000C7
:10DA8000652E67002E2072003A313000760953006F
:10DA9000686F770020766F006C7473002F737400CA
:10DAA00061746500730909003B09420069747300E1
:10DAB00020746F002072650061642F007772690026
:10DAC00074652000652E67002E2030007835350003
:10DAD0003B3277002F5709005053550020286F0024
:10DAE00066662F004F4E290009093C00783E2F0042
:10DAF0003C783D00203E2F003C303E00095573002D
:10DB000065726D00616372006F2078002F61730091
:10DB1000736967006E2078002F6C690073742000B1
:10DB2000616C6C000200FA00000F78009E00780023
:10DB30000040EB00804878009E0078000040EB0039
:10DB4000904098001E0178006000B8001001980015
:10DB5000210198009E0078000000EB00B0009800C2
:10DB60009E0078000040EB00B04898009E007800CE
:10DB70000040EB00804898009E00780010C0B30081
:10DB8000904898009E00780010C0B300A04898000C
:10DB90001E0178006000B800000998001109980083
:10DBA0009E0078000000EB00A00898001E0178009D
:10DBB0006000B80060019800710198000000EB005F
:10DBC0000080FA00000006000200FA00000F780052
:10DBD0000080FA00000006000800FA00008FBE0076
:10DBE00072002000030020003E004100AE8049008A
:10DBF00020079800310798002E009000BE0090008A
:10DC0000E00F5000E08F580006003D002E0190000C
:10DC1000BE01900067014100E081490022079800A1
:10DC2000330798002E019000BE0190004D1ADD00D0
:10DC30004310DE0000007200C398DE000080FA008E
:10DC4000000006000200FA00000F78009E00780035
:10DC50001000200002FB0200000000008000EB002A
:10DC60000000EB0002FB0200000000001100200099
:10DC70000000EB0002FB0200000000000080FA0040
:10DC8000000006000C00FA00200798006147980089
:10DC90000000EB00000F78006E4090000004E000F0
:10DCA00017003A0010002000E6FF07000000EB001C
:10DCB000100798000B0037008000EB000000EB001D
:10DCC00002FB020000000000110020000000EB0039
:10DCD00002FB0200000000001E0090000000E800AF
:10DCE000100798001E009000E40F5000F2FF34006F
:10DCF000AE0090000040EB0080487800080137003B
:10DD00002E009000904078006E40900080CF500030
:10DD1000110032006E409000E74F500004003A00BE
:10DD20002E00900010407800E64F500007003A00A7
:10DD30006E409000EE4F500007003A002E00900019
:10DD400010407800ED4F50000300320050002000DA
:10DD5000000F7800F20037002E009000904078000D
:10DD60006E40900080CF5000E8003A006E40900076
:10DD7000E64F500006003A0010002000B1FF0700F7
:10DD8000AE00900070C0B30080487800DF0037001C
:10DD90006E409000ED4F5000DC003A001000200073
:10DDA000A8FF0700AE009000E0C0B30080487800F4
:10DDB000D60037002E009000104078000080FB0055
:10DDC0006101B9004207980053079800F000200055
:10DDD000010020004E019000DE019000800F5100F4
:10DDE000818F5900C4003E004E009000DE0090007C
:10DDF000006001000F0037001400370019003700E1
:10DE000027003700350037003A0037004800370058
:10DE10004D0037005B003700690037006E003700A7
:10DE20007C003700810037008F00370094003700F6
:10DE3000A20037000000EB0082FF0700AE00900058
:10DE400010C0B30080487800B000370010002000F8
:10DE50007CFF0700AE00900020C0B300804878002F
:10DE6000AA0037006E409000E84F500006003600D0
:10DE70001000200073FF0700AE00900090C0B300B8
:10DE800080487800A10037000000EB006DFF07001C
:10DE9000AE00900030C0B300804878009B0037008F
:10DEA0006E409000E44F500006003A000000EB0086
:10DEB00064FF0700AE00900040C0B30080487800C7
:10DEC00092003700100020005EFF0700AE009000B7
:10DED00050C0B300804878008C003700100020004C
:10DEE00058FF0700AE00900050C0B3008048780093
:10DEF000860037006E409000E64F500006003A0062
:10DF00000000EB004FFF0700AE00900060C0B300C0
:10DF1000804878007D0037001000200049FF07008E
:10DF2000AE00900080C0B3008048780077003700D2
:10DF30001000200043FF0700AE00900070C0B30047
:10DF400080487800710037006E409000E44F500028
:10DF500006003A000000EB003AFF0700AE00900018
:10DF600040C0B300804878006800370010002000EF
:10DF700034FF0700AE00900080C0B30080487800F6
:10DF8000620037006E409000E14F500006003A00FA
:10DF90000000EB002BFF0700AE00900010C0B300A4
:10DFA00080487800590037001000200025FF070046
:10DFB000AE00900020C0B3008048780053003700C6
:10DFC0000000EB001FFF0700AE009000A0C0B300F0
:10DFD000804878004D0037006E409000EB4F5000B5
:10DFE00006003A000000EB0016FF0700AE009000AC
:10DFF000B0C0B30080487800440037001000200013
:10E0000010FF0700AE009000C0C0B3008048780049
:10E010003E003700100020000AFF0700AE0090000D
:10E02000C0C0B30080487800380037006E409000D0
:10E03000ED4F500006003A000000EB0001FF070022
:10E04000AE009000D0C0B300804878002F003700A9
:10E0500010002000FBFE0700AE009000F0C0B300EF
:10E06000804878002900370010002000F5FE0700E6
:10E07000AE009000E0C0B300804878002300370075
:10E080006E409000EB4F500006003A000000EB009D
:10E09000ECFE0700AE009000B0C0B30080487800EE
:10E0A0001A00370010002000E6FE0700AE009000C6
:10E0B000F0C0B30080487800140037006E40900034
:10E0C000E14F500006003A000000EB00DDFE0700C3
:10E0D000AE00900010C0B300804878000B003700FD
:10E0E00010002000D7FE0700AE00900020C0B30053
:10E0F000804878000500370050002000000F7800AD
:10E100002E009000EE409000014878002E00900014
:10E11000904078006E40900080CF500025FF3A007C
:10E120001E0078000080FA00000006001400FA00CB
:10E13000500798006107980072079800030F980035
:10E14000140F98000000EB00300798000E089000B4
:10E150000000E0000A0032007E009000900078008D
:10E160000E089000010878000E0890008080E800FA
:10E170007E0090001000780000804000300798007A
:10E180007E0090008080E8007E0090001000780003
:10E1900000804000400798004F0037004E0090007C
:10E1A0000000E900400798004E0090009040780081
:10E1B000414798000040EB00304798000000EB001A
:10E1C000000F7800330037005E009000EE009000F2
:10E1D00061005000E08058005007980061079800E7
:10E1E0001E0890000000E000090032005E00900070
:10E1F000EE009000E00F5000E08F580004003A005D
:10E20000110020001000200002FB020000000000AE
:10E210004E4090000080FB00E100600020002000E4
:10E2200002FB0200000000004E4090000080FB0056
:10E230000000D100404798008000EB000000EB0098
:10E2400002FB0200000000003E0090000000E00021
:10E250000B003200C2FB02000000000020479800C3
:10E260002E4090008080FB001E0078000008DD003A
:10E27000804078003E40900000C070003047980019
:10E28000110020000000EB0002FB02000000000073
:10E290001E0FE8005E009000EE009000E00F5000BE
:10E2A000E08F580003003200700020009E0F100025
:10E2B000C5FF34003E0090000000E0000600320080
:10E2C0003E0090000000E900300798003E009000FA
:10E2D000BE409000014878005E009000EE00900083
:10E2E000E00F5000E08F5800ACFF3A000080FA00C9
:10E2F000000006001C00FA0040079800214F98001B
:10E300006207980073079800040F9800150F980093
:10E31000260F9800370F98000000EB003007980098
:10E320000000EB00200798000040EB002047980019
:10E330000000EB00500F9800AE4890000EF89700D8
:10E3400080CF50000200320014002000540F9800CB
:10E350005E089000000F78006E009000FE009000B4
:10E36000E00F5000E08F58000D003A002EB89700E3
:10E37000BEB89700E00F5000E08F580066003200F2
:10E3800011C0B3004E0090003EFE07002EB897006B
:10E39000BEB89700D2FB0200000000005E0037000C
:10E3A000AE4890004E00900036FE07001E02780036
:10E3B0009E0990000E0990006E009000FE009000F3
:10E3C0005AFF07002E0890000000E0000C00320009
:10E3D0003E0990009E0890002E089000C8F60200AA
:10E3E00000000000800078000000EB00200798008B
:10E3F0000100E00002003A00100020002007980011
:10E400001E00E000330032004E0090001040780003
:10E410008040E8004E009000014878002E009000F7
:10E420000000E0001C0032002EB89700BEB8970034
:10E43000E00F5000E08F580017003200AE4090000F
:10E440002EF0970080CF50001300310061C0B30060
:10E450004E0090000BFE070041C0B3004E0090003C
:10E4600008FE07002EB89700BEB89700C289DE00EC
:10E470004E0ADD004201DE00020172002EB8970054
:10E48000BEB89700000041008180490020BF9F0076
:10E4900031BF9F00030037008EF897004E009000B8
:10E4A000F8FD07002EB89700BEB89700E00F5000A7
:10E4B000E08F58000700320011C0B3004E009000FA
:10E4C000F0FD07002EB89700BEB89700D2FB0200FF
:10E4D000000000002E0090000000E0000E0032005E
:10E4E0000040EB00005F9800AE4090002EF09700D7
:10E4F00080CF50000200310014C0B300045F9800C8
:10E500002E4090000040E800204798000E589000F0
:10E510000004E000A2FF3A002E0090000000E0009E
:10E520000C0032002EF097000004E00007003200DB
:10E53000AE4090002EF0970080CF500003003600D0
:10E540003000200030079800020037002000200033
:10E55000300798003E0090000080FA00000006009E
:10E560001000FA00000F78001207980023079800A7
:10E5700031079800440798005507980066079800EF
:10E5800077079800BE0090004E00900006F8020049
:10E59000000000006E0090000000E0000400320067
:10E5A000BE0090006E00900006F80200000000001F
:10E5B0008F87E8002EF09700E0FF9F002EB89700AD
:10E5C000BEB89700809FBE008F87E8008EF8970046
:10E5D000E1FF9F00FE0390006E039000DE029000BA
:10E5E0004E0290001E019000AE01900041C0B300A9
:10E5F0001E0078003FFF0700E88757000080FA0000
:10E60000000006001200FA00500798006107980009
:10E6100072079800030F98007E019000DE009000C2
:10E620005E00900098F70200000000000040EB0040
:10E63000304798000040EB00204798006E009000A3
:10E64000100F78000E089000100078000000E9001C
:10E6500040079800480037004E0090008E08900058
:10E660000080E80001004000904078004147980099
:10E670004E4090000004E0003C0032004E0090004C
:10E68000DE0090000080E80001004000904078002B
:10E690006147980010C0B300504798002A00370027
:10E6A0004E4090000080FB00610060000004E0002C
:10E6B0001E0032002E4090000004E00009003A00E5
:10E6C0001E0FE9001E007800EE0090000080E800B8
:10E6D00001004000904078003147980010C0B3001E
:10E6E000204798003E409000AE40900001406000FE
:10E6F0000004E000050032006E409000DE40900013
:10E700000140700060479800050037005E409000AF
:10E7100080C0EA006E40900000C060006047980032
:10E720002E40900000404000204798005E4090003E
:10E7300000404000504798004E4090000080FB0091
:10E740000000D100404798004E4090000004E000D7
:10E75000D3FF3A004E009000DE0090000080E800F9
:10E7600001004000EE409000014878004E0090000B
:10E770000000E900400798004E0090000000E00013
:10E78000B5FF3D000080FA00000006000200FA001C
:10E79000000F78009E00780040002000B000980034
:10E7A0001E007800300090000080FA000000060093
:10E7B0000200FA00000F78009E00780010C0B3003D
:10E7C000804878000000EB000080FA00000006009E
:10E7D0000200FA00000F78001E007800A0089000E8
:10E7E000820B20001E00410006F80200000000001D
:10E7F0000000EB000080FA00000006000800FA00AC
:10E80000889FBE008A1F7800300798006400470088
:10E8100058FB0200000000004E4090000080FB000A
:10E8200001002000ECFC0700100798009E009000FB
:10E8300020032000808F500003003400600020007F
:10E84000000F7800240037004E4090000080FB004D
:10E8500001002000E0FC0700800078003E009000EE
:10E860007600400006F80200000000003E00900024
:10E8700060019000F00190003E00900090489000F0
:10E880003E009000760240004E4090000084FB0065
:10E89000090020003E009000680540008F87E800D6
:10E8A0000040EB00E0FF9F00829FBE008F87E800E2
:10E8B000E1FF9F008003EB000003EB008002EB0010
:10E8C0000801BE00B1C0B3000A00780089FE07004D
:10E8D000E8875700000F78001E00E00003003200B8
:10E8E0003E0090009E007800310098001E007800E5
:10E8F0004F0578004F04BE000080FA0000000600BB
:10E900000A00FA00881F7800400798004E00900027
:10E91000760040002100200006F802000000000000
:10E920004E0090007600400062F6020000000000F9
:10E9300020079800310798002E009000BE0090003C
:10E94000A5FC0700100798009E00900020032000FF
:10E95000808F50000300340060002000000F78001A
:10E96000210037002E009000BE0090009AFC0700A6
:10E97000800078004E0090007600400006F802000B
:10E98000000000004E00900060019000F001900037
:10E990004E009000904890004E009000760240009B
:10E9A0004E009000680440008F87E8000040EB00B4
:10E9B000E0FF9F00829FBE008F87E800E1FF9F007D
:10E9C0008003EB000003EB008002EB002E019000BF
:10E9D000BE019000B1C0B3000800780045FE0700FA
:10E9E000E8875700000F78001E00E00003003200A7
:10E9F0004E0090009E007800310098001E007800C4
:10EA00004F0478000080FA00000006000400FA00BD
:10EA1000889FBE008A9FBE00100798001E009000CD
:10EA2000A00890001E0090007600400006F802004A
:10EA3000000000001E009000B04890001E009000F2
:10EA400060019000F00190001E009000204A9000AC
:10EA50001E009000870B2000808343001E00900062
:10EA6000C5042000808242001E0090002A08200079
:10EA7000000545001E009000F60540001E009000B5
:10EA8000000C9000900C90001E0090006800400068
:10EA90008F87E800E1FF9F00829FBE008F87E8001C
:10EAA000E4FF9F00050378008A0278000B027800DB
:10EAB0000801BE0041C0B3000EFE0700E887570002
:10EAC000000F78001E00E000030032001E009000DE
:10EAD0009E007800310098001E0078004F05BE00AF
:10EAE0004F04BE000080FA00000006000200FA0099
:10EAF000000F78009E0078007680400041002000E2
:10EB000006F80200000000009E00780076804000B9
:10EB100062F60200000000001E017800600198000B
:10EB2000710198000000EB000080FA000000060070
:10EB30000200FA00000F78009E0078006B80400011
:10EB400058FB0200000000000000EB000080FA000B
:10EB5000000006000400FA00100798000000EB0017
:10EB6000000F78001E009000760040004100200059
:10EB700006F80200000000001E0090007600400031
:10EB800062F60200000000001E01900000099800DB
:10EB9000110998001E009000900890000008900055
:10EBA0000DFC0700800078001E00900021089800EE
:10EBB0001E009000A008900020032000808F5000CD
:10EBC0000500340060002000000F78001E00900057
:10EBD0009E007800310098001E0078000080FA0046
:10EBE000000006000400FA00889FBE008A9FBE0055
:10EBF0008C1F7800100798001E009000B04890000D
:10EC00001E00900060019000F00190001E00900036
:10EC1000204A90001E009000870B20008083430054
:10EC20001E009000C5042000808242001E0090005B
:10EC30002A082000000545001E009000F60540004F
:10EC40001E009000200E90001E009000000C90000E
:10EC5000900C90001E009000680040008F87E80034
:10EC6000E1FF9F00829FBE008F87E800E4FF9F00C6
:10EC7000050378008A0278000B0278008C00780087
:10EC80000801BE0036FE0700E8875700000F780035
:10EC90001E00E000030032001E0090009E0078007D
:10ECA000310098001E0078004F0678004F05BE0026
:10ECB0004F04BE000080FA00000006000200FA00C7
:10ECC000000F78001E007800A0089000E20E2000DF
:10ECD0001E00410006F80200000000001E0078003F
:10ECE000A0089000421220001E00410006F8020019
:10ECF000000000000000EB000080FA0000000600A9
:10ED00000A00FA00889FBE008A9FBE004007980054
:10ED10004E009000A00890004E0090007600400049
:10ED200006F80200000000004E009000B04890007D
:10ED30004E00900060019000F00190004E009000A5
:10ED4000204A90004E009000870B200080834300F3
:10ED50004E009000C5042000808242004E009000CA
:10ED60002A082000000545004E009000F6054000EE
:10ED70004E009000000C9000900C90004E0090000F
:10ED8000680040008F87E800E1FF9F00829FBE007F
:10ED90008F87E800E4FF9F00050378008A0278006F
:10EDA0000B0278000801BE0041C0B30051FD07000E
:10EDB000E8875700200798002E0090000000E00030
:10EDC00066003A000000EB00100798000040EB00DE
:10EDD000004F7800150037001E80FB00CE00900029
:10EDE0006012B00001004000904078001147980088
:10EDF0000A0037001E4090000080FB00E100600028
:10EE00001E00900001004000100798001E40900076
:10EE10000080FB000000D100104798001E409000C9
:10EE20000004E000F3FF3A001E4FE8001E80FB00E4
:10EE3000CE009000A1109100810F5000E6FF350038
:10EE40006600470058FB0200000000000040EB0095
:10EE5000004F78003B0037001E009000CF80DE009E
:10EE60005DFB0700800078004E009000A015B00008
:10EE700006F80200000000004E0090004212200040
:10EE8000000141004E009000E40E2000000242000C
:10EE90004E009000A1152000808040004E009000A0
:10EEA000760040008201780004017800D5FD07005B
:10EEB0004E009000B04890004E009000600190001D
:10EEC000F00190004E009000204A90004E0090000B
:10EED000870B2000808343004E009000C504200073
:10EEE000808242004E0090002A0820000005450064
:10EEF0004E009000F60540004E009000000C90007F
:10EF0000900C90004E009000680040008F87E80051
:10EF1000E1FF9F00829FBE008F87E800E4FF9F0013
:10EF2000050378008A0278000B0278000801BE0011
:10EF300041C0B300EFFC0700E887570020079800A6
:10EF40001E4FE8002E0090000000E00003003A0091
:10EF50006E4090009E4F1000BFFF39002E009000C1
:10EF60000000E000030032004E009000AE00900070
:10EF7000310098002E0090004F05BE004F04BE00E7
:10EF80000080FA00000006000800FA00889FBE001A
:10EF9000200798002E00900010409000EE4F500087
:10EFA00004003A002E00900020489000604798002E
:10EFB0000200370040C0B30060479800EE40900068
:10EFC000214798002E009000760240002E0090000D
:10EFD000200C90002E0090000009900090099000F5
:10EFE0002E009000E80440008F87E8000040EB000E
:10EFF000E0FF9F006000B800809FBE008F87E800A0
:10F000002E409000E0FF9F008003EB000003EB0028
:10F010008002EB00880078000900780050FD0700AE
:10F02000E8875700000F78001E00E0000300320060
:10F030002E0090009E007800310098001E0078009D
:10F040004F04BE000080FA00000006000800FA002D
:10F05000889FBE008A1F7800200798002E0090002D
:10F0600010409000F14F500004003A002E00900034
:10F0700020489000604798000200370040C0B3006D
:10F0800060479800EE409000214798002E009000C5
:10F09000C4042000000242002E0090002508200039
:10F0A000808242002E009000760440002E009000E6
:10F0B000A00C90002E009000000990009009900094
:10F0C0002E009000680540008F87E8000040EB00AC
:10F0D000E0FF9F006000B800809FBE008F87E800BF
:10F0E0002E409000E0FF9F008003EB0004037800B7
:10F0F00008027800890078000A00780018FD0700EF
:10F10000E8875700000F78001E00E000030032007F
:10F110002E0090009E007800310098001E007800BC
:10F120004F0578004F04BE000080FA000000060082
:10F130000600FA00200798000E80E80058FB020045
:10F1400000000000AE4090002E00900068004000DB
:10F15000CCFA0700000F78001E00E0000300320028
:10F160002E0090009E007800310098001E0078006C
:10F170000080FA00000006000600FA002007980050
:10F180000000EB00000F78000E80E80058FB020042
:10F19000000000002E4090000004E0000600320055
:10F1A0002E409000E14F500003003200500020003C
:10F1B000000F7800190037002E00900010409000DA
:10F1C000F34F50000B003A002E4090000004E00086
:10F1D00004003A00AE00900010C0B30090489800C0
:10F1E0000E003700AE009000D0C0B30090489800E9
:10F1F0000A0037002E4090000004E00004003A00AE
:10F20000AE00900010C0B300A04898000300370083
:10F21000AE00900060C0B300A04898001E00E0005F
:10F22000030032002E0090009E007800310098000C
:10F230001E0078000080FA00000006000400FA00BA
:10F24000100798000E00780058FB02000000000034
:10F250001E4078000004E000FAFF3A009E00900093
:10F260000000EB00B00098001E00900030009000FD
:10F270000080FA00000006000800FA00300798003D
:10F280003E009000760040001100200006F80200C9
:10F29000000000003E009000805890005147980008
:10F2A0003E009000760040001100200006F80200A9
:10F2B000000000003E0090008058900041479800F8
:10F2C0003E009000760040004100200006F8020059
:10F2D000000000003E0090007600400062F6020050
:10F2E00000000000008FBE003E00900080489000AB
:10F2F0005E40900080CF5000040032003E0090003D
:10F3000068004000DE4090005EFA07001E00BE006C
:10F31000D2FB0200000000003E00900080489000F8
:10F320004E40900080CF5000040032003E0090001C
:10F3300068004000CE40900052FA07000000EB0049
:10F340000080FA00000006000200FA00000F7800BA
:10F350001E007800F3F90700800078001E00780096
:10F36000310098001E007800300090000000E0009E
:10F3700007003A009E007800688040008040EB0063
:10F3800040FA0700800078001E00780031009800E5
:10F390001E007800300090000080FA000000060097
:10F3A0000200FA00000F78001E0078003000900084
:10F3B0000000E0001F003A001E00780010407800B6
:10F3C0000004E0001B003A001E00E80058FB0200A9
:10F3D000000000001E007800A000900010009000C7
:10F3E00061004000E08048001E0178001001980094
:10F3F000210198001E00780010409000F74F500047
:10F400000A003E001E007800104090000080FB00C3
:10F41000800040008054230000804000900078006D
:10F420001E00780001000100020037001E00780075
:10F43000D6FC07001E007800300090000080FA0023
:10F44000000006000200FA00000F78001E0078009D
:10F45000DDF907000080FA00000006009001FA00C4
:10F460000E007800B8FF0700020037000E00780099
:10F47000CBFF07003E0090000000E00003003A00D0
:10F480001E4078000004E000F8FF32000E00780013
:10F49000ECFF07003E0090000080FA00000006002C
:10F4A0000000FA0001DF2200114078000060A00097
:10F4B0008048780080622300104078006840600037
:10F4C0000004E00002003200DA82A90001003700E7
:10F4D000DA82A80080622300104078006840600053
:10F4E0000004E00003003200F0C2B300FED30200CB
:10F4F00000000000A100200000BD2000BAF80200BA
:10F50000000000000080FA00000006000000FA0081
:10F5100001DF2200114078000060A10080487800DF
:10F520008062230010407800684060000004E00022
:10F5300002003200DA82A90001003700DA82A80056
:10F540008062230010407800684060000004E00002
:10F5500003003200F0C2B300FED30200000000003E
:10F56000A100200000BD2000BAF802000000000049
:10F570000080FA00000006000000FA00806223000C
:10F5800010407800684060000004E0000200320093
:10F59000DA82A80001003700DA82A9008062230025
:10F5A00010407800684060000004E0000300320072
:10F5B000F0C2B300FED3020000000000B100200042
:10F5C000A0BD2000BAF80200000000000080FA0090
:10F5D000000006000000FA0000C0EB005202070025
:10F5E0000080FB000080FA00000006000600FA0020
:10F5F000100798001E0090004B020700004F780093
:10F6000000DF2200104078000044B2000004E00057
:10F61000030032001E80FB00200798000200370024
:10F620000000EB00200798002E0090000080FA00F8
:10F63000000006000000FA0001022000C0DA2000ED
:10F6400030F8020000000000E0DD220010407800E9
:10F650000040E800A0D202000000000000C2B30099
:10F66000FED302000000000080622300904078007A
:10F6700061C06000A0D202000000000000C2B30020
:10F68000FED3020000000000806223001080FB0017
:10F690000000D10061406000A0D202000000000024
:10F6A00000C2B300FED3020000000000806223000D
:10F6B0001080FB004200DE0061406000A0D202002A
:10F6C0000000000000C2B300FED3020000000000F2
:10F6D000806223001080FB004300DE006140600078
:10F6E000A0D202000000000000C2B300FED302005E
:10F6F0000000000000DF22001080FB004400DE005C
:10F7000061406000A0D202000000000000C2B3000F
:10F71000FED30200000000003100200090BF200056
:10F7200030F80200000000000080FA00000006002F
:10F730000C00FA00B040020000000000263D02006C
:10F740000000000050079800B040020000000000D8
:10F75000263D02000000000040079800B040020073
:10F7600000000000263D0200000000003007980065
:10F77000B040020000000000263D02000000000032
:10F7800020079800B040020000000000263D020063
:10F7900000000000000F7800B040020000000000F0
:10F7A000263D020000000000100798005E00900057
:10F7B0000000E000090034005E009000E40F5000FB
:10F7C00006003C005E0090000040E90080407800A8
:10F7D000E0DD220001487800020037000000EB0065
:10F7E000500798004E0090000000E0000C0034002C
:10F7F0004E009000E20F500009003C004E009000C7
:10F800000040E900E14060008062230061C16000C7
:10F81000E1CFB30010C8600010487100020037004B
:10F820000000EB00500798003E0090000000E00050
:10F830000D0034003E009000E20F50000A003C0032
:10F840003E0090000040E9006140600081622300BA
:10F850006140600000414000D0CFB300914860009B
:10F8600091487100020037000000EB00500798003B
:10F870002E0090000000E0000D0034002E009000EB
:10F88000E20F50000A003C002E0090000040E9000A
:10F89000E140600080622300E1C060004209DD00B9
:10F8A000B1CFB30010C860001048710002003700EB
:10F8B0000000EB00500798001E00E0000D0034002F
:10F8C000200020009E0F10000A003C001E0078005F
:10F8D0000040E900E140600080622300E1C0600078
:10F8E0004309DD0071CFB30010C8600010487100FB
:10F8F000020037000000EB00500798001E00900047
:10F900000000E0000F0034001E009000E20F5000E5
:10F910000C003C001E0090000040EA00E140600046
:10F9200003DF220013407800E1C060004409DD00DD
:10F93000F1CEB300014060000240700080497800C1
:10F94000020037000000EB00500798005E009000B6
:10F950000000E0006C003A000000EB00F097890026
:10F9600071032000C0CC2000BAF8020000000000A3
:10F970008001EB0042002000110020001000200058
:10F9800018430200000000000040E90080407800B9
:10F99000E0DD2200014878005103200030D0200033
:10F9A000BAF80200000000008001EB0022002000F5
:10F9B0001100200010002000184302000000000089
:10F9C0000040E900E14060008062230061C1600006
:10F9D000E1CFB30010C8600010487100310420006E
:10F9E00080D32000BAF80200000000008001EB0084
:10F9F00022002000110020002000200018430200F7
:10FA0000000000000040E9006140600081622300C6
:10FA10006140600000414000D0CFB30091486000D9
:10FA20009148710011032000B0D72000BAF80200FD
:10FA3000000000008001EB002200200011002000E7
:10FA40001000200018430200000000000040E90000
:10FA5000E140600080622300E1C060004209DD00F7
:10FA6000B1CFB30010C8600010487100D101200070
:10FA7000B0362100BAF80200000000008001EB005F
:10FA80002200200011002000200020001843020066
:10FA9000000000000040E900E140600080622300B7
:10FAA000E1C060004309DD0071CFB30010C8600001
:10FAB00010487100F104200050A52000BAF802009F
:10FAC000000000008001EB00220020001100200057
:10FAD0001000200018430200000000000040EA006F
:10FAE000E140600003DF220013407800E1C06000C5
:10FAF0004409DD00F1CEB300014060000240700017
:10FB00008049780001003700CAFE070001DF2200AB
:10FB1000114078000060A10080487800E0DD2200FC
:10FB2000104078008080FB00A05E230061407800D8
:10FB300094000700806223001080FB004300DE0079
:10FB400061406000614060004401DD00A12D2000A3
:10FB500091407800F0CEB30000C060000240700019
:10FB6000DAE2B7000080FA00000006000000FA00A8
:10FB7000D60007000080FA00000006000600FA0028
:10FB8000000F78001E0078006101B800120798008D
:10FB900023079800F0002000010020001E019000C3
:10FBA000AE019000800F5100818F590068003E0027
:10FBB0001E009000AE009000006001000F003700B2
:10FBC000130037001E003700650037006000370063
:10FBD0005F0037005E0037005D0037005C003700D3
:10FBE0005B00370022003700250037002700370070
:10FBF0002A0037002C0037002F0037004103200077
:10FC0000C0DC2000BAF802000000000054003700F9
:10FC100071002000D05A2000BAF802000000000055
:10FC2000F100200000332100BAF8020000000000BB
:10FC300011C0B3000040EB00C900070048003700C6
:10FC400071002000D05A2000BAF802000000000025
:10FC5000F100200000332100BAF80200000000008B
:10FC600011C0B30010C0B300BD0007003C00370056
:10FC700081622300E0CFB30091486000100037009C
:10FC8000806223001004A0000D0037008162230071
:10FC9000D0CFB30091486000090037008062230094
:10FCA0001014A0000600370081622300B0CFB3001B
:10FCB0009148600002003700806223001024A000F9
:10FCC000806223009040780061C060006140600065
:10FCD0004601DD002124200091407800F0CBB300E4
:10FCE00000C060000240700042E2B7008062230062
:10FCF0001080FB000000D1006140600061416000A5
:10FD00003124200091407800E0CFB30000C06000B3
:10FD10000240700043E2B700806223001080FB00C5
:10FD20004200DE0061406000614060000041400030
:10FD30003124200091407800D0CFB30000C0600093
:10FD40000240700043E2B7003AFE070004003700AB
:10FD500041022000E01D2000BAF80200000000006F
:10FD60000080FA00000006000000FA0001012000F7
:10FD700010422100BAF80200000000000080FA00E2
:10FD8000000006000200FA00004F780041E2A900DE
:10FD900000DF220010407800704060000004E000A6
:10FDA00004003200DE62A800DE42A800DE82A80065
:10FDB00003003700DE62A900DE42A900DE82A9004E
:10FDC000816A20009140780000CCB30000C0600040
:10FDD0006041B300A8E6B700816D20009140780033
:10FDE00000CCB30000C060007040B300D8E6B7009C
:10FDF000716D20009140780000CCB30000C060001D
:10FE00000034A000D7E6B700DA82A800D882A900A3
:10FE1000D842A900D862A800D822A9001E80FB0001
:10FE20001012880042A2A80080622300904078004F
:10FE300061C06000614060004601DD0021242000B7
:10FE400091407800F0CBB30000C060000240700029
:10FE500042E2B700806223001080FB000000D10066
:10FE600061406000614160003124200091407800D1
:10FE7000E0CFB30000C060000240700043E2B70072
:10FE8000806223001080FB004200DE0061406000C1
:10FE90006140600000414000312420009140780022
:10FEA000D0CFB30000C060000240700043E2B70052
:10FEB0000000EB00201288000000EB000012880018
:10FEC00041E2A8000080FA00000006000000FA00ED
:10FED00041E2A900816A20009140780000CCB30083
:10FEE00000C06000F041B300A8E6B700816D2000BB
:10FEF0009140780000CCB30000C06000D8E6B700A5
:10FF0000716D20009140780000CCB30000C060000B
:10FF1000D7E6B700DE62A900DE42A900DE82A900B2
:10FF20000080FA00000006000200FA00004F78008E
:10FF30001E80FB004012880085C0BF006440600046
:10FF40000004E000FCFF320040128000004F780007
:10FF50008540A9001E80FB000080FA00000006001A
:10FF60000400FA00204798003147980010C0B30001
:10FF7000004F78007AD4020000000000D3FF070091
:10FF8000810007002E4090000004E00002003A00CB
:10FF900042E2A80062E2A8002E409000E14F50002B
:10FFA00002003E0041E2A80061E2A8001E04E00059
:10FFB00009003A00DAC2BF00704060000004E000AF
:10FFC00005003200D0C5B30016D4020000000000C6
:10FFD00010C0B300004F780040C2BF000042B20022
:10FFE0000004E0002F003A0060C2BF000042B200EF
:10FFF0000004E0002B003A004012800010479800F7
:020000040001F9
:1000000010C0B3009E4F100005003A00B0C5B30009
:1000100016D40200000000000040EB00004F780002
:100020003E4090000004E000050032001E409000B9
:100030000080FB0028D3020000000000060037000B
:10004000C0C5B30016D40200000000001E4090009E
:1000500016D40200000000004013800010479800F2
:100060003E4090000004E0000B00320080C2B3006C
:1000700016D40200000000001E4090000080FB002B
:1000800028D302000000000090C2B30016D4020082
:1000900000000000030037001E40900016D402004C
:1000A0000000000040C2BF000044B2000004E000B5
:1000B00009003A0060C2BF000044B2000004E00042
:1000C00005003A0040AE81000140200001006000C0
:1000D0000000E0001400320040AE8100014020002A
:1000E000010060000000E00002003A0068D4020055
:1000F000000000000000EB00001288000000EB0090
:10010000001388003E4090000004E000040032002C
:1001100060982A0034D002000000000093FF3700EE
:10012000CB02A9000F00370080D4020000000000BD
:1001300034D4020000000000E14F50009BFF3A0061
:100140005CD4020000000000104798003E40900080
:100150000004E0000300320070992A0034D002004D
:100160000000000083000700E0DD2200104078005E
:100170008080FB00A05E23006140780001FF070043
:100180000080FA00000006000000FA00D882A800F3
:10019000D842A800D862A800D822A800A16A2000EE
:1001A0009140780000CCB30000C060009041B300E3
:1001B000AAE6B700E16A20009140780000CCB300C5
:1001C00000C060009041B300AEE6B700816A200035
:1001D0009140780000CCB30000C060008041B300C3
:1001E000A8E6B700916A20009140780000CCB300E7
:1001F00000C060007041B300A9E6B700C16A2000EA
:100200009140780000CCB30000C060006041B300B2
:10021000ACE6B700D16A20009140780000CCB30072
:1002200000C060007041B300ADE6B700E0DD220021
:10023000104078008080FB00A05E230061407800C1
:100240000080FB001012880080622300904078003C
:1002500061C06000614060004601DD002124200093
:1002600091407800F0CBB30000C060000240700005
:1002700042E2B700806223001080FB000000D10042
:1002800061406000614160003124200091407800AD
:10029000E0CFB30000C060000240700043E2B7004E
:1002A0000000EB00201288000000EB000012880024
:1002B000E0DD2200104078008080FB00A05E23007B
:1002C000614078000080FB001013880080622300EA
:1002D0009040780061C06000614060004601DD0030
:1002E0002126200091407800F0CBB30000C06000D0
:1002F0000240700062E2B700806223001080FB00C1
:100300000000D100614060006141600031262000A2
:1003100091407800E0CFB30000C060000240700060
:1003200063E2B7000000EB00201388000000EB0040
:10033000001388000000EB00401288000000EB0072
:10034000401388004322A9006322A9004362A80049
:1003500042A2A9006362A80062A2A90040C2A9004B
:1003600060C2A9004402A8006402A8000080FA004C
:10037000000006000000FA0041E2A9004362A90063
:1003800061E2A9006362A900A16A2000914078009F
:1003900000CCB30000C06000F041B300AAE6B70093
:1003A000E16A20009140780000CCB30000C06000FA
:1003B000F041B300AEE6B700816A200091407800BA
:1003C00000CCB30000C06000F041B300A8E6B70065
:1003D000916A20009140780000CCB30000C060001A
:1003E000F041B300A9E6B700C16A2000914078004F
:1003F00000CCB30000C06000F041B300ACE6B70031
:10040000D16A20009140780000CCB30000C06000A9
:10041000F041B300ADE6B7000080FA00000006002E
:100420000000FA0080992A0008D0020000000000B5
:100430000080FA00000006001400FA00881F78000F
:10044000E1DD220010C0B300804878008162230003
:10045000E0CFB30091486000806223001014A00038
:1004600081622300B0CFB3009148600001DF220019
:10047000114078000040A00080487800E0DD2200B4
:10048000104078008080FB00E05E2300614078002F
:100490003CFE0700E2FF0700000037005CD40200CA
:1004A000000000008040780060622300014878006E
:1004B00060622300104078000080FB004400DE00F2
:1004C0008040780050622300014878005062230089
:1004D000104078000080FB00100F98001E0890006C
:1004E000E40F5000A80132009E089000E48F5000F5
:1004F00007003C001E0890000000E0000B003200E6
:100500009E089000E18F50007C013200F701370017
:100510001E089000E60F5000A30132009E089000D4
:10052000E88F5000B4013200F00137006062230010
:10053000104078000080FB00000F98000E0890002B
:10054000E50F500014003C008E089000E48F50002E
:100550003C003D000E089000E10F50001A003200F0
:100560008E089000E18F500004003C000E089000BF
:100570000000E000120032005C0137008E0890009D
:10058000E28F5000120032000E089000E30F50007E
:1005900017003200550137008E089000ED8F500093
:1005A0001A0032000E089000EE0F50001E003200BC
:1005B0008E089000E68F5000980032004B01370003
:1005C00042FE0700CD01370095FF0700B3FF37005B
:1005D000E0168000F1FE2F0001006000E0168800A8
:1005E00010C0B300FED3020000000000ABFF3700D4
:1005F000E01680000040A000E016880010C0B300A4
:10060000FED3020000000000A4FF370010C0B300BA
:10061000FED30200000000008040EB0010C0B300D9
:100620004FFE07009DFF370010C0B300FED302004D
:10063000000000008040EB000040EB0048FE070097
:1006400096FF37005CD40200000000000080FB0031
:10065000500798005E0090004800DD0050079800A9
:100660005CD40200000000008080FB005E0090006F
:1006700001007000500798005CD4020000000000E8
:100680000080FB00400798004E0090004800DD000D
:10069000400798005CD40200000000008080FB004E
:1006A0004E0090000100700040079800DE009000AE
:1006B00000002100808F500004003E00CE0090001A
:1006C00000002100808F5000040036000040EB0045
:1006D000FED302000000000070FF37000000EB00B6
:1006E0006007980009003700E1AD81006E009000BE
:1006F000008440005CD4020000000000004C780040
:100700006E0090000000E80060079800EE00900086
:100710005E009000808F5000F3FF3900606223007C
:1007200010407800E44F500001003A00DA82A9003E
:100730000000EB006007980008003700E1AD810081
:100740006E0090000080400010407800F6FD070029
:100750006E0090000000E80060079800EE00900036
:100760005E009000808F5000F4FF390010002000E0
:10077000E4F50200000000000000EB0060079800B4
:1007800009003700E1AD81006E0090000084400058
:1007900000C0EB00E4FD0700004C78006E00900004
:1007A0000000E80060079800EE0090004E00900006
:1007B000808F5000F3FF3900606223001040780002
:1007C000E44F500001003A00DA82A80010C0B300E4
:1007D000FED30200000000000000EB00600798005C
:1007E00009003700E1AD81006E00900000804000FC
:1007F00010407800FED30200000000006E00900060
:100800000000E80060079800EE0090004E009000A5
:10081000808F5000F3FF390020FF370010C0B30075
:10082000FED302000000000022C2BF006140600051
:100830000004E000FCFF32003011800080407800AE
:100840006062230001487800606223001040780055
:100850000080FB00700798007E009000E10F5000C0
:100860000B003200FE009000E28F500012003200B8
:100870007E0090000000E000010032009700370089
:1008800010C0B300FED302000000000003FF3700D9
:1008900010C0B300FED30200000000000040EB00D7
:1008A000FED302000000000010C0B300FED302001F
:1008B00000000000F9FE37006000B8002007980033
:1008C000310798000000EB0060079800190037001E
:1008D00022C2BF00614060000004E000FCFF320063
:1008E0003011800080407800606223000148780069
:1008F0002E009000BE0090004809DD00C801DE0017
:10090000830171004801DD0060622300104078001F
:100910000080FB0001002000000071008180710058
:1009200020079800310798006E0090000000E80052
:10093000600798006E009000E30F5000E4FF36005F
:100940006000B800008FBE000000EB006007980058
:100950001600370022C2BF00614060000004E000C2
:10096000FCFF32003011800080407800606223007C
:10097000014878001E00BE004809DD00C801DE0005
:10098000830171004801DD0060622300104078009F
:100990000080FB0001002000001F71000197710022
:1009A0006E0090000000E800600798006E00900064
:1009B000E30F5000E7FF36002E019000BE019000CB
:1009C000F0FF2F0001002000800F5100818F59009F
:1009D0000E003E00F0FF2F0001002000BE0F1000AF
:1009E000AE8F180009003E002E009000BE0090005F
:1009F0003E014000AE814800F0FF2F0001002000C2
:100A0000800F5100818F5900040036000040EB0038
:100A1000FED3020000000000A0FE370010C0B300AB
:100A2000FED3020000000000AE00900061079800B5
:100A30002500370000C2B3003BFD07006E009000A8
:100A40004800DE0038FD07006E00900036FD07000C
:100A50000040EB0034FD0700FED302000000000060
:100A60000080EB008080EB001E0F40005E97480086
:100A70001E00BE00E00F5000E08F580087FE3200DD
:100A800080C2B30028FD07006E0090004800DE0021
:100A900025FD07006E00900023FD07000040EB00DD
:100AA00021FD0700FED30200000000000080EB00E3
:100AB0008080EB001E0F40005E9748006E009000A3
:100AC0000000E800600798001E00BE00E00F500024
:100AD000E08F5800D7FF3A0070FE37000040EB006F
:100AE000FED30200000000006CFE37000040EB0067
:100AF000FED302000000000068FE370060622300A1
:100B000090407800F0C0B30080C0600060622300B5
:100B10000148780060622300104078008040E800BF
:100B2000606223000148780010C0B300FED30200C9
:100B300000000000416223000040EB008048780084
:100B40000A0037005CD4020000000000F6FC070039
:100B5000FED3020000000000406223001040780035
:100B60008040E80040622300014878004062230092
:100B700090407800606223001040780080CF5000E1
:100B8000F0FF390045FE3700606223001040780016
:100B90000A0002000100000010C0B300FED30200F2
:100BA000000000003DFE37006062230090407800A6
:100BB00070C0B30080C0600060622300014878000C
:100BC0006062230090407800E0DD22000148780058
:100BD000E0DD2200104078008080FB00E05E230012
:100BE0006140780067FC070010C0B300FED302002C
:100BF0000000000029FE370081622300E0CFB3002F
:100C00009148600081622300D0CFB300914860001A
:100C100081622300B0CFB3009148600001DF220061
:100C2000114078000040A1008048780060622300F5
:100C3000104078000080FB004200DE006100600090
:100C40000004E00002003200806223001004A000D3
:100C500060622300104078000080FB000000D1009B
:100C6000610060000004E0000200320080622300A6
:100C70001014A00060622300104078000080FB0088
:100C8000610060000004E000020032008062230086
:100C90001024A00060622300104078000080FB0058
:100CA0004300DE000000A200610060000004E000DC
:100CB0000400320001DF2200114078000040A00053
:100CC00080487800E0DD2200104078008080FB0042
:100CD000E05E2300614078002AFC070010C0B300EA
:100CE000FED3020000000000ECFD37000040EB00E6
:100CF000FED3020000000000E8FD37004F0478003A
:100D00000080FA00000006000400FA00BAFE0200AB
:100D1000000000000004E0002200320032C2BF00E8
:100D2000684060000004E000040032003100200050
:100D300000E0200030F802000000000032C2BF00D6
:100D4000644060000004E000040032003100200034
:100D500030E0200030F8020000000000AAFE02008F
:100D600000000000000F780032C2BF006240600047
:100D70000004E00008003200F100200060E02000E4
:100D800030F802000000000090118000D1FF2F0019
:100D900001006000901188001E0078001007980084
:100DA00006003700F100200050E1200030F802007A
:100DB000000000000000EB00100798001E009000EB
:100DC0000080FA00000006000200FA00000F780020
:100DD0001E00780096FE0200000000000000EB00FC
:100DE0000080FA00000006000000FA000102200066
:100DF000B0EC200030F8020000000000E0DD22002E
:100E000010407800A0D202000000000000C2B30031
:100E1000FED3020000000000E0DD22001040780058
:100E2000E94F500007003A00C011800042D2020092
:100E30000000000000C2B300FED30200000000006A
:100E40000C003700E0DD2200104078000080FB003D
:100E50008000400080572300008040001000780090
:100E600042D202000000000000C2B300FED3020024
:100E700000000000A06123009040780063C0600083
:100E8000A0D202000000000000C2B300FED30200A6
:100E900000000000A06123001080FB004200DE0083
:100EA00061406000A0D202000000000000C2B30058
:100EB000FED3020000000000A06123001080FB00B0
:100EC0004300DE0061406000A0D20200000000008C
:100ED00000C2B300FED302000000000000DF2200C9
:100EE0001080FB004400DE0061406000A0D20200E0
:100EF0000000000000C2B300FED3020000000000AA
:100F00003100200090BF200030F8020000000000F7
:100F10000080FA00000006001000FA000000EB005C
:100F2000200798006000B800008FBE00B0400200AB
:100F300000000000263D020000000000700798003D
:100F40007E009000EA0F500005003A00B040020019
:100F500000000000263D020000000000200798006D
:100F6000B040020000000000263D0200000000002A
:100F700060079800B040020000000000263D02001B
:100F80000000000050079800B04002000000000080
:100F9000263D02000000000040079800B04002001B
:100FA00000000000263D020000000000300798000D
:100FB0007E0090000000E000090034007E009000F8
:100FC000EA0F500006003C007E0090000040E9005F
:100FD00080407800E0DD2200014878000200370000
:100FE0000000EB00700798006E0090000000E00029
:100FF0000C0034006E009000E40F500009003C002B
:101000006E0090000040E900E3406000A061230012
:1010100063C16000C1CFB30010C860001048710008
:10102000020037000000EB00700798005E0090009F
:101030000000E0000D0034005E009000E20F500060
:101040000A003C005E0090000040E900E1406000C2
:10105000A0612300E1C060004209DD00B1CFB30010
:1010600010C8600010487100020037000000EB005B
:10107000700798004E0090000000E0000D00340062
:101080004E009000E20F50000A003C004E0090001D
:101090000040E900E1406000A0612300E1C0600081
:1010A0004309DD0071CFB30010C860001048710023
:1010B000020037000000EB00700798003E0090002F
:1010C0000000E0000F0034003E009000E20F5000EE
:1010D0000C003C003E0090000040EA00E14060004F
:1010E00003DF220013407800E1C060004409DD0006
:1010F000F1CEB300014060000240700080497800EA
:10110000020037000000EB00700798007E0090009E
:101110000000E00085003A000000EB00F097890035
:10112000E10B2000C0952000BAF80200000000008A
:101130008001EB00B2002000110020001000200010
:1011400018430200000000000040E90080407800E1
:10115000E0DD220001487800E0DD22001040780048
:10116000EA4F500009003A00E1DD220080C0B300E0
:10117000804878001000200001002000008FBE0091
:10118000608A2A0034D0020000000000E0DD220066
:1011900010407800E94F50001A003A0091012000F9
:1011A000702F2100BAF80200000000008001EB005F
:1011B000F4232400F50020001200200000202C0061
:1011C00011002000A444020000000000008FBE00B7
:1011D0001E01BE0000902000D1032000C8240200A0
:1011E000000000000081EB008081EB00021F400046
:1011F000039748009E017800230798006000B8001C
:10120000008FBE004105200040E2200030F80200BF
:10121000000000008001EB004200200011002000CF
:101220001000200018430200000000000040E90008
:10123000E3406000A061230063C16000C1CFB30040
:1012400010C86000104871001102200080E72000E3
:1012500030F80200000000008001EB0022002000B6
:1012600011002000100020001843020000000000C0
:101270000040E900E1406000A0612300E1C060009F
:101280004209DD00B1CFB30010C860001048710002
:101290002103200090E9200030F802000000000047
:1012A0008001EB002200200011002000100020002F
:1012B00018430200000000000040E900E140600027
:1012C000A0612300E1C060004309DD0071CFB300DD
:1012D00010C8600010487100F104200050A52000E3
:1012E000BAF80200000000008001EB00220020009C
:1012F0001100200010002000184302000000000030
:101300000040EA00E140600003DF22001340780063
:10131000E1C060004409DD00F1CEB300014060008F
:10132000024070008049780001003700AEFE0700DF
:10133000E0DD220010407800E94F500019003A002B
:10134000A06123001080FB004200DE0061406000CD
:1013500080417800A06123009040780063C0600065
:1013600080427800A06123001080FB004300DE0073
:10137000614060000041780000DF22001080FB0027
:101380004400DE0061406000804078002E00900044
:101390000342780085417800E4FD0200000000006F
:1013A0001F003700A06123001080FB004200DE0018
:1013B0006140600000417800A06123009041780006
:1013C00063C0610080417800A06123001080FB00B1
:1013D0004300DE00614060008042780000DF2200B0
:1013E0001080FB004400DE00614060000043780094
:1013F000E0DD2200104078000080FB00800040000B
:1014000080572300008040001000780002427800DE
:101410000541780086407800E4FD020000000000ED
:10142000A06123001040780063406000E34F50004B
:1014300003003A00F1DD220090C0B300804878003C
:1014400068FE020000000000C11180004011800011
:10145000808F500004003100010220000031210083
:10146000BAF80200000000001E00BE00E00F5000AD
:10147000E08F58005900320074FE020000000000A6
:10148000008C2A0034D00200000000000000EB00B5
:10149000B701070068010700008FBE00008C2A001A
:1014A00034D00200000000001E00BE00E00F50001B
:1014B000E08F580019003A00A06123001080FB0063
:1014C0004200DE006140600080417800A06123009E
:1014D0009040780063C0600080427800A0612300E3
:1014E0001080FB004300DE00614060000041780096
:1014F00000DF22001080FB004400DE00614060003D
:101500008040780040AC810003427800854178003B
:10151000E4FD02000000000026003700E1DD2200AB
:1015200090C0B300804878001E01BE0000902000EB
:10153000D1032000C8240200000000000081EB005D
:101540008081EB00021F4000039748009E01780055
:1015500023079800A06123001080FB004200DE00FA
:101560006140600080417800A061230090407800D5
:1015700063C0600080427800A06123001080FB00FF
:101580004300DE00614060000041780000DF22007F
:101590001080FB004400DE00614060008040780065
:1015A0002E0090000342780085417800E4FD02009F
:1015B0000000000068FE020000000000C111800071
:1015C00040118000808F5000040031000102200093
:1015D00000312100BAF80200000000000080FA008B
:1015E000000006000000FA0074FE02000000000087
:1015F0000080FA00000006000400FA00000F7800E6
:101600001E007800100798001E009000E20F5000A6
:10161000480032001E009000E20F500007003E001C
:101620001E0090000000E0000B0032001E00900041
:10163000E10F50000D0032006E0037001E009000D8
:10164000E30F5000090032001E009000E40F50002C
:101650005900320067003700C1072000B0EE2000BB
:1016600030F802000000000066003700B1002000E2
:1016700070F62000BAF8020000000000E10020002F
:1016800040522100BAF802000000000060F9020098
:10169000000000000000E0005A00320090118000BD
:1016A000D1FF2F000100600090118800000037007A
:1016B000D3C2BF000044B2000004E0005100320079
:1016C00032C2BF00614060000004E000030032004D
:1016D000B0118000FED302000000000034D40200EC
:1016E00000000000E14F500008003A0033C2BF0084
:1016F000624060000004E00004003A005CD4020094
:10170000000000000080FB00A011880032C2BF0072
:10171000624060000004E000E5FF320090118000AC
:10172000D1FF2F000100600090118800CB02A900BA
:10173000DFFF3700E1002000F0F72000BAF80200D8
:1017400000000000F100200000332100BAF8020080
:101750000000000090118000D1FF2F000100600008
:1017600090118800D3C2BF000044B2000004E00022
:1017700024003200BAFE0200000000000004E00075
:1017800004003200AAFE020000000000FED30200A6
:101790000000000034D4020000000000E14F5000BF
:1017A000F0FF3A005CD40200000000000080FB0063
:1017B000000F78001300370074FE020000000000E4
:1017C0000000EB00EA00070068FE020000000000D5
:1017D000C111800040118000808F5000090031004D
:1017E0000102200000312100BAF8020000000000D0
:1017F0000400370041022000E01D2000BAF802007A
:10180000000000000080FA00000006000000FA005E
:1018100091118000D0FF2F0000806000901188009F
:10182000A06123001044A00001DF220011407800D5
:101830000020A00080487800C1012000D0F82000DE
:10184000BAF80200000000000080FA000000060064
:101850000000FA00A1612300F0CEB30091486000BF
:1018600001DF2200114078000020A10080487800AC
:101870004101200090FA2000BAF8020000000000A8
:101880000080FA00000006000200FA000000EB00F1
:10189000000F780034003700A0612300104078006A
:1018A000704060000004E0002B003200208C2A0011
:1018B00034D002000000000061002000E07420002D
:1018C00030F802000000000032C2BF006840600033
:1018D0000004E000040032003100200000E020009D
:1018E00030F802000000000032C2BF006440600017
:1018F0000004E000040032003100200030E020004D
:1019000030F8020000000000AAFE02000000000003
:1019100012F502000000000032C2BF006240600009
:101920000004E00008003200F100200060E0200028
:1019300030F802000000000090118000D1FF2F005D
:101940000100600090118800208C2A0034D0020031
:101950000000000002003700AAFE020000000000A4
:1019600010002000000F7800BAFE02000000000006
:101970000004E000C8FF3A001E0078000080FA0072
:10198000000006000000FA00B1002000A043210082
:10199000BAF80200000000000080FA000000060013
:1019A0000000FA000000EB00F00888000000EB00E7
:1019B0008008880080002000800888000000EB007C
:1019C000400888000000EB00300888000000EB00B1
:1019D000B00888000000EB00A0088800800020000C
:1019E000F00888000080FA00000006000000FA00FD
:1019F00011E1A9001FE1A900616820009140780071
:101A000000CCB30000C06000F041B30086E6B70030
:101A10000000EB00F00888000000EB008008880060
:101A20000000EB00300888000000EB004008880050
:101A30000080FA00000006001600FA007007980007
:101A4000010F98006000B8005007980061079800E7
:101A50006000B80030079800410798006000B800A7
:101A6000100798002107980010002000000F780050
:101A7000380037001E007800C200DD00408C2A00CC
:101A8000008040001001BE007E0090008E08900093
:101A9000800F5100818F59002D0036001E00E90093
:101AA000C200DD00408C2A00008040001001BE0012
:101AB00032079800430798001E007800C200DD003E
:101AC000408C2A00008040001001BE0052079800A0
:101AD000630798005E019000EE0190003E009000C8
:101AE000CE00900000005100818059008101D1009A
:101AF0000081D3003E009000CE0090000201400023
:101B0000838148007E0090008E089000800F510075
:101B1000818F5900050031005E009000EE009000BA
:101B2000100F9800210F9800040037003E0190002C
:101B3000CE019000120F9800230F98001E0890000D
:101B4000AE089000100798002107980004003700A5
:101B50001E0FE800E10020009E8F1000C5FF34003A
:101B60001E009000AE0090000080FA000000060009
:101B70001000FA00500798000000EB0040079800A2
:101B80006000B80020079800310798006000B80096
:101B9000008FBE00DA62A900D862A8005E00900043
:101BA0000000E00006003A0031012000205321002F
:101BB000BAF8020000000000010037000000000039
:101BC000DAC2BF00684060000004E0000400320098
:101BD00022C2BF00614060000004E000F7FF320055
:101BE00022C2BF00614060000004E0000B00320030
:101BF00030118000400798007CFF0700E1002000C2
:101C000050542100BAF80200000000006000B80043
:101C10006007980071079800760037000000EB001D
:101C200040079800420037005DFF0700DAC2BF009E
:101C3000684060000004E000FCFF32001FE1A800E3
:101C400011E1A800DAC2BF00684060000004E000B3
:101C5000FCFF3A0011E1A9001FE1A9006168200022
:101C60009140780000CCB30000C06000F041B300A8
:101C700086E6B7000000EB00F00888000000EB00EB
:101C8000800888004008800001002000200798009C
:101C9000310798002E009000BE009000C000DD00CB
:101CA00000002000200798003107980030088000CD
:101CB0006101B8002E009000BE00900000004100BD
:101CC0008180490020079800310798004E0090005D
:101CD0000000E000100032001E00BE00E00F5000C7
:101CE000E08F580004003A002E009000BE009000E3
:101CF000008FBE00080037002E009000BE0090004C
:101D0000BE0F1000AE8F1800030036002E009000AA
:101D1000BE009000008FBE006000B8002007980051
:101D2000310798004E0090000000E800400798003E
:101D30004E009000F80F5000BBFF36002BFF07004D
:101D40001E01BE0000402200410F2000C8240200F6
:101D500000000000008FBE005E0090000000E00068
:101D600021003A00009F240021002000BE0F100037
:101D7000AE8F180005003600810320003055210089
:101D8000BAF802000000000017003700F100200040
:101D9000B058210030F80200000000001E00BE0014
:101DA000A2D002000000000041002000905A210053
:101DB000BAF8020000000000F1002000A059210044
:101DC00030F80200000000001E00BE001AFF0700ED
:101DD000A2D002000000000041002000905A210023
:101DE000BAF80200000000001E00BE006007980064
:101DF000710798006E009000FE0090000080FA00CD
:101E0000000006000000FA0040902A0008D00200FE
:101E1000000000000080FA00000006000400FA0044
:101E2000A1612300C0CFB30091486000A1612300ED
:101E3000B0CFB30091486000A161230070CFB30020
:101E40009148600001DF2200114078000040A000AE
:101E50008048780060AC8100A0B08900A1612300B7
:101E6000F0CEB30091486000A06123001080FB0019
:101E70004200DE006140600080417800A0612300E4
:101E80009040780063C0600080427800A061230029
:101E90001080FB004300DE006140600000417800DC
:101EA00000DF22001080FB004400DE006140600083
:101EB00080407800A0B0810003427800854178001E
:101EC000E4FD02000000000068FE020000000000C7
:101ED000CCFF070000003700BAFE0200000000003F
:101EE0000004E0000C003200A061230010407800E4
:101EF000704060000004E00005003200AAFE02000D
:101F000000000000FED302000000000002003700C5
:101F1000AAFE02000000000032C2BF006240600062
:101F20000004E0000400320090118000D1FF2F0077
:101F3000010060009011880034D40200000000000D
:101F4000E14F5000E4FF3A005CD4020000000000C2
:101F50008040780080612300014878008061230080
:101F6000104078000080FB004400DE0080407800D4
:101F700070612300014878007061230010407800F0
:101F80000080FB00100798001E009000E40F500036
:101F9000C10032009E009000E48F500007003C001A
:101FA0001E0090000000E0000F0032009E00900034
:101FB000E18F500092003200600137001E00900057
:101FC000E60F5000BC0032009E009000E68F5000EB
:101FD0005A0135009E00900068805000E10F5000CB
:101FE00056013E00E9003700806123001040780070
:101FF0000080FB00000F78001E007800E20F500008
:10200000190032009E007800E28F500007003C006B
:102010001E0078000000E0000E0032009E007800F4
:10202000E18F50000E003200710037001E00780072
:10203000E70F5000210032009E007800EF8F500023
:102040004F0032001E007800E30F500014003200F1
:102050006700370074FE0200000000003B013700FB
:1020600068FF07009CFF370010C0B300FED30200DA
:102070000000000032C2BF00624060000004E000C7
:102080000400320090118000D1FF2F000100600099
:1020900090118800A06123001044A0008EFF37003B
:1020A000A1612300F0CEB3009148600010C0B300DE
:1020B000FED302000000000087FF370010C0B3000D
:1020C000FED302000000000074FE020000000000C9
:1020D0005CD40200000000000080FB004800DD002E
:1020E000A0B0890010C0B300FED3020000000000C1
:1020F0005CD40200000000008080FB00A0B08100E2
:1021000000807000A0B08900A06123001080FB0057
:102110004200DE006140600080417800A061230041
:102120009040780063C0600080427800A061230086
:102130001080FB004300DE00614060000041780039
:1021400000DF22001080FB004400DE0061406000E0
:1021500080407800A0B0810003427800854178007B
:10216000E4FD02000000000068FE02000000000024
:1021700010C0B300FED302000000000056FF37007D
:1021800010C0B300FED302000000000090118000D8
:10219000D1FF2F000100600090118800000037007F
:1021A00032C2BF00614060000004E0000300320062
:1021B000B0118000FED302000000000034D4020001
:1021C00000000000E14F5000F5FF3A0033C2BF00AD
:1021D000624060000004E000F1FF3A005CD40200BD
:1021E000000000000080FB00A0118800ECFF370019
:1021F0000040EB00FED302000000000036FF370075
:102200008061230090407800F0C0B30080C060007F
:10221000806123000148780080612300104078002D
:102220008040E800806123000148780010C0B300BE
:10223000FED3020000000000616123000040EB00BB
:10224000804878000D0037005CD4020000000000D8
:102250000080FB0096FE02000000000010C0B300EA
:10226000FED30200000000006061230010407800EF
:102270008040E8006061230001487800606123002D
:1022800090407800806123001040780080CF50009B
:10229000EDFF390010FF3700806123001040780007
:1022A0000A0002000100000010C0B300FED30200CB
:1022B0000000000008FF3700806123009040780094
:1022C000F0C0B30080C06000806123000148780046
:1022D0008061230010407800EA4F50000300360070
:1022E00081612300A0C0B300804878008061230092
:1022F000104078000080FB0080004000C0582300A0
:102300000080400010007800A0B0890074FE020038
:1023100000000000A06123001080FB004200DE00EE
:102320006140600080417800A06123009040780007
:1023300063C0600080427800A06123001080FB0031
:102340004300DE00614060000041780000DF2200B1
:102350001080FB004400DE00614060008040780097
:10236000A0B081000342780085417800E4FD0200BE
:102370000000000068FE02000000000010C0B30072
:10238000FED3020000000000D3FE3700A16123004D
:10239000C0CFB30091486000A1612300B0CFB3006B
:1023A00091486000A161230070CFB30091486000A4
:1023B00001DF2200114078000040A1008048780031
:1023C00080612300104078000080FB004300DE00A5
:1023D000610060000004E0000A003200A0612300F8
:1023E0009040780063C060000014A000E3406000EB
:1023F000A061230063C16000C1CFB30010C86000BA
:102400001048710080612300104078000080FB00BC
:102410004200DE00610060000004E0000A003200BB
:10242000A06123009040780063C060000004A00019
:10243000E3406000A061230063C16000C1CFB3002E
:1024400010C86000104871008061230010407800BF
:102450000080FB000000D100610060000004E0008B
:1024600002003200A06123001024A000806123003C
:10247000104078000080FB00610060000004E00074
:1024800002003200A06123001034A000806123000C
:10249000104078000080FB004400DE000000A20035
:1024A000610060000004E0000400320001DF22004F
:1024B000114078000040A0008048780074FE0200BF
:1024C00000000000A06123001080FB004200DE003D
:1024D0006140600080417800A06123009040780056
:1024E00063C0600080427800A06123001080FB0080
:1024F0004300DE00614060000041780000DF220000
:102500001080FB004400DE006140600080407800E5
:10251000A0B081000342780085417800E4FD02000C
:102520000000000068FE02000000000010C0B300C0
:10253000FED302000000000067FE37000040EB0001
:10254000FED302000000000063FE37000080FA00A6
:10255000000006000000FA00409E2A0008D0020099
:10256000000000000080FA00000006000E00FA00E3
:10257000881F780001DF2200114078000040A00091
:102580008048780001DF2200114078000030A1006F
:1025900080487800E1DD220010C0B3008048780058
:1025A000F1DD220080C0B30080487800615D230027
:1025B00020C0B3008048780080C0EB0020C0B3008A
:1025C000C6E3020000000000D822A900D842A900FA
:1025D000D862A80010C0B30056E602000000000058
:1025E000DCFF0700000037005CD4020000000000A0
:1025F00080407800A05D230001487800A05D2300A2
:10260000104078000080FB004400DE00804078002D
:10261000905D230001487800905D23001040780011
:102620000080FB00400798004E009000E40F50002F
:1026300057033200CE009000E48F500011003C00A0
:102640004E019000E10F5100AC003200CE0190002D
:10265000E18F510004003C004E0090000000E000BB
:1026600019003200CD033700CE009000E28F5000F9
:10267000F80032004E019000E30F510008013200D3
:10268000C6033700CE019000E88F51005F0332008F
:102690004E009000E80F500004003C00CE00900077
:1026A000E68F500042033200BC0337004E01900019
:1026B000EA0F510031013200CE019000EF8F51003E
:1026C0008B033200B5033700A05D23001040780073
:1026D0000080FB006101B900520798006307980071
:1026E000D0002000010020005E019000EE0190006B
:1026F000800F5100818F59007C003E005E009000E9
:10270000EE00900000600100A80337000C003700C5
:102710000D00370012003700170037001D0037008A
:102720002300370044003700480037004C003700D2
:1027300052003700580037005E0037006400370051
:1027400084FF0700A8FF370054E4020000000000E7
:1027500010C0B300FED3020000000000A2FF37004B
:1027600094E402000000000010C0B300FED3020099
:10277000000000009CFF37000040EB0056E602001E
:102780000000000010C0B300FED3020000000000F3
:1027900095FF370010C0B30056E6020000000000AD
:1027A00010C0B300FED30200000000008EFF37000F
:1027B000605D230010407800E24F500006003A00B0
:1027C0007AE502000000000080407800805D230070
:1027D0000148780006003700F00F2000B4E4020042
:1027E0000000000080407800805D230001487800F0
:1027F00000DF220010407800684060000004E00024
:1028000008003200805D2300104078000080FB004B
:102810001AF602000000000080407800805D23006E
:1028200001487800805D230010407800FED302004C
:10283000000000006CFF3700C8E502000000000047
:10284000FED302000000000067FF370068E60200C8
:1028500000000000FED302000000000062FF37000D
:1028600010C0B3000CE602000000000010C0B3006E
:10287000FED30200000000005BFF37000040EB00C9
:1028800044E602000000000010C0B300FED30200C6
:102890000000000054FF370010C0B30044E60200FF
:1028A0000000000010C0B300FED3020000000000D2
:1028B0004DFF37000040EB0032E602000000000050
:1028C00010C0B300FED302000000000046FF370036
:1028D00010C0B30032E602000000000010C0B300D8
:1028E000FED30200000000003FFF37000040EB0075
:1028F000FED30200000000003BFF3700A05D230074
:1029000090407800F0C0B30080C06000A05D23005C
:1029100001487800A05D2300104078008040E80066
:10292000A05D23000148780010C0B300FED3020070
:1029300000000000815D23000040EB00804878002B
:102940003D0037005CD402000000000080407800A9
:10295000705D23000148780000DF220010407800FD
:10296000684060000004E00008003200705D230051
:10297000104078000080FB001AF602000000000002
:1029800080407800705D230001487800605D23007E
:1029900010407800E24F500009003A00705D2300BB
:1029A000104078000080FB0026E5020000000000D7
:1029B00010C0B300FED30200000000001900370071
:1029C000705D2300104078000080FB00B4E402003A
:1029D0000000000080407800705D2300014878000E
:1029E00000DF220010407800684060000004E00032
:1029F00008003200705D2300104078000080FB006A
:102A00001AF602000000000080407800705D23008C
:102A100001487800705D230010407800FED302006A
:102A200000000000805D2300104078008040E80036
:102A3000805D230001487800805D2300904078008D
:102A4000A05D23001040780080CF5000BDFF39000A
:102A5000E5FE3700A05D230090407800F0C0B30091
:102A600080C06000A05D230001487800A05D2300C5
:102A7000104078008040E800A05D23000148780005
:102A8000A05D2300104078000CE60200000000006A
:102A900010C0B300FED3020000000000D2FE3700D9
:102AA000A05D230090407800F0C0B30080C06000BB
:102AB000A05D230001487800A05D2300104078004D
:102AC0008040E800A05D23000148780010C0B300FA
:102AD000FED30200000000005CD4020000000000F1
:102AE00080407800905D230001487800815D2300DC
:102AF0000040EB008048780016003700905D23000E
:102B0000104078000004E00004003D0010C0B30055
:102B1000EAE5020000000000030037000040EB007F
:102B2000EAE5020000000000905D230010407800FC
:102B30000040400080407800905D2300014878000C
:102B4000805D2300104078008040E800805D230015
:102B500001487800805D230090407800A05D23004C
:102B60001040780080CF5000E4FF390010C0B3005F
:102B7000FED30200000000009BFE3700A05D230092
:102B8000104078000080FB0030079800400A2000C9
:102B9000BE009000808F50001B003200400A2000D1
:102BA0003E019000800F510005003C00000A20000B
:102BB000BE019000808F51000A003200F001370002
:102BC000500A2000BE009000808F5000B8003200F4
:102BD000700A20003E019000800F51002001320059
:102BE000E70137005CD4020000000000804078005C
:102BF000806423000148780010C0B300FED30200B7
:102C00000000000078FE3700806423001040780048
:102C10000080FB0020079800AE019000E18F51007A
:102C2000040032002E009000E20F50003600320007
:102C30009B0037005CD40200000000000080FB0015
:102C4000A0AE8900A0AE81006300B900A0AE8900EB
:102C50000000EB0070AE890009003700E1AD810093
:102C600070AE8100008440005CD4020000000000CF
:102C7000004C780070AE81000000E80070AE890062
:102C800071AE8100A0AE8100808F5000F3FF39004B
:102C90000000EB0070AE890013003700E1AD810049
:102CA00070AE8100008040000080E8001041780094
:102CB000E1AD810070AE8100008040000000E800BE
:102CC00090417800E1AD810070AE8100008040004D
:102CD00010407800834078009702070070AE8100B2
:102CE0006300400070AE890071AE8100A0AE81002B
:102CF000808F5000E9FF390010C0B300FED30200FE
:102D00000000000038FE37005CD402000000000024
:102D10000080FB00A0AE8900A0AE81004200DD0073
:102D2000A0AE89000000EB0070AE890009003700FA
:102D3000E1AD810070AE8100008440005CD40200EF
:102D400000000000004C780070AE81000000E80038
:102D500070AE890071AE8100A0AE8100808F5000FE
:102D6000F3FF39000000EB0070AE8900440037002B
:102D70000040EB00EAE50200000000000040EB002C
:102D8000EAE50200000000000040EB00EAE5020076
:102D9000000000000040EB00EAE502000000000037
:102DA000E1AD810070AE81000080400010407800ED
:102DB0000080FB0026E5020000000000E1AD81007C
:102DC00070AE8100008040000000E80010407800F4
:102DD0000080FB0026E5020000000000E1AD81005C
:102DE00070AE8100008040000080E8001040780054
:102DF0000080FB0026E5020000000000E1AD81003C
:102E000070AE81000080400063014000E1AD8100B0
:102E100070AE8100008040006300400010407800E8
:102E20006F40600000497800815D23000040EB00A6
:102E3000804878000600370079020700805D230093
:102E4000104078008040E800805D23000148780051
:102E5000E1AD810070AE8100008040006300400061
:102E600090407800805D23001040780080CF5000B3
:102E7000F1FF3E0070AE81006400400070AE89003A
:102E800071AE8100A0AE8100808F5000B8FF390084
:102E900010C0B300FED3020000000000D2FD3700D6
:102EA0000040EB00FED3020000000000CEFD370022
:102EB00080642300104078000080FB001007980019
:102EC0009E009000E18F5000040032001E0190002F
:102ED000E20F510040003200C3FD37005CD4020015
:102EE000000000000080FB00A0AE89005CD402005E
:102EF0000000000080407800905D230001487800C9
:102F00000000EB0070AE89002E003700905D2300BA
:102F100090407800705D230001487800815D2300B7
:102F20000040EB008048780019003700705D2300F6
:102F3000104078000080FB00610060000004E000A9
:102F40000400320010C0B300EAE5020000000000F7
:102F5000030037000040EB00EAE50200000000003B
:102F6000705D2300104078000080FB000000D1005D
:102F700080407800705D230001487800805D230068
:102F8000104078008040E800805D23000148780010
:102F9000805D230010407800E34F5000E3FF3600CF
:102FA0007AE50200000000007AE50200000000005F
:102FB000FED302000000000070AE81000000E800B7
:102FC00070AE890071AE8100A0AE8100808F50008C
:102FD000CEFF390084FD37005CD402000000000001
:102FE0000080FB00A0AE89000000EB0070AE8900FD
:102FF0001600370022C0B30060B92000A10B2000EA
:103000004A0207007D02070022C0B30060BB2D000A
:10301000A10B20004502070022C0B300603D2D0037
:10302000A10B2000410207007402070022C0B30078
:1030300060BB2000A10B20003C0207006F020700CC
:1030400070AE81000000E80070AE890071AE8100B2
:10305000A0AE8100808F5000E6FF390062FD37008E
:103060005CD40200000000000080FB0090AE8900EC
:103070005CD40200000000000080FB0080AE8900EC
:103080008064230010407800E24F500007003A00AF
:1030900090AE81006500B9008000780080AE8100AC
:1030A00000804000A0AE89001C003700806423002F
:1030B00010407800E14F500008003A0090AE8100C7
:1030C000000040008000780080AE81000080400059
:1030D00000004000A0AE890010003700806423008B
:1030E00010407800E34F500008003A0090AE810095
:1030F000000040008000780080AE81000080400029
:1031000000004000A0AE8900040037000040EB0042
:10311000FED302000000000033FD37000000EB008A
:1031200070AE890009003700E1AD810070AE81000A
:10313000008440005CD4020000000000004C7800D5
:1031400070AE81000000E80070AE890071AE8100B1
:10315000A0AE8100808F5000F3FF390080AE810067
:103160000000E0000300320010C0B300FED30200F4
:10317000000000000000EB0070AE89007500370011
:10318000E1AD810070AE8100008040001040780009
:10319000E14F500045003A00806423001040780061
:1031A000E34F500015003A00E1AD810070AE8100A0
:1031B000008040006300400010417800E1AD8100D4
:1031C00070AE8100008040000080E80090417800EF
:1031D000E1AD810070AE8100008040000000E80099
:1031E00010407800834078000E01070070AE810027
:1031F0006400400070AE89005600370080642300F0
:1032000010407800E14F500015003A00E1AD810018
:1032100070AE8100008040006300400010417800E3
:10322000E1AD810070AE8100008040000080E800C8
:1032300090417800E1AD810070AE810000804000D7
:103240000000E80010407800834078003A01070051
:1032500070AE81006400400070AE89003D00370010
:103260008064230010407800E24F500039003A009B
:10327000E1AD810070AE810000804000640040003C
:1032800010417800E1AD810070AE81000080400007
:103290000000E800824078007901070070AE8100EC
:1032A0006500400070AE89002A003700E1AD810062
:1032B00070AE81000080400010407800E24F500066
:1032C00024003A008064230010407800E34F50004F
:1032D0000A003A00E1AD810070AE8100008040003C
:1032E0000000E80010407800B300070070AE8100D5
:1032F0000080E80070AE890016003700806423006B
:1033000010407800E14F50000A003A00E1AD810022
:1033100070AE8100008040000000E800104078009E
:10332000E400070070AE81000080E80070AE890004
:10333000080037008064230010407800E24F5000FE
:1033400004003A00AD01070070AE81000000E80003
:1033500070AE890071AE8100A0AE8100808F5000F8
:1033600087FF390080AE81000000E0009EFC3A003B
:1033700010C0B300FED30200000000009AFC37002A
:103380000040EB00FED302000000000096FC370076
:10339000A05D2300104078000A0002000100000038
:1033A00010C0B300FED30200000000008EFC370006
:1033B000A05D23009040780030C0B30080C0600062
:1033C000A05D230001487800A05D230090407800B4
:1033D000E0DD220001487800E0DD22009040780026
:1033E000605D230010407800C6E30200000000008A
:1033F00010C0B30056E602000000000010C0B30089
:10340000FED302000000000077FC370001DF22003D
:10341000114078000040A10080487800A05D2300A2
:10342000104078000080FB004300DE000000A20096
:10343000610060000004E0000400320001DF2200AF
:10344000114078000040A00080487800615D2300B2
:1034500020C0B30080487800A05D230010407800B1
:103460000080FB004200DE00610060000004E0001C
:1034700003003200615D230030C0B3008048780053
:1034800001DF2200114078000030A1008048780060
:10349000A05D2300104078000080FB000000D100F8
:1034A000610060000004E0000400320001DF22003F
:1034B000114078000030A00080487800E0DD220054
:1034C00090407800605D230010407800C6E3020061
:1034D0000000000010C0B30056E60200000000002B
:1034E00010C0B300FED30200000000003EFC370015
:1034F000A05D2300104078000080FB00000F7800E2
:10350000000F20009E017800808F510005003200DE
:10351000100F20009E007800808F500004003200C1
:103520000900370042FF0200000000002EFC3700B7
:103530001CFF02000000000010C0B300FED3020018
:103540000000000028FC3700A05D23001040780038
:103550000080FB006F00600060AE890060AE8100FB
:103560004800DD0060AE89005CD40200000000006D
:103570008080FB0060AE81000080700060AE89003A
:1035800060AE8100C6FE02000000000010C0B30063
:10359000FED302000000000013FC37000040EB00E7
:1035A000FED30200000000000FFC37004F0478003B
:1035B0000080FA00000006000400FA00204798008E
:1035C0000040EB00004F7800090037002E409000CB
:1035D00061406000EAE50200000000002E4090001B
:1035E0000080FB000000D100204798001E4FE8003B
:1035F00050C0B3009E4F1000F4FF36007AE5020081
:1036000000000000FED30200000000007AE5020086
:1036100000000000FED30200000000000080FA005D
:10362000000006000600FA00204798003147980085
:103630004247980000C8B300AE40900000CF600041
:103640000040EB00104798000B0037002E40900020
:1036500061406000EAE50200000000002E4090009A
:103660000080FB000000D100204798001E40900021
:103670000040E800104798001E409000E54F5000C1
:10368000F2FF36001E04E00008003A003E409000C1
:103690000080FB0026E50200000000004E40900084
:1036A0000080FB0026E50200000000000080FA0018
:1036B000000006000400FA00204798000040EB00DC
:1036C000004F7800110037002E4090000080FB0072
:1036D000610060000004E0000400320010C0B3008C
:1036E000EAE5020000000000030037000040EB00A4
:1036F000EAE50200000000002E4090000080FB0080
:103700000000D100204798001E4FE80030C0B300F1
:103710009E4F1000ECFF36007AE50200000000002A
:103720007AE5020000000000FED302000000000065
:103730000080FA00000006000600FA00204798000A
:1037400031479800424798002E4090000080FB00CF
:103750004600DE00004F78000040EB001047980064
:10376000220037001E409000E34F50000C003A004A
:103770001E04E0000A00320010C0B30044E602005C
:10378000000000001E80FB00B8F5020000000000F1
:103790000040EB0044E6020000000000100037008B
:1037A0002E4090000080FB00610060000004E000FB
:1037B0000400320010C0B300EAE50200000000007F
:1037C000030037000040EB00EAE5020000000000C3
:1037D0002E4090000080FB000000D10020479800A0
:1037E0001E4090000040E800104798001E409000E6
:1037F000E34F5000DBFF36003E4090000080FB00AE
:1038000026E50200000000004E4090000080FB0012
:1038100026E50200000000000080FA00000006001B
:103820000000FA000040EB00EAE5020000000000A2
:103830000040EB00EAE50200000000000040EB0061
:10384000EAE50200000000000040EB00EAE50200AB
:10385000000000000000EB0026E502000000000070
:103860000000EB0026E50200000000000000EB0075
:1038700026E50200000000000080FA0000000600BB
:103880000400FA00000F7800214798000040EB0088
:10389000EAE50200000000000040EB00EAE502005B
:1038A000000000000040EB00EAE50200000000001C
:1038B0000040EB00EAE50200000000001E00780076
:1038C000104078000080FB0026E5020000000000A8
:1038D0001E00E800104078000080FB0026E5020092
:1038E000000000001E80E800104078000080FB000F
:1038F00026E50200000000002E4090006F406000AE
:103900002047980001003700C5FF07002E409000B7
:103910000040E900204798002E409000E14F400011
:10392000F9FF3A000080FA00000006000800FA00E3
:103930001007980021079800624798000040EB00AC
:10394000EAE50200000000000040EB00EAE50200AA
:10395000000000000040EB00EAE50200000000006B
:103960000040EB00EAE50200000000001E009000AD
:103970001AF602000000000026E502000000000028
:103980001E009000AE0090004809DD004800DE00F7
:1039900000007100C808DE001AF6020000000000F6
:1039A00026E50200000000001E009000AE0090001E
:1039B0004008DE00010020001AF6020000000000AE
:1039C00026E50200000000006E4090006F4060009D
:1039D000604798000040EB00004F7800020037007D
:1039E0008FFF07001E4FE8006E4090009E4F1000B2
:1039F000FBFF39000080FA00000006000200FA0018
:103A000010C0B300EAE50200000000000040EB0037
:103A1000EAE50200000000000040EB00EAE50200D9
:103A2000000000000040EB00EAE50200000000009A
:103A30000000EB0026E50200000000007AE502002D
:103A400000000000004F78007AE50200000000004E
:103A5000FED30200000000001E407800FED30200EA
:103A6000000000006EFF07006DFF07000080FA00F5
:103A7000000006000200FA000040EB00004F780052
:103A8000F06F81000000E0001500320000C2B300BA
:103A9000FED3020000000000310020003041200071
:103AA00030F802000000000000C2B300FED30200A4
:103AB00000000000E06F81000000E00004003A0018
:103AC0000040EB00EAE502000000000002003700C1
:103AD0000040EB00410207000000EB00F06F89009E
:103AE000E06F81000000E00004003A007AE5020087
:103AF00000000000004F780002003700730207004A
:103B0000004F780010002000F06F89001E80FB003D
:103B10000080FA00000006000400FA00000F7800A0
:103B2000F06F81000000E0001500320000C2B30019
:103B3000FED30200000000003100200030412000D0
:103B400030F802000000000000C2B300FED3020003
:103B500000000000E06F81000000E00004003A0077
:103B60000040EB00EAE50200000000000200370020
:103B70000040EB00190207000000EB00F06F890025
:103B8000E06F81000000E00008003A001E007800AD
:103B900026E5020000000000C8E502000000000069
:103BA0000080FB00000F7800050037001E00780041
:103BB00031020700F60107000080FB00000F7800CB
:103BC00000C2B300FED30200000000001E00E000AF
:103BD00007003A00310020003041200030F8020098
:103BE0000000000000302000100798000600370099
:103BF000410020006041200030F802000000000079
:103C000000102000100798001E0090000080FA00AD
:103C1000000006000000FA00F06F81000000E000E4
:103C200012003200410020006041200030F8020004
:103C300000000000A0902A0034D002000000000024
:103C4000E06F81000000E00004003A0010C0B30003
:103C5000EAE50200000000000200370010C0B300D7
:103C6000DE0107000000EB00F06F8900E06F8100CB
:103C70000000E00010003A0054E4020000000000E0
:103C80000000E0000D00320091002000C020200064
:103C900030F80200000000005101200050212000F7
:103CA00030F8020000000000A0902A0034D002008A
:103CB000000000000100370091010700D100200042
:103CC000A0412000BAF80200000000000080FA00C5
:103CD000000006000000FA00F06F81000000E00024
:103CE00012003200410020006041200030F8020044
:103CF00000000000A0902A0034D002000000000064
:103D0000E06F81000000E00004003A0010C0B30042
:103D1000EAE50200000000000200370010C0B30016
:103D2000AE0107000000EB00F06F8900E06F81003A
:103D30000000E00003003A0094E4020000000000EC
:103D40000100370080010700C10020007042200000
:103D5000BAF80200000000000080FA00000006002F
:103D60000000FA0001012000404F200030F802005E
:103D700000000000E06F8100A0D2020000000000FF
:103D800000C2B300FED3020000000000E0DD22000C
:103D900010407800A0D202000000000000C2B30072
:103DA000FED3020000000000B0902A0034D00200D0
:103DB000000000000080FA00000006000400FA0085
:103DC0000000EB0010079800B04002000000000067
:103DD000263D02000000000010079800B0400200DD
:103DE00000000000263D020000000000000F7800E7
:103DF0001E0090000000E000070034001E0090004C
:103E0000E20F500004003C001E0090000000E9009A
:103E1000E06F8900020037000000EB00000F78001F
:103E20001E00E00009003400400020009E0F10003A
:103E300006003C001E0078000040E9008040780049
:103E4000E0DD220001487800020037000000EB00AE
:103E5000000F78001E00E0002F003A000000EB0089
:103E6000F09789005102200030432000BAF8020088
:103E7000000000008001EB00220020001100200063
:103E80001000200018430200000000000000E900BC
:103E9000E06F8900E06F81000000E0000F003A0051
:103EA000B103200080452000BAF8020000000000A5
:103EB0008001EB00420020001100200010002000D3
:103EC00018430200000000000040E9008040780034
:103ED000E0DD22000148780012003700C102200016
:103EE000804C200030F80200000000008001EB0050
:103EF00032002000110020001000200018430200B2
:103F0000000000000040E90080407800E0DD220071
:103F1000014878000300370091FF07000000EB0024
:103F2000F06F890000DF2200904078000140A0007F
:103F300001487800E06F81000000E0000A003A00CC
:103F4000D822A800D842A800DA42A900DA22A900A3
:103F5000E0DD22009040780020C0B300C6E30200FC
:103F60000000000001003700730107000080FA0024
:103F7000000006000000FA000000EB00F06F89006E
:103F8000E06F8100E10F500002003A0007E2A90053
:103F900077E2A9000080FA00000006000600FA009F
:103FA000100798001E009000200798002E00900037
:103FB000E20F5000920032002E009000E20F5000FD
:103FC00007003E002E0090000000E0000B003200D1
:103FD0002E009000E10F50000D003200BB003700B2
:103FE0002E009000E30F5000980032002E00900049
:103FF000E40F5000AC003200B4003700B1072000DD
:104000004050200030F8020000000000B3003700EC
:104010008040EB006000200074E602000000000019
:10402000E1022000F0572000BAF802000000000072
:1040300000632300104078000004E00008003A000C
:10404000DAC2BF00644060000004E00010003200EB
:10405000DAC2BF00624060000004E0000C003200E1
:104060000063230010407800E14F500014003A0034
:10407000DBC2BF00624060000004E00010003A00B4
:10408000DBC2BF00644060000004E0000C003A00A6
:1040900091002000C020200030F802000000000045
:1040A000510120005021200030F8020000000000E3
:1040B000A0902A0034D002000000000087003700E2
:1040C0000000EB00000F780046003700E06F810031
:1040D0000000E0000A003A0054E402000000000082
:1040E0001E00780026E5020000000000C8E502007E
:1040F000000000000080FB00100798000600370059
:104100007F0007001E007800DB000700A00007000A
:104110000080FB00100798001E0090000000E000E7
:1041200028003A001E00780012F50200000000008E
:1041300080C2B300FED30200000000001E00780021
:104140000080D10012F50200000000001E0078007F
:104150000000A200610060000004E00004003200E2
:10416000D0902A0008D00200000000000F003700A5
:10417000E06F81000000E00006003A007AE50200EE
:104180000000000010C0B300EAE5020000000000DB
:1041900003003700CD00070010C0B3008F000700F8
:1041A00000912A0008D0020000000000B0902A0010
:1041B00008D002000000000000C2B300FED30200DD
:1041C00000000000E06F81000000E00003003A0002
:1041D00094E4020000000000010037005A000700CC
:1041E0001E0FE800F00F20009E0F1000B7FF3400F4
:1041F000A0902A0034D002000000000037003700F1
:10420000E06F8100E10F500001003A0007E2A900D1
:1042100071002000D05A2000BAF80200000000000F
:10422000F100200000332100BAF802000000000075
:1042300010C0B300D2000700E06F8100E10F500012
:1042400026003A00BC0007002400370030912A0005
:1042500034D00200000000000163230010C0B3004E
:10426000804878000742A9000782A9000000EB00FF
:10427000501088000000EB00601088000702A900C1
:10428000E0DD2200104078008080FB0010632300F6
:10429000614078000080FB002010880007E2A80041
:1042A00077E2A9000D00370000632300104078007A
:1042B000E14F500009003A00B0932A0034D00200C8
:1042C00000000000DB62A90004003700410220006A
:1042D000E01D2000BAF80200000000000080FA0093
:1042E000000006000000FA00B10020005044210048
:1042F000BAF80200000000000080FA00000006008A
:104300000000FA0000632300104078000004E00081
:1043100006003A007602A80076C2BF006140600045
:104320000004E000FCFF3A00050037000602A80088
:1043300006C2BF00614060000004E000FCFF3A00DC
:104340000080FA00000006000000FA00006323006D
:10435000104078000004E00006003A007642A80011
:1043600076C2BF00644060000004E000FCFF3A0039
:10437000050037000642A80006C2BF006440600086
:104380000004E000FCFF3A000080FA000000060094
:104390000200FA0000632300104078000004E000EF
:1043A00006003A0079C2BF000080FB004700DE0033
:1043B0000080FB00000F78000500370009C2BF0035
:1043C0000080FB004700DE000080FB00000F78004B
:1043D0001E0078000080FA00000006000200FA00CB
:1043E000004F780000632300104078000004E000D4
:1043F00010003A009E40780061C06000614060009B
:104400004501DD006127200091407800F0CDB30028
:1044100000C060000240700076E2B7007682A8001B
:1044200076C2BF00704060000004E000FCFF3A006C
:104430000F0037009E40780061C06000614060005E
:104440004501DD006120200091407800F0CDB300EF
:1044500000C060000240700006E2B7000682A800BB
:1044600006C2BF00704060000004E000FCFF3A009C
:104470000080FA00000006000200FA00004F7800F9
:1044800000632300104078000004E00007003A00B9
:104490001E80FB009013880079C2BF000044B20068
:1044A0000004E000FCFF3A00060037001E80FB001D
:1044B0001010880009C2BF000044B2000004E000F0
:1044C000FCFF3A000080FA00000006000400FA0039
:1044D00000632300104078000004E0000A003A0066
:1044E0007662A80076C2BF00684060000004E00069
:1044F000FCFF3A0080138000004F78001E80FB0014
:1045000010079800090037000662A80006C2BF0025
:10451000684060000004E000FCFF3A0000108000EA
:10452000004F78001E80FB00100798001E009000CE
:104530000080FA00000006000000FA007742A9009F
:104540007782A9000000EB00D01388000000EB0088
:10455000E01388007702A900E0DD22001040780017
:104560008080FB0010632300614078000080FB0026
:10457000A013880077E2A8000080FA00000006007F
:104580000A00FA00004F98000040EB002047980016
:104590000040EB00104798000040EB00004F78000F
:1045A0007AD4020000000000D822A800D842A80057
:1045B000DA42A900DA22A9006640A8006660A800D5
:1045C0008660A900DAC2BF000080FB000000D100B5
:1045D00061406000604798006E409000504798002E
:1045E000DAC2BF000080FB004200DE0061406000D4
:1045F000604798006E4090003047980000003700F8
:1046000086C0BF00684060000004E0000F003A0070
:1046100080D402000000000034D40200000000003A
:104620000004E000F6FF32005CD40200000000004D
:10463000004F78006640A9006660A9000E4890000F
:104640000004E00063003A00650037008660A900BE
:10465000DAC2BF000080FB000000D10061406000B2
:1046600060479800DAC2BF000080FB004200DE0015
:1046700061406000404798002E4090000004E00038
:104680002E0032003E4090000004E0002B003A0073
:104690004E4090000004E000280032001E409000D0
:1046A000E74F50000B003E001E40780000404000E5
:1046B000004F78006E4090000004E00001003200DE
:1046C0001E04A0001E4090000040E8001047980023
:1046D0003B0037000E4890000004E0000400320068
:1046E0001E80FB0028D302000000000006003700F7
:1046F000C0C5B30016D40200000000001E407800C0
:1047000016D40200000000006E4090000004E0009B
:1047100004003200D0C2B30016D402000000000032
:1047200003003700B0C2B30016D40200000000003E
:104730000040EB0010479800210037003E409000F9
:104740000004E0001E0032004E4090000004E00033
:104750001B0032005E4090000004E0000B003200BD
:104760006E4090000004E00008003A0010C0B30062
:10477000204798000040EB0010479800B0C5B300F8
:1047800016D40200000000000D0037005E409000CB
:104790000004E0000A003A006E4090000004E000CF
:1047A000070032000040EB00204798000040EB007B
:1047B00010479800D0C5B30016D4020000000000D6
:1047C0006E409000504798004E409000304798004F
:1047D0008BFF3700A0902A0034D0020000000000B8
:1047E0000080FA00000006000000FA0020962A006F
:1047F00008D00200000000000080FA00000006005F
:104800000E00FA00881F7800D822A800D842A8001D
:10481000DA42A900DA22A900D882A90001DF220029
:10482000114078000040A0008048780001DF22009D
:10483000114078000030A1008048780080C0EB0073
:1048400020C0B300C6E3020000000000E6FF07003E
:10485000000037005CD402000000000080407800B7
:10486000A0DF220001487800A0DF2200104078007D
:104870000080FB004400DE008040780090DF2200D2
:104880000148780090DF2200104078000080FB0093
:10489000400798004E009000E10F50001C013200CC
:1048A000CE009000E18F500004003C004E019000CB
:1048B0000200E0000800320053013700CE019000F2
:1048C000E48F5100480132004E009000E60F500086
:1048D000360132004C013700A0DF22001040780082
:1048E0000080FB006101B90052079800630798003F
:1048F000F0002000010020005E019000EE01900019
:10490000800F5100818F5900FD003E005E00900035
:10491000EE009000006001003F0137000E003700FC
:104920000F0037001400370019003700F40037007B
:104930001C0037002200370028003700A200370093
:10494000EF003700EE003700ED003700EC003700D5
:10495000EB003700E4003700A3FF0700BDFF37007E
:1049600054E402000000000010C0B300FED30200B7
:1049700000000000B7FF370094E4020000000000D0
:1049800010C0B300FED3020000000000B1FF3700EA
:104990007AE5020000000000FED3020000000000E3
:1049A000ACFF37000040EB00EAE502000000000029
:1049B00010C0B300FED3020000000000A5FF3700C6
:1049C00010C0B300EAE502000000000010C0B30010
:1049D000FED30200000000009EFF37005CD40200FE
:1049E000000000000080FB00100798001E009000EF
:1049F0004800DD00100798005CD4020000000000B1
:104A00008080FB001E0090000100700010079800DD
:104A10005CD40200000000000080FB00000F780062
:104A20001E0078004800DD00000F78005CD4020012
:104A3000000000000080FB001E0F70009E00900030
:104A400000002100808F500003003E000000210084
:104A50009E0F1000040036000040EB00FED3020061
:104A6000000000007BFF37000000EB0020079800EB
:104A700009003700E1AD81002E0090000084400065
:104A80005CD4020000000000004C78002E00900072
:104A90000000E80020079800AE0090001E00900083
:104AA000808F5000F3FF390054E402000000000042
:104AB0000000EB00200798000E003700E1AD8100F8
:104AC0002E00900000804000104078000080FB0025
:104AD00026E5020000000000C8E50200000000001A
:104AE000E14F5000DCFF32002E0090000000E80093
:104AF00020079800AE0090001E009000808F5000AC
:104B0000EEFF39001E00E900100798000000EB00DE
:104B10002007980014003700E1AD81002E009000BE
:104B2000008440007AE5020000000000004C78009C
:104B3000AE0090001E009000808F500004003100F5
:104B40000040EB00EAE5020000000000030037002F
:104B500010C0B300EAE50200000000002E00900043
:104B60000000E800200798002E0090009E0F5000E3
:104B7000E9FF390094E402000000000010C0B30017
:104B8000FED30200000000000000EB0020079800A8
:104B900009003700E1AD81002E0090000080400048
:104BA00010407800FED30200000000002E009000AC
:104BB0000000E800200798002E0090009E0F500093
:104BC000F4FF390023FF370010C0B300FED302000A
:104BD0000000000022C2BF00614060000004E0004D
:104BE000FCFF32003011800080407800A0DF2200FE
:104BF0000148780010002000000F7800A0DF22009C
:104C0000104078000080FB0030079800BE00900044
:104C1000E28F50001B0032003E019000E20F510075
:104C200007003C00BE0190000300E0000F003200CE
:104C30003E009000E10F50000F00320024003700CA
:104C4000BE009000F08F50001500320000022000DE
:104C50003E019000800F510017003200BE0190000D
:104C6000E38F51000A0032001900370064C30200CC
:104C7000000000001800370014C30200000000000C
:104C800015003700CCC202000000000012003700FF
:104C9000B4C3020000000000000F78000E003700CF
:104CA00001DF2200114078000000A1000010A100E7
:104CB000804878000800370001DF220011407800AA
:104CC0000000A0000010A10080487800020037001A
:104CD0000000EB00100798001E007800FED30200D1
:104CE00000000000DBFE37000040EB0024FE070060
:104CF00010C0B300FED3020000000000D5FE370054
:104D00000040EB00FED3020000000000D1FE37009F
:104D1000A0DF220090407800F0C0B30080C06000A7
:104D2000A0DF220001487800A0DF220010407800B8
:104D30008040E800A0DF22000148780010C0B300E6
:104D4000FED302000000000081DF22000040EB00E3
:104D5000804878000E0037005CD40200000000009C
:104D60000080FB0026E5020000000000C8E502000C
:104D700000000000FED302000000000080DF2200DF
:104D8000104078008040E80080DF22000148780071
:104D900080DF220090407800A0DF220010407800E1
:104DA00080CF5000ECFF3900AAFE3700A0DF2200C0
:104DB0009040780030C0B30080C06000A0DF2200C7
:104DC00001487800A0DF22009040780020C0B300A6
:104DD000C6E302000000000010C0B300FED30200D2
:104DE000000000009BFE3700A0DF2200104078008A
:104DF0000A0002000100000010C0B300FED3020050
:104E00000000000093FE37000040EB00FED30200DC
:104E1000000000008FFE37004F0478000080FA0089
:104E2000000006000800FA00000F78001107980043
:104E300022079800330798001E00780040A58900DB
:104E40001E00900050A589002E00900060A58900EA
:104E50003E00900070A589000000EB0080A589004D
:104E60000000EB0090A589000000EB00A0A58900E0
:104E70008000EB000000EB00D40307008000EB0093
:104E80000000EB00DC030700380007000000EB0027
:104E9000302588000000EB004025880000E022005B
:104EA0004800DE00C024880000082000302488006C
:104EB0008804A80094A4A9000080FA00000006005D
:104EC0000000FA00010037009404A80094C4BF0059
:104ED000614060000004E000FBFF3200A14F2300AE
:104EE00010C0B3008048780094C4BF000044B200F2
:104EF0000004E000FCFF3A00A14F230040C0B300D3
:104F0000804878000080FA00000006000000FA00E7
:104F1000F00F2000702488000080FA0000000600D6
:104F20000000FA0080002000502488000000EB0000
:104F3000C0A78900A14F230040C0B300804878007B
:104F4000B14F23000040EB00804878008AC4BF00C6
:104F5000684060000004E000F2FF3A000300070030
:104F600094A4A9000080FA00000006000200FA00E4
:104F70000000EB0080A589000000EB0090A58900EF
:104F80000000EB00A0A589000000EB00B024880021
:104F90009424A8009424A900F00F20007024880015
:104FA0000000EB00000F7800150037001E007800AD
:104FB0004200DD008080E800604B230080804000DC
:104FC0000000EB00800878001E007800C200DD00C1
:104FD000604B2300808040000000EB0080087800D8
:104FE0001E0078000000400080007800A04A2000E9
:104FF000808040000000EB00800878001E0FE80071
:105000001E007800EF0F5000E8FF36000000EB00B4
:10501000000F7800070037001E007800C200DD0096
:1050200000E02200808040000040EB0090409800AB
:105030001E0FE8001E007800E50F5000F6FF360056
:10504000D0002000502588000000EB00B0A78900A8
:10505000A14F23000040EB00804878000000EB00E7
:10506000C0A78900B14F23000040EB0080487800C2
:1050700001E0220080C0B3008048780080E1220077
:105080001070890011E0220080C8B30080487800C9
:1050900041E022000040EB008048780000E222005E
:1050A0003070890051E0220080C4B300804878004D
:1050B0000080FA00000006000000FA008AC4BF0069
:1050C000704060000004E00004003200CCFC0200EC
:1050D0000000000000012000502488008AC4BF00A6
:1050E000614060000004E000030032008CFF070014
:1050F00010002000502488008AC4BF006240600075
:105100000004E00004003200F00F2000702488004A
:1051100020002000502488008AC4BF0001C8B300CA
:10512000014060000004E00002003200000820009E
:10513000502488008AC4BF00644060000004E0007E
:105140000700320080A581000000E000020032006C
:1051500080A581000000010040002000502488004C
:105160008AC4BF00684060000004E000080032000C
:10517000902480004400DE006F0060000000E0002A
:1051800001003A000400070080002000502488003D
:105190000080FA00000006000200FA00015023001F
:1051A0000040EB0080487800902480008040780028
:1051B000204A230001487800204A2300104078004C
:1051C0000080FB004300DE000080FB004200DD00A9
:1051D0008000780000E022000080400020A58900C7
:1051E000204A2300104078000034A0000080FB001B
:1051F0004300DE000080FB004200DD0080007800FC
:1052000000E022000080400030A5890020A5810038
:10521000104090008080FB00C00320008080600070
:10522000010F7800400220009E007800808F50001F
:105230000C003200400320009E007800808F500058
:10524000040032001E007800E40F5000030032001A
:10525000050037000600070003003700AD02070015
:1052600001003700910207000080FA0000000600EC
:105270000800FA0031A5810080C0B300904098007A
:1052800094A4A90020A5810010009000104078008F
:105290008080FB00000620008080600031079800BD
:1052A00000022000BE009000808F500023003200DA
:1052B00000042000BE009000808F500025003200C6
:1052C0003E0090000000E00001003200270037009F
:1052D00020A5810010009000104078000080FB00A5
:1052E0006300600020079800AE009000E18F50003E
:1052F0000A0032002E009000E20F50000A00320037
:10530000AE0090000100E00001003200090037000B
:1053100020A58100360007001500370020A5810078
:105320007B0107001200370020A58100B9010700AA
:105330000F003700C90207000D00370090A581005B
:105340000000E0000A00320090A58100000001008A
:1053500007003700A0A581000000E0000400320033
:10536000A0A581000000010001003700BB0207007A
:1053700021A5810080C0B3008048780020A581006D
:105380001007980020A581001000900010407800C0
:105390000004E0000F00350020A5810010009000FF
:1053A00066004000104078000004E00006003A006B
:1053B00020A5810010009000670040001040780098
:1053C0000004E0000300320081CCB300014F7800FC
:1053D0000200370080C8B300004F78001E407800FC
:1053E0009E009000904098000080FA0000000600A7
:1053F0000A00FA00200798002E009000900090000C
:10540000110798001E0090000000E800104078008E
:105410000080FB00400798004E009000E50F500010
:105420003F003200CE009000E58F50000A003C00A3
:105430004E009000E10F50001E003200CE009000A0
:10544000E38F5000290032004E0090000000E00081
:105450000B0032002B013700CE009000E88F500087
:10546000060132004E009000E90F50000A013200A0
:10547000CE009000E68F500040003200210137003E
:1054800030A5810090009000B0A78100804878008E
:1054900030A58100100090008000E800B0A78100D6
:1054A0004800DE0080487800200020005E020700EF
:1054B000150137001E0090000080E80010407800C1
:1054C000E14F500007003A00B0A78100D1FF2F0044
:1054D00001006000B0A789000000EB005202070045
:1054E000090137005D020700070137001E00900028
:1054F0000080E80010407800E14F500006003A00BC
:10550000B0A781000010A000B0A789000000EB0048
:1055100045020700FC00370050020700FA00370080
:105520001E00900063004000104078000004E0007E
:1055300010003A001E0090000080E8001040780043
:105540000004E0000B0035001E0090000080E80021
:1055500090407800B04F23000148780061F42A00A1
:105560000000EB00190207000000EB002E0207000C
:10557000E500370039020700E30037001E00900005
:1055800063004000104078000080FB003007980066
:105590003E009000E20F50001F003200BE0090005D
:1055A000E38F5000720032003E009000E10F500087
:1055B00001003200A300370040A58100E0A7890068
:1055C00040A58100104078000080FB00F0A7890012
:1055D0001E00900067004000104078000004E000CA
:1055E0009B003A001E00900066004000904078004A
:1055F000E0A781001040780080CF50009400310077
:105600001E00900066004000104078000080FB0003
:10561000F0A789008E0037001E0090000080E8008F
:105620009040780040A58100710040001040780053
:1056300080CF5000040039000150230010C0B30097
:10564000804878008200370050A58100E0A78900DB
:10565000E0A781000080E800104078008080FB0017
:10566000E0A7810063004000104078000080FB004C
:105670004800DD0000804000F0A789000000EB003A
:10568000000F780010003700E1A78100F0A781002B
:1056900000804000E0A78900E0A781000080E800CA
:1056A000104078008080FB00E0A78100630040008C
:1056B000104078000080FB004800DD0000804000C2
:1056C000F0A789001E0FE8001E0090000080E8008F
:1056D000104078000080FB009E0F5000EAFF3C0065
:1056E0001E0090006700400090407800E0A7810015
:1056F000630040001040780080CF50001000390057
:105700001E0090006700400090407800E0A78100F4
:10571000630040001040780080CF50004C003A00F9
:105720001E0090006600400090407800E0A78100D5
:105730000080E8001040780080CF50004400310025
:105740001E00900066004000104078008080FB0042
:105750001E00900067004000104078000080FB00B1
:105760004800DD0000804000F0A7890038003700C5
:105770001E0090000080E800104078008080FB0050
:1057800070A58100808F5000040035000150230077
:1057900010C0B300804878002D00370060A581005C
:1057A000E0A78900E0A78100104078000080FB009E
:1057B000F0A789000000EB00000F78000900370017
:1057C000E1A78100F0A7810000804000E0A78900E8
:1057D000E0A78100104078000080FB00F0A789005E
:1057E0001E0FE8001E0090000080E80010407800C6
:1057F0000080FB009E0F5000F1FF3C001E00900057
:1058000067004000104078000004E00010003A00FB
:105810001E0090006600400090407800E0A78100E4
:105820001040780080CF5000090031001E00900029
